:10000000F8FF022099010000B1B5010069B50100B7
:1000100069B5010069B5010069B5010069B5010064
:1000200069B5010069B5010069B50100B1B501000C
:10003000B1B5010069B5010085DF010089E001006B
:10004000B1B50100B1B50100B1B50100B1B5010014
:10005000B1B50100B1B50100B1B50100B1B5010004
:10006000B1B50100B1B50100B1B50100B1B50100F4
:10007000B1B50100B1B50100B1B50100B1B50100E4
:10008000B1B50100B1B50100B1B50100B1B50100D4
:10009000B1B50100B1B50100B1B50100B1B50100C4
:1000A000B1B50100B1B50100B1B50100B1B50100B4
:1000B000B1B50100B1B50100B1B501000DC001003D
:1000C000B1B501007DC70100B1B5010011CD01003E
:1000D000B1B5010009EE0100B1B50100B1B50100F3
:1000E000B1B50100B1B50100D5AD0100B1B5010058
:1000F000B1B50100B1B50100B1B50100B1B5010064
:10010000F9E401000DE5010021E5010035E50100FC
:10011000B1B501009DCF0100B1B50100B1B501003D
:10012000B1B50100B1B50100B1B50100B1B5010033
:10013000B1B50100B1B50100B1B50100B1B5010023
:10014000B1B50100B1B5010001EF0100B1B5010089
:10015000F9EF0100B1B50100B1B50100B1B5010081
:10016000B1B50100B1B50100B1B50100B1B50100F3
:10017000B1B50100B1B50100B1B50100B1B50100E3
:10018000B1B50100B1B50100B1B50100B1B50100D3
:10019000B1B50100B1B50100584B4CF2205210B579
:1001A0001A804DF628121A8000BF00BF1BF004FA17
:1001B000534B4FF030621A60524A9A60524ADA60EA
:1001C000524B4FF470021A60514A136813F4807353
:1001D00004D150490B604FF4A85313604E4B1A786A
:1001E000110703D51A7842F008021A704B4B4C499C
:1001F0002A221A704B4A4C4B8B4204D252F8040FFD
:1002000043F8040BF8E7494B494900228B4202D2DC
:1002100043F8042BFAE74749474A002352F82300E2
:1002200041F823000133662BF8D1444B444A802126
:1002300003F8011B9342FBD1424B3E4A1A60424BEA
:100240008A221A70A3F5805324225A70A0221A70B1
:100250009A799207FCD59A79D406FCD43B4A9379D3
:1002600003F00C03082B394BF9D103221A714622F3
:100270005A719A799006FCD5344A9179334B4906E4
:10028000FBD5334A4FF08271116009215160202261
:100290001A709A7902F00C020C2AFAD12D4B2E4AD0
:1002A0001A602E4B2E4A1A6000225A60072243F829
:1002B000042C2C4AC3F80C2D62B61BF097FA154B90
:1002C0001B68DA0705D528481BF016FA274B284A81
:1002D0001A60284B1B785B0609D5244C244B2268F6
:1002E0009A4204D120481BF007FA0023236021F032
:1002F00075F81BF067F91EF027F9FEE70E200540A0
:1003000030800440823F04000100002B88ED00E0B3
:1003100010D0034014D0034002D0074000E0074053
:100320004812FF1F0C820200F806FF1F4812FF1F31
:10033000F41FFF1F0002FF1F0000000000E400E0A8
:1003400056E400E008ED00E00050064000400640A2
:100350004480044004800440C010050014E000E024
:10036000BFD401000000202083C15F601CE0034077
:10037000A5C3945A00F00740FFFFFFFFFFFFFFFFF8
:10038000FFFFFFFFFFFFFFFFFFFFFFFFFFFFFFFF7D
:10039000FFFFFFFFFFFFFFFFFFFFFFFFFFFFFFFF6D
:1003A000FFFFFFFFFFFFFFFFFFFFFFFFFFFFFFFF5D
:1003B000FFFFFFFFFFFFFFFFFFFFFFFFFFFFFFFF4D
:1003C000FFFFFFFFFFFFFFFFFFFFFFFFFFFFFFFF3D
:1003D000FFFFFFFFFFFFFFFFFFFFFFFFFFFFFFFF2D
:1003E000FFFFFFFFFFFFFFFFFFFFFFFFFFFFFFFF1D
:1003F000FFFFFFFFFFFFFFFFFFFFFFFFFFFFFFFF0D
:10040000FFFFFFFFFFFFFFFFFFFFFFFFDEF9FFFF23
:1004100010B5054C237833B9044B13B10448AFF33E
:1004200000800123237010BD4812FF1F0000000050
:1004300008820200084B10B51BB108490848AFF309
:1004400000800848036803B910BD074B002BFBD0A0
:10045000BDE81040184700BF000000004C12FF1F0D
:10046000088202004812FF1F0000000000690B69AB
:100470009842D4BF00200120704700BF80698B697B
:100480000028B8BF4042002BB8BF5B429842D4BF9F
:1004900000200120704700BFF0B586460120DEF83D
:1004A0005870DEF83030BA6A106079683A680A44E9
:1004B0007A600EF1300493B15A69002A08DB9A6A17
:1004C00010605E6819683D695A6931445960521B71
:1004D00019690A445A6154F8043F002BECD1DEF844
:1004E0002430144ADEF81840DEF86C000021116058
:1004F000DB00516803F1804303F5603321440D2490
:1005000019611460DA68502122F08002DA60D96043
:1005100000B1F0BD7A68FB689A4200D0F0BDDEF809
:100520005C3001228EF82820002BF7D0BDE8F04087
:10053000184700BF00800340C36A00F12C0233B1AA
:100540000120D96A52F8043F0860002BF9D17047A6
:100550000C4BD3F8902072B9596A1A6AD3ED0A7A13
:1005600002FB01F207EE102A60EE277AB8EE477A16
:1005700087EE870A7047D3F89810D3F89420D3ED0C
:10058000277AEDE7DC17FF1F836D012280F89020AA
:100590005B6872B6DFED0B6AD0ED207A90ED1F7AC2
:1005A00067EEA67AF4EEC77AC0ED1E7AD0ED227A15
:1005B000F1EE10FAD8BFF1EE677AC0ED237A62B699
:1005C000704700BF00000000036A8B4210B523D0C3
:1005D000C369994200D010BD8369002BFBD072B66D
:1005E000194AC369846900211160DB00516803F175
:1005F000804303F5603321440D2419611460DA68E7
:10060000502122F08002DA60D96062B60069036886
:10061000BDE810405B6818470446006903689B68A2
:10062000984794F82430002BD5D004F108001DF031
:1006300041FF0023E06963601AF0B4FB206ABDE863
:1006400010401AF0AFBB00BF008003402DE9F0411D
:100650008568002D31D0816D836F04464868D4F8D9
:10066000AC101B1A002BB8BF5B428B423ADBD4F8AC
:10067000B0108B422A4608DBE16F8B4265DB936842
:1006800023F002039360BDE8F081D4F888100029BC
:10069000F5D02B683B4A93421ED96A683A48B0FBB2
:1006A000F1F19B1A99420AD3CB1A002401200322AC
:1006B000AC60E8602B60AA602960BDE8F0816069E9
:1006C0000368002601240322AE601B68EC602960E9
:1006D000AA60BDE8F04118472B4BB3FBF1F129604C
:1006E000BDE8F081D4E92401D4F8A82002FB03F38B
:1006F000C61841F100073046394620F057FC07EE96
:10070000900AB1EEE70AB4EE400AF1EE10FA2ED1EB
:10071000FDEEC07A2A4617EE903A17EE901ADBB13A
:10072000002DB6D11949184D0E68B5FBF3F51EB171
:1007300002210120B047A26800200121032390601C
:10074000D16015609360BDE8F081CB1AD4F8A82081
:10075000D4E92601013BC9E7002D90D10B4B1B6862
:10076000002B8CD0022101209847A26887E73946E8
:10077000304620F01BFC00EE100A1EF04DFEA5686E
:10078000C6E700BF7FA90300008793034C1BFF1F30
:10079000F8B50446D0ED1F7A94ED1E7A806DF4EE24
:1007A000477AF1EE10FA436838D1FDEEC77A17EEBA
:1007B000905A94F890300BB1002D76D08368AB42FC
:1007C0002BD0002D0368B4BF4FF0FF3201229A42B4
:1007D00015D004F12801012608E013685B42012BC3
:1007E00013600BBF126B536B13601E6051F8042F24
:1007F000002AF2D1636F03EB8303DB003FD185EA6C
:10080000E572A2EBE572A368FAB9002B7AD09A6878
:1008100022F002029A608560F8BDF8BDD4ED236A2B
:10082000F5EEC06A77EEA67AF1EE10FAB4EEE77A4A
:100830002FDDF1EE10FAD8BFF0EE477ABDEEE77A81
:10084000C4ED1F7A17EE105AB3E7002B47D0196892
:10085000314EB14223D95E68304FB7FBF2F2891BAB
:100860008A4232D26069002601689E600127032611
:10087000DF6009681A609E608847A06DCBE7013B86
:10088000FDD185EAE572A2EBE572A368002ABCD02F
:10089000DBE7F1EE10FA58BFF0EE477ACEE71F49DA
:1008A000B1FBF2F21A608560F8BD04F10C001DF096
:1008B00001FE206AA5601AF075FA606A1AF072FAF1
:1008C000A36D9D6084F89050F8BD511A0027012651
:1008D00003249F60DE6019609C601A609BE71049EA
:1008E0000E4E0F68B6FBF2F627B101200221B84781
:1008F000A368A06D0024012103229C60D9601E60C2
:100900009A6088E7064B1B68002B80D001200221EB
:100910009847A368A06D7AE77FA903000087930337
:100920004C1BFF1F70B5044608460D4621F0E8FD3C
:1009300023680246294620465B68BDE87040184798
:1009400038B5044608460D4621F0DAFD2368024614
:1009500029465B6820469847054620461DF03CFE28
:10096000284438BD38B505461DF086FE04462846A5
:100970001DF032FE204438BD38B505461DF07CFE22
:10098000044628461DF028FE204438BD38B50A220A
:10099000002305461DF030FE044628461DF01CFECF
:1009A000204438BD38B5C9B205461DF06DFE044679
:1009B00028461DF011FE204438BD00BF10B50921A6
:1009C0002C481DF079F92C481DF006FEFE212B481D
:1009D00017F0E4FF00282FD10A21284817F0DEFF86
:1009E00098B91821254817F0D9FF00283AD10F21CE
:1009F000224817F0D3FF50BB09212048204C17F0A4
:100A0000CDFF002832D1206009E01D4C1D480A238B
:100A1000194623601DF050F917481DF0DDFD0C212B
:100A200019481DF049F9216813481DF025FE1248A8
:100A3000BDE810401DF0D0BD114C14480123092120
:100A400023601DF039F90C481DF0C6FDE7E70C4C9A
:100A50000F480F230A2123601DF02EF906481DF0D0
:100A6000BBFDDCE7064C0B481823F3E70A480923D3
:100A7000CEE700BFC84B0200E407FF1FD018FF1FDE
:100A80009C16FF1FE04B0200104C0200D44B0200EA
:100A9000F84B0200EC4B0200044C020010B584B08D
:100AA000C9B9344A344B11680191019C1968136823
:100AB0000093009B1B1B9942F9D8032809D8DFE853
:100AC00000F02E3602262D4B112093F877101AF0E5
:100AD00025FE04B010BD03280BD8DFE800F002307B
:100AE0003942264B93F875100E2081F001011AF05F
:100AF00015FE204A204B116803910398196813686A
:100B00000293029B1B1A9942F9D804B010BD1B4BEB
:100B1000042093F874101AF001FE04B010BD174BB6
:100B20000E2093F875101AF0F9FD04B010BD134BA8
:100B3000162093F876101AF0F1FD04B010BD0F4B9B
:100B400093F87610162081F001011AF0E7FDD0E746
:100B50000A4B93F87710112081F001011AF0DEFDA5
:100B6000C7E7064B93F87410042081F001011AF0D6
:100B7000D5FDBEE7841BFF1F2007FF1FDC17FF1FEB
:100B8000F0B52DED028B85B0044601AE0DF10F07D7
:100B90000FE0FF2D58D001A8357021F0B1FC0146BF
:100BA00001A81DF089F82C481DF016FD0136BE4243
:100BB00029D0236820465B6998470021C5B22748A1
:100BC0001DF07AF824481DF007FD332124481DF05C
:100BD00073F828461DF0F4F8022122481DF06CF845
:100BE00029461D481DF048FD1B481DF0F5FC042D4D
:100BF000CFD119211C481DF05FF8013616481DF0B1
:100C0000EBFCBE42D5D101A820F0D8FB0721174844
:100C1000B0EE408AF0EE608A1DF04EF8B0EE480A61
:100C2000F0EE680A04210C481DF02EFD0A481DF064
:100C3000D3FCB0EE480AF0EE680A05B0BDEC028BBA
:100C4000F0BD23685B699847236820461B69984775
:100C500000282046F5DCA9E7E407FF1FB463020083
:100C6000204C0200544C0200584C0200744C02000C
:100C700003280FD8DFE800F00B0805020A48FFF749
:100C80007FBF0A48FFF77CBF0948FFF779BF0948D3
:100C9000FFF776BF9FED020B704700BFAFF30080F8
:100CA000000000000000F0BFC407FF1FB407FF1FD3
:100CB000A407FF1FE407FF1F012828D0022813D034
:100CC00010B19FED140A7047134A1169D368D2ED31
:100CD000056A03FB01F307EE103A60EE267AB8EEE0
:100CE000477A87EE870A70470B4B5A6B012AE8D880
:100CF000D96B9A6BD3ED116A02FB01F207EE102A51
:100D000060EE267AB8EE477A87EE870A7047FFF7DB
:100D10001FBC00BF00000000DC17FF1F38B5434DAB
:100D20004348EA6BAB6B95ED107AD5ED127A414CE6
:100D300003FB02F32DED048B08EE103AB8EE488A5F
:100D4000DFED3D8A28EE078A0D2167EEA88AF0EED6
:100D5000409A1CF0B1FF18EE100A1FF0BBFC41ECEA
:100D6000100B022120461DF08FFC20461DF034FCA4
:100D7000112132481CF0A0FF286C1FF0ABFC41ECA5
:100D8000100B022120461DF07FFC20461DF024FCA4
:100D90000F212B481CF090FF89EEA89A18EE900ABC
:100DA0001FF098FC41EC100B022120461DF06CFC5A
:100DB00020461DF011FC102122481CF07DFF19EE89
:100DC000900A1FF087FC41EC100B022120461DF019
:100DD0005BFC20461DF000FC07211B481CF06CFF4B
:100DE00019EE100A1FF076FC41EC100B0221204690
:100DF0001DF04AFC28EE098A20461DF0EDFB082173
:100E000012481CF059FF18EE100A1FF063FC41EC69
:100E1000100B022120461DF037FC20461DF0DCFBA4
:100E2000B0EE480ABDEC048B38BD00BFDC17FF1FD5
:100E3000AC4C0200E407FF1FDB0FC940BC4C0200B2
:100E4000D04C0200E04C0200F44C0200FC4C0200CA
:100E5000144A1548D2ED117AD16B936B80EE270AB4
:100E600010B503FB01F31921104C2DED028B08EE98
:100E7000103AB8EE488A28EE008A1CF01DFF18EEE2
:100E8000100A1FF027FC41EC100B022120461DF038
:100E9000FBFB20461DF0A0FBB0EE480ABDEC028B28
:100EA00010BD00BFDC17FF1F084D0200E407FF1F45
:100EB0000128F0EE407A1CD0022813D010B19FED2B
:100EC000160A7047154AD2ED056A1169D36887EE94
:100ED000A67A03FB01F300EE103AB8EE400A20EECA
:100EE000070A70470D4B5B6B9BB1012BE7D1FFF7F6
:100EF000AFBF0A4AD2F8903023B9D2ED0A6A516ADC
:100F0000136AE4E7D2ED276AD2F89810D2F8943049
:100F1000DDE7FFF703BF00BF00000000DC17FF1F85
:100F200038B52F4D2F4C95ED007AD4ED007AB5EE03
:100F3000C07AF1EE10FA48BFB1EE477AF5EEC07A0A
:100F400048BF85ED007AF1EE10FA44BFF1EE677A02
:100F5000C4ED007A67EEA77A2DED048BE7EE077AF1
:100F600008EE100A17EE900A08EE901A1FF0B2FB76
:100F700041EC100B1EF090F951EC100B1FF0F6FE37
:100F800094ED006AD5ED006A07EE900A87EE867A46
:100F900087EEA69AF8EEE88AB8EEC88A67EE287A55
:100FA00017EE900A1FF096FB41EC100B1EF0D4F8E0
:100FB00051EC100B1FF0DAFE68EE097A206017EE94
:100FC000900A1FF087FB41EC100B1EF0C5F851ECA6
:100FD000100B1FF0CBFEBDEC048B286038BD00BFAA
:100FE000E013FF1F2C16FF1FF8B51D212DED028BFE
:100FF000914D924C924E08EE100A92481CF05CFE05
:1010000091481DF0E9FA95E8090003FB00F307EEAB
:10101000903A95ED027AD4ED036A8C4A8C49F8EE49
:10102000677AB8EEC88A67EE877A002387EEA67AD9
:101030000B601360C7EE087A17EE900A1FF04AFBA8
:1010400041EC100B1EF088F851EC100B1FF046FE1F
:1010500027683060012F00F0B98065D3022F41D09E
:101060007C4F7D4815211CF027FE316876481DF025
:1010700003FB75481DF0B0FA242178481CF01CFED3
:10108000E0681FF027FB41EC100B02216E481DF0B9
:10109000FBFA6D481DF0A0FA292171481CF00CFEE6
:1010A000A0691FF017FB41EC100B022166481DF0F0
:1010B000EBFA65481DF090FA14216A481CF0FCFD1B
:1010C000396861481DF0D8FA5F481DF085FA14218F
:1010D00065481CF0F1FDBDEC028B5B48BDE8F840B3
:1010E0001DF07ABA2B21614894ED068A1CF0E4FDCC
:1010F000A0691FF0EFFA41EC100B394652481DF081
:10110000C3FA51481DF068FA6B6B002B00F0898020
:10111000012BA5D1B0EE480AFFF79AFE4D4FBDEE68
:10112000C00A87ED000A9CE794ED067AD5ED057AB2
:10113000484F87EE278AD5ED047A95ED037AF8EECD
:10114000677AB8EE477A67EE887A67EE877A17EEA5
:10115000900A1FF0BFFA41EC100B1DF0FDFF51EC9F
:10116000100B1FF0BBFD1821386041481CF0A4FD96
:10117000A0691FF0AFFA41EC100B022132481DF0BC
:1011800083FA31481DF028FA24213A481CF094FDD6
:1011900068691FF09FFA41EC100B02212A481DF0EC
:1011A00073FA29481DF018FA112133481CF084FD08
:1011B00018EE100A1FF08EFA41EC100B02212248A3
:1011C0001DF062FA20481DF007FA4AE7D5F8903082
:1011D000D4ED065AF3B195ED276A95ED267AD5ED53
:1011E000257A1C4FC5EE866AB8EE477AF8EE677A24
:1011F00026EE877A67EE277A17EE900A1FF06AFAD2
:1012000041EC100B1DF0A8FF51EC100B1FF066FD18
:10121000386026E795ED0A6A95ED097AD5ED087AEA
:10122000DFE7B0EE480AFFF779FD0A4FBDEEC00ACE
:1012300087ED000A15E700BFDC17FF1FF813FF1F3B
:101240006014FF1F244D0200E407FF1F7412FF1FEC
:101250004017FF1FCC12FF1FC84D0200E04D0200D7
:10126000084E0200344E0200F87002009C4D02004D
:10127000444D0200604D0200884D02000C4B1B687B
:10128000032B13D8DFE803F00E0A060201460948D3
:101290001DF07CB9014608481DF078B901460748A1
:1012A0001DF074B9014606481DF070B9704700BFC3
:1012B0001007FF1FC407FF1FB407FF1FA407FF1F6E
:1012C000E407FF1F70B584B06649674C674D6846F8
:1012D0001DF04EFB00216846FFF7D0FF68461DF069
:1012E00007FB634968461DF043FB00216846FFF792
:1012F000C5FF68461DF0FCFA5E4968461DF038FBE4
:1013000000216846FFF7BAFF68461DF0F1FA584918
:1013100068461DF02DFB00216846FFF7AFFF6846C9
:101320001DF0E6FA544968461DF022FB002168468C
:10133000FFF7A4FF68461DF0DBFA4D4968461DF033
:1013400017FB00216846FFF799FF68461DF0D0FAA9
:101350004A4968461DF00CFB00216846FFF78EFFE6
:1013600068461DF0C5FA424968461DF001FB0021A0
:101370006846FFF783FF68461DF0BAFA404A2168C5
:101380001668536892ED027ADFED3E6A2D683E489A
:1013900003FB06F307EE903A06EE101AF8EE677AB2
:1013A000B8EEC66A67EE877A012D86EE277A374E49
:1013B00067EE267AC0ED007A4DD031D3022D0ED1E2
:1013C000D6ED007A2846B8EEE70AFFF775FC304BF9
:1013D0000021284683ED000AFFF760FB21682D4AB3
:1013E0002D4B1160002508212C481D601CF064FC69
:1013F00021682B481DF040F929481DF0EDF8052122
:1014000028481CF059FC316825481DF035F924485E
:101410001DF0E2F829460320FFF740FB04B070BD41
:10142000D6ED007A1169D36892ED057A184AF8EE84
:10143000E77A03FB01F327EE877A07EE903AF8EE9E
:10144000677A0021C7EE276A0846C2ED006AFFF7F7
:1014500025FB2168C3E7D6ED007AB8EEE70AFFF76F
:1014600077F8B4E74C4E02004017FF1FF813FF1F38
:10147000604E0200644E0200784E02008C4E020064
:10148000DC17FF1F0000B4433016FF1F7412FF1F4C
:101490009015FF1F6815FF1FB812FF1F9C65020003
:1014A000E407FF1F1062020010B5F0EE407A002141
:1014B000F2EE046ABDEEE77AB8EEC77AB4EE677A68
:1014C000F1EE10FA04D00131062967EEA67AF1D1C7
:1014D0001E4B1B68032B37D8DFE803F0291C0F02D3
:1014E00010EE100ACCB21FF0F5F841EC100B2146BB
:1014F0001748BDE810401DF0C7B810EE100ACCB276
:101500001FF0E8F841EC100B21461248BDE81040EE
:101510001DF0BAB810EE100ACCB21FF0DBF841ECA7
:10152000100B21460C48BDE810401DF0ADB810EE80
:10153000100ACCB21FF0CEF841EC100B2146074840
:10154000BDE810401DF0A0B810BD00BF1007FF1F80
:10155000C407FF1FB407FF1FA407FF1FE407FF1FF7
:10156000084B1B68032B0BD8DFE803F008060402C6
:101570001BF022BB1AF0A6BF1AF03ABC1CF020BC2C
:10158000704700BF1007FF1F2DE9F041DFF85080C2
:10159000104F114E114D0446014640461CF0F6FF17
:1015A00040461DF019F8214638461CF0EFFF38463A
:1015B0001DF012F8214630461CF0E8FF30461DF0C1
:1015C0000BF8214628461CF0E1FF2846BDE8F04113
:1015D0001DF002B8A407FF1FB407FF1FC407FF1FB9
:1015E000E407FF1F2DE9F04FB24CA3B001210D20FD
:1015F0001AF0A8F823680893089A23680793079BB2
:10160000AC4D9B1A0E2BF8D9AB4BAC491E681EA8EB
:101610001DF0AEF900211EA8FFF730FE1EA81DF038
:1016200067F90A2231461EA81DF0D4F91EA8FFF75B
:10163000ABFF1EA81DF05CF94FF482701AF0BCF9E4
:101640000C219F481AF0DEFB03219E481AF0DAFBBA
:101650002B680693069A23680593059B954D9B1A64
:10166000312BF8D90C2196481AF0CCFB0321954870
:101670001AF0C8FB2B680493049A23680393039B16
:101680008C4D9B1A312BF8D907218F481AF0BAFBE1
:1016900003218C481AF0B6FB2B680293029A236848
:1016A0000193019B9B1A312BF9D91AF02DFC0028CC
:1016B000864D0CDD01230C2185482B601CF0FCFAC3
:1016C000296884481CF0D8FF82481CF085FF4FF43D
:1016D00082701AF021FD0C2179481AF04BFF03218A
:1016E00078481AF047FF23680E930E9A23680D93EB
:1016F0000D9B704E9B1A312BF8D90C2170481AF0B3
:1017000039FF03216F481AF035FF33680C930C9AA8
:1017100023680B930B9B674E9B1A312BF8D907213B
:1017200069481AF027FF032166481AF023FF33683F
:101730000A930A9A23680993099B9B1A312BF9D9BA
:101740001AF09AFF00280CDD02230C2162482B605E
:101750001CF0B2FA29685F481CF08EFF5D481CF04F
:101760003BFF82201BF0E2F80C2155481BF02EFABB
:10177000032154481BF02AFA23681493149A23680F
:101780001393139B4B4E9B1A312BF8D90C214C48C9
:101790001BF01CFA03214B481BF018FA3368129314
:1017A000129A23681193119B424E9B1A312BF8D940
:1017B000072145481BF00AFA032142481BF006FAAC
:1017C00033681093109A23680F930F9B9B1A312B49
:1017D000F9D91BF02FFA00280CDD03230C213F4818
:1017E0002B601CF069FA29683A481CF045FF39481B
:1017F0001CF0F2FE0A213A483A4E1CF05DFA2968C4
:1018000034481CF039FF33481CF0E6FE364B1B68A9
:101810003746C6EB03083D46A43608EB050019F031
:10182000E9FD05F8010BB542F7D1304B304E1B688E
:10183000B346C6EB03085D46343608EB050019F0E5
:10184000D9FD05F8010BB542F7D12A4B2A4E1B688A
:101850003246C6EB03081546403608EB050019F082
:10186000C9FD05F8010BAE42F7D1244B244E1B688D
:10187000B246C6EB03085546343608EB050019F0AE
:10188000B9FD05F8010BB542F7D11E4B1E4D1E6880
:10189000A946761BC846103506EB080019F0AAFDCC
:1018A00008F8010BA845F7D1184B194D1E68A8463A
:1018B00030E000BF841BFF1FE41FFF1FA04E02008B
:1018C000A84E0200604E0200B84E02001007FF1F33
:1018D000C04E0200E407FF1FD04E0200E04E02009F
:1018E000F04E0200DC17FF1FE413FF1F2C07FF1F41
:1018F0009818FF1F0407FF1F6C13FF1F5007FF1FDF
:10190000AC13FF1F5807FF1F6C15FF1F1807FF1FA1
:10191000B814FF1F761B183506EB080019F06AFD96
:1019200008F8010B4545F7D1C24BC34D1E68A846C8
:10193000761B183506EB080019F05CFD08F8010B62
:10194000A845F7D1BD4BBE4D1E68A846761B18357D
:1019500006EB080019F04EFD08F8010BA845F7D179
:10196000B84BB94D1E682B46761B9846403506EBA2
:10197000080019F03FFD08F8010B4545F7D1B34BBE
:10198000B34D1E682B46761B98465C3506EB080067
:1019900019F030FD08F8010BA845F7D1AD4BAE4D5D
:1019A0001E682B46761B9846543506EB080019F046
:1019B00021FD08F8010B4545F7D1A84BA84D1E683D
:1019C0002B46761B9846603506EB080019F012FD91
:1019D00008F8010BA845F7D11321A2481CF06CF9B7
:1019E000DBF83010A0481CF047FE9F481CF0F4FDC7
:1019F00012219E481CF060F9DAF830109A481CF069
:101A00003BFE99481CF0E8FD1A2199481CF054F956
:101A1000D9F8001094481CF02FFE93481CF0DCFD10
:101A2000132194481CF048F9874B8F4819680A2203
:101A300000231CF0E1FD8C481CF0CEFD13218E48E4
:101A40001CF03AF98D4B884819680A2200231CF0D3
:101A5000D3FD85481CF0C0FD122189481CF02CF9EB
:101A60007D4B8148996C0A2200231CF0C5FD7E48FD
:101A70001CF0B2FD172183481CF01EF9784B7A4800
:101A800019680A2200231CF0B7FD77481CF0A4FD5A
:101A900013217D481CF010F96D4B7348996B0A2295
:101AA00000231CF0A9FD70481CF096FD01210420C4
:101AB00019F048FE01210E2019F044FE01211620E4
:101AC00019F040FE0121112019F03CFE00210320F5
:101AD000FEF7E4FF00210846FEF7E0FF00210120A9
:101AE000FEF7DCFF00210220FEF7D8FF0221387E3E
:101AF00019F028FE0221387F19F024FE23681A937A
:101B00001A9A23681993199B604D9B1A092BF8D9CF
:101B10000121387E19F002FE0121387F19F0FEFD07
:101B2000022197F82C0019F00DFE022197F83000E1
:101B300019F008FE2B681893189A23681793179BBF
:101B4000524D9B1A092BF8D9012197F82C0019F056
:101B5000E5FD012197F8300019F0E0FD022197F82A
:101B60004C0019F0EFFD022197F8500019F0EAFD42
:101B7000012197F84C0019F0D1FD97F85000012190
:101B800019F0CCFD2B681693169A23681593159BB4
:101B90009B1A092BF9D90121182019F0D3FD012135
:101BA000182019F0BBFD01210F2019F0CBFD0121F8
:101BB0000F2019F0B3FD01210A2019F0C3FD012106
:101BC0000A2019F0ABFD0121092019F0BBFD01210C
:101BD000092019F0A3FDFEF7F1FE00210320FEF716
:101BE0005DFF2A4E032501210D2019F097FD236882
:101BF0001E931E9A23681D931D9B9B1A312BF9D9A6
:101C000000210D2019F08AFD33681C931C9A23686B
:101C10001B931B9B9B1AB3F5967FF8D3013DE2D132
:101C20000E211B481CF048F80F481CF0D5FC23B0CF
:101C3000BDE8F08F1C07FF1F3816FF1F3407FF1F7A
:101C40005016FF1F3807FF1F9815FF1FFC06FF1FC8
:101C5000D012FF1F0007FF1F6414FF1F1407FF1F90
:101C6000F813FF1FFC4E0200E407FF1F104F020095
:101C7000244F0200404F0200544F02006C13FF1F1C
:101C8000684F02007C4F0200944F0200841BFF1F2C
:101C9000A84F020003280BD8DFE800F00806040272
:101CA0001AF0D8BF1AF0F8BC1AF03EB91BF09EBF6C
:101CB0000020704708B51AF027F9002801DD01203F
:101CC00008BD1AF0D9FC002801DD022008BD1AF079
:101CD000B1FF0028D4BF0020032008BD38B50D4C4B
:101CE0002068FFF7D7FFC5B202E02068FFF7D2FFF8
:101CF000FFF7E0FF0028F8DC042107481BF0DCFFB9
:101D0000294606481CF0B8FC04481CF065FC28462F
:101D100038BD00BF1007FF1FB84F0200E407FF1FC8
:101D200008B5FFF7C7FF002808DB134B1868FFF75B
:101D3000B1FF124BC0B25328187001D0002008BD6B
:101D400000210320FEF7AAFE0D4B1B68012B08D0D3
:101D500003D3022B09D0012008BD00210120FEF78A
:101D60009DFE00210120FEF799FE00210220FEF7D2
:101D700095FE012008BD00BF1007FF1FE816FF1FDA
:101D8000F813FF1FF0B51C2183B02748274C284DBE
:101D9000284E294F1BF090FF28481CF01DFC0E21F7
:101DA00027481BF089FF216824481CF065FC234864
:101DB0001CF012FC0023019309E0019B30681844D9
:101DC00019F032FB019B0133142B019314DC2868BA
:101DD000FFF760FFC0B2FF282368014619D0032B2C
:101DE000EBD1019B3A680146D01819F01DFB019B0D
:101DF0000133142B0193EADD2368032B0CBF114B35
:101E0000114B042219680DEB020019F035FB03B0E9
:101E1000F0BD032B0CBF084A064A019B1068002145
:101E2000184419F001FBE7E7C04F02004C07FF1F01
:101E30001007FF1F4807FF1F0C07FF1FE407FF1FC6
:101E4000E04F02005407FF1F2807FF1F2DE9F04F46
:101E500095B0074604A816F05DFD88201CF07CFBB9
:101E60000823102280E80C00C61800F188083546C7
:101E700034462046002110341CF07AFDA045F8D1EC
:101E80001721BF481BF018FFBE481CF0A5FB0CA88B
:101E90000123BD4ABD4916F02DFE0E9A9DF83C3037
:101EA0009DF8341006928DF81C308DF814100FAA8E
:101EB0000DF11D030DF12A0012F8011F03F8011B9B
:101EC0008342F9D1139B0B930CA816F031FD04A8A3
:101ED00016F05CFD002800F0AF8104A816F044FD68
:101EE0000A210446AA481BF0E7FE214600230A22E5
:101EF000A4481CF081FBA3481CF06EFB002F4AD0C5
:101F000017F1060900F1B7800024A24610E0013C59
:101F10000CA816F03BFD8046002842D00CA816F015
:101F200027FD01340CA816F003FD4C4500F3A380F7
:101F3000012204A90CA816F051FE0CA816F0FAFC18
:101F4000804620F0DDFA014640461BF0B5FE8D4884
:101F50001CF042FB0CA816F0EFFC0028D7D10CA80F
:101F600016F0E8FC01468B4820F0EEF80A21002824
:101F70005CD189481BF0A0FE0CA816F0DBFC804663
:101F800020F0BEFA014640461BF096FE7D48013C1B
:101F90001CF022FBC2E7814B64221A604FF0060955
:101FA000B2E70F217E48DFF8F4B11BF085FE214631
:101FB00074481CF061FB03217A481BF07DFEDBF8BE
:101FC000001070481CF058FB04F108030321754809
:101FD000CBF800301BF070FEDBF8001069481CF0F5
:101FE0004BFB68481CF0F8FA68466F491CF0C0FCCF
:101FF00041466846FFF742F968461CF079FC22200A
:10200000FFF7AEFA631E00EE103A4046B8EEC00A83
:10201000FFF74AFA684665491CF0AAFC6846414643
:10202000FFF72CF968461CF063FC77E760481BF06B
:1020300043FE214653481CF01FFB032159481BF067
:102040003BFE0CA816F076FC804620F059FA0146BB
:1020500040461BF031FE032152481BF02DFEA742E3
:1020600040F3F48006EB0A1146481CF08FFA45480D
:102070001CF0B2FA4CE70126741E03214D481BF0F8
:102080001BFE21463F481CF0F7FA032145481BF090
:1020900013FE29463B481CF079FAB41E39481CF05F
:1020A0009BFA052C04D8DFE804F068666462359575
:1020B00041490CA81CF05CFC00210CA8FFF7DEF8DD
:1020C0000CA81CF015FC3D490CA81CF051FC00218B
:1020D0000CA8FFF7D3F80CA81CF00AFC29460CA8A2
:1020E0001CF05AFC00210CA8FFF7C8F80CA81CF043
:1020F000FFFB2E490CA81CF03BFC00210CA8FFF7AD
:10210000BDF80CA81CF0F4FB072E00F08F801035F2
:102110000136B1E72A490CA81CF02AFC00210CA8C2
:10212000FFF7ACF80CA81CF0E3FB24490CA81CF04A
:102130001FFC00210CA8FFF7A1F80CA81CF0D8FB8D
:1021400029460CA81CF028FC00210CA8FFF796F8E3
:102150000CA81CF0CDFB15490CA81CF009FC0CA820
:102160000021FFF78BF80CA81CF0C2FBCFE7154944
:10217000D1E71549CFE71549CDE71549CBE700BFB2
:10218000F04F0200E407FF1F08500200D018FF1FA5
:102190000C50020028500200345002004007FF1F7C
:1021A000505002004C500200605002007450020077
:1021B000405002007C500200805002009850020003
:1021C000FC500200E4500200CC500200B450020067
:1021D0009C50020023490CA81CF0CAFB00210CA84B
:1021E000FFF74CF80CA81CF083FB1F490CA81CF04F
:1021F000BFFB00210CA8FFF741F80CA81CF078FBEE
:1022000029460CA81CF0C8FB00210CA8FFF736F8E3
:102210000CA81CF06DFB15490CA81CF0A9FB0CA820
:102220000021FFF72BF80CA81CF062FB04A816F0A5
:102230007FFB15B0BDE8F08F0E210D481BF03CFD73
:1022400004A816F075FB15B0BDE8F08F0CA816F0C9
:1022500071FB06EB0A18014640461CF011FC0AF11E
:10226000010AFFE614510200985002007450020067
:102270001850020008B5084BDFED080AD3ED007ACC
:1022800027EE800A1DF068F81CF0BEFF044BD3ED6A
:10229000007A20EE270A08BD5814FF1FDB0FC94043
:1022A0008C15FF1F08B52C4A2C4B92ED010A93EDBB
:1022B000007ADFED2B6A2B4BB8EEC77A9B6BC6EE2C
:1022C000877A012BB8EEC00A2DED028B27EE800A2B
:1022D0003BD034D3022B2CD09FED238AFFF7CAFFCB
:1022E000224A234B92ED007A002283F8902072B6A6
:1022F000DFED207A93ED206AD3ED1F6A30EE480AB5
:10230000B8EEC77AC0EE275AC5EE877A67EE867AAE
:10231000F4EEE67AC3ED1E7AD3ED227AF1EE10FAEE
:10232000D8BFF1EE677AC3ED237A62B6BDEC028BBB
:1023300008BD114B93ED018AB8EEC88ACEE70F4B6A
:1023400093ED018AB8EEC88AC8E70D4B93ED018A78
:10235000B8EEC88AC2E700BF7812FF1FCC18FF1F73
:10236000DB0FC940D012FF1F000000009816FF1FAE
:10237000D414FF1FCDCCCC3CD815FF1FEC16FF1F8B
:10238000A416FF1F2DE9F04F1621ADB00446B14849
:102390001BF092FCB0481CF01FF90A2C00F27C8460
:1023A000DFE814F095007A04CD01AA026C017A04EA
:1023B0002703F901D403D4030B00A84B1D680DF1CA
:1023C0005008C8EB050544462BAE281919F012F841
:1023D00004F8010BA642F8D1A14907A81CF0C8FADD
:1023E000002107A8FEF74AFF07A81CF081FA222067
:1023F000FFF7B6F8DDED147A0020B8EEE70AFFF734
:1024000053F8984907A81CF0B3FA002107A8FEF773
:1024100035FF07A81CF06CFA934907A81CF0A8FA2E
:10242000002107A8FEF72AFF07A81CF061FA222066
:10243000FFF796F8DDED187A0020B8EE670AFFF78F
:1024400033F8884907A81CF093FA07A80021FEF783
:1024500015FF07A81CF04CFA229B012B00F0EC861C
:10246000C0F0B886022B40F09582804907A81CF086
:102470007FFA002107A8FEF701FF07A81CF038FA31
:102480002220FFF76DF8DDED177A0020B8EE670A1D
:10249000FFF70AF8734907A81CF06AFA002107A899
:1024A000FEF7ECFE07A81CF023FA714907A81CF000
:1024B0005FFA002107A8FEF7E1FE07A81CF018FA52
:1024C0002220FFF74DF80020DDED1B7A1AE3694B5F
:1024D0001D6807AC2E1B0DF15008301918F08AFF4B
:1024E00004F8010BA045F8D1C8EB050521AE444620
:1024F000281918F07FFF04F8010BA642F8D15849BB
:1025000003A81CF035FA002103A8FEF7B7FE03A8C4
:102510001CF0EEF9584903A81CF02AFA002103A880
:10252000FEF7ACFE03A81CF0E3F9DDED087A00200D
:10253000B8EEE70AFEF7B8FF4A4903A81CF018FAFC
:10254000002103A8FEF79AFE03A81CF0D1F9464922
:1025500003A81CF00DFA002103A8FEF78FFE03A8C4
:102560001CF0C6F9444903A81CF002FA002103A894
:10257000FEF784FE03A81CF0BBF9DDED107A002005
:10258000B8EEE70AFEF790FF364903A81CF0F0F911
:1025900003A80021FEF772FE03A81CF0A9F9139C02
:1025A000012C00F03B85022C00F0D184002C40F07F
:1025B000F1812E4903A81CF0DBF9214603A8FEF7A0
:1025C0005DFE03A81CF094F92B4903A81CF0D0F978
:1025D000214603A8FEF752FE03A81CF089F9DDEDA1
:1025E000097A2046B8EEE70AFEF75EFF1D4903A808
:1025F0001CF0BEF9214603A8FEF740FE03A81CF01C
:1026000077F91B4903A81CF0B3F9214603A8FEF78C
:1026100035FE03A81CF06CF9174903A81CF0A8F9B3
:10262000214603A8FEF72AFE03A81CF061F9DDEDA0
:10263000117A2046B8EEE70AFEF736FF094903A8EB
:102640001CF096F903A82146FEF718FE03A81CF01B
:102650004FF99FE12C510200E407FF1FFC06FF1F0A
:102660004451020074500200585102006C510200A3
:10267000805102002C07FF1F98500200924B1D68EA
:102680000DF15008C8EB0505444624AE281918F092
:10269000B1FE04F8010BA642F8D1149A052A00F203
:1026A00079810123934013F0300440F0E98313F063
:1026B0000C0540F03A869B0700F06C8107A883491F
:1026C0001CF056F9294607A8FEF7D8FD07A81CF00C
:1026D0000FF92220FEF744FFDDED157A2846B8EE0B
:1026E000E70AFEF7E1FE07A879491CF041F92946FF
:1026F00007A8FEF7C3FD07A81CF0FAF807A875495C
:102700001CF036F9294607A8FEF7B8FD07A81CF00B
:10271000EFF82220FEF724FFDDED167A2846B8EE0A
:10272000670AFEF7C1FE07A869491CF021F907A84E
:102730002946FEF7A3FD07A81CF0DAF82AE1664B4C
:102740001D680DF15008C8EB0505444621AE281957
:1027500018F050FE04F8010BA642F8D11E9B5F480A
:1027600001930B21DDF854B0DDF874A0DDF858902A
:10277000179F1F9E189D149C1BF09EFA58481BF033
:102780002BFF209B032B00F20581DFE813F03103C0
:10279000FD02C9028802534B1D680DF15008C8EBB9
:1027A0000505444629AE281918F024FE04F8010B4B
:1027B000A642F8D14C4907A81CF0DAF8002107A876
:1027C000FEF75CFD07A81CF093F82220FEF7C8FE78
:1027D000DDED147A0020B8EEE70AFEF765FE3C490D
:1027E00007A81CF0C5F8002107A8FEF747FD07A8B9
:1027F0001CF07EF83D4907A81CF0BAF8002107A894
:10280000FEF73CFD07A81CF073F82220FEF7A8FE97
:10281000DDED1C7A0020B8EE670AFEF745FE2C4974
:1028200007A81CF0A5F8002107A8FEF727FD07A8B8
:102830001CF05EF807212E481BF03EFA269C284823
:10284000214600230A221BF0D7FE25481BF0C4FEB8
:10285000012C00F04983C0F01584022C40F09A80CE
:102860001A4907A81CF084F8002107A8FEF706FD06
:1028700007A81CF03DF82220FEF772FE1D4B93EDD9
:10288000030A0020B8EEC00AFEF70EFE104907A8A2
:102890001CF06EF8002107A8FEF7F0FC07A81CF05A
:1028A00027F80C4907A81CF063F8002107A8FEF7D9
:1028B000E5FC07A81CF01CF82220FEF751FE0020C2
:1028C000DDED1F7A1EE100BF3807FF1F6C510200CB
:1028D00074500200805102005007FF1FF0510200A7
:1028E000E407FF1F0007FF1F445102005851020078
:1028F000E85102006414FF1F8A4B1D6807AC2D1BB2
:102900000BAE281918F076FD04F8010BA642F8D199
:102910000DF15008844940461CF02AF80021404639
:10292000FEF7ACFC40461BF0E3FF2220FEF718FE4A
:10293000DDED087A0020B8EEE70AFEF7B5FD7B4929
:1029400040461CF015F800214046FEF797FC404633
:102950001BF0CEFF764940461CF00AF800214046A5
:10296000FEF78CFC40461BF0C3FF2220FEF7F8FD6B
:10297000DDED0A7A0020B8EE670AFEF795FD6B4997
:1029800040461BF0F5FF40460021FEF777FC40462D
:102990001BF0AEFF674940461BF0EAFF00214046AE
:1029A000FEF76CFC40461BF0A3FF634940461BF05A
:1029B000DFFF00214046FEF761FC40461BF098FF18
:1029C0005E4940461BF0D4FF00214046FEF756FC0E
:1029D00040461BF08DFF584940461BF0C9FF0021BF
:1029E0004046FEF74BFC40461BF082FF2DB0BDE891
:1029F000F08F534B1D680DF15008C8EB0505444698
:102A000024AE281918F0F6FC04F8010BA642F8D100
:102A1000454907A81BF0ACFF002107A8FEF72EFCD4
:102A200007A81BF065FF2220FEF79AFDDDED157A61
:102A30000020B8EEE70AFEF737FD3C4907A81BF077
:102A400097FF002107A8FEF719FC07A81BF050FF0D
:102A5000374907A81BF08CFF002107A8FEF70EFCE2
:102A600007A81BF045FF2220FEF77AFDDDED167A60
:102A70000020B8EE670AFEF717FD2C4907A81BF0E7
:102A800077FF07A80021FEF7F9FB07A81BF030FF2E
:102A9000149B012B00F02883C0F06A83022B7FF483
:102AA00079AF284907A81BF063FF002107A8FEF7AC
:102AB000E5FB07A81BF01CFF2220FEF751FDDDED12
:102AC0001B7A0020B8EEE70AFEF7EEFC174907A8CC
:102AD0001BF04EFF002107A8FEF7D0FB07A81BF054
:102AE00007FF194907A81BF043FF002107A8FEF7BD
:102AF000C5FB07A81BF0FCFE2220FEF731FDDDED33
:102B00001C7A0020B8EE670AFEF7CEFC074907A83A
:102B10001BF02EFF07A80021FEF7B0FB07A81BF053
:102B2000E7FE37E75807FF1F4451020074500200C8
:102B30005851020024520200604E02003C52020032
:102B40000407FF1F6C51020080510200C24B1D6838
:102B50000DF15008C8EB050544462CAE281918F0B5
:102B600049FC04F8010BA642F8D1BC49BC4C07A8AB
:102B70001BF0FEFE002107A8FEF780FB07A81BF054
:102B8000B7FE2220FEF7ECFCDDED207A0020B8EE47
:102B9000E70AFEF789FCB34907A81BF0E9FE00210C
:102BA00007A8FEF76BFB07A81BF0A2FEAE4907A81B
:102BB0001BF0DEFE002107A8FEF760FB07A81BF054
:102BC00097FE2220FEF7CCFC289D07EE905A0020AD
:102BD000B8EE670AFEF768FCA24907A81BF0C8FE1A
:102BE000002107A8FEF74AFB07A81BF081FE0F2172
:102BF0009E481BF061F800230A22216D9C481BF0BF
:102C0000FBFC9B481BF0E8FC16219A481BF054F88B
:102C1000002329460A2296481BF0EEFC94481BF03C
:102C2000DBFC2368012B00F04D83C0F01983022BDD
:102C30007FF4B0AE904907A81BF09AFE002107A8C8
:102C4000FEF71CFB07A81BF053FE2220FEF788FCB2
:102C5000DDED237A0020B8EEE70AFEF725FC814976
:102C600007A81BF085FE002107A8FEF707FB07A8B1
:102C70001BF03EFE814907A81BF07AFE002107A841
:102C8000FEF7FCFA07A81BF033FE2220FEF768FCD3
:102C90000020DDED2B7A35E70DF150087AE66F491B
:102CA00007A81BF065FE002107A8FEF7E7FA07A8B2
:102CB0001BF01EFE2220FEF753FC07EE90BA002008
:102CC000B8EEE70AFEF7F0FB664907A81BF050FED6
:102CD000002107A8FEF7D2FA07A81BF009FE6249F7
:102CE00007A81BF045FE002107A8FEF7C7FA07A8B2
:102CF0001BF0FEFD2220FEF733FC07EE90AAB8EE93
:102D0000E70A0020FEF7D0FB07A856491BF030FE6B
:102D100007A80021FEF7B2FA07A81BF0E9FD39E683
:102D2000554907A81BF024FE002107A8FEF7A6FAC4
:102D300007A81BF0DDFD2220FEF712FC07EE905ADB
:102D40000020B8EEE70AFEF7AFFB464907A81BF0E4
:102D50000FFE002107A8FEF791FA07A81BF0C8FD97
:102D6000464907A81BF004FE002107A8FEF786FAD3
:102D700007A81BF0BDFD2220FEF7F2FB07EE904AEC
:102D80000020B8EEE70ABDE73B4907A81BF0F0FDBD
:102D9000002107A8FEF772FA07A81BF0A9FD222060
:102DA000FEF7DEFB07EE907A0020B8EEE70AFEF7AA
:102DB0007BFB2C4907A81BF0DBFD002107A8FEF7D1
:102DC0005DFA07A81BF094FD2C4907A81BF0D0FD65
:102DD000002107A8FEF752FA07A81BF089FD222060
:102DE000FEF7BEFB07EE906A0020B8EEE70A89E71F
:102DF000214907A81BF0BCFD002107A8FEF73EFAF9
:102E000007A81BF075FD2220FEF7AAFB07EE909A9B
:102E10000020B8EEE70AFEF747FB124907A81BF0AF
:102E2000A7FD002107A8FEF729FA07A81BF060FDFF
:102E3000124907A81BF09CFD002107A8FEF71EFA07
:102E400007A81BF055FD2220FEF78AFBDDED017A75
:102E50000020B8EEE70A55E71407FF1F44510200AF
:102E6000F813FF1F7450020058510200FC51020079
:102E7000E407FF1F0C5202006C5102008051020057
:102E8000B24907A81BF074FD002107A8FEF7F6F968
:102E900007A81BF02DFD2220FEF762FBDDED1B7A5B
:102EA0000020B8EEE70AFEF7FFFAA94907A81BF0D1
:102EB0005FFD002107A8FEF7E1F907A81BF018FD48
:102EC000A44907A81BF054FD002107A8FEF7D6F976
:102ED00007A81BF00DFD2220FEF742FBDDED1C7A5A
:102EE0000020B8EE670A0DE7984907A81BF040FDDF
:102EF000002107A8FEF7C2F907A81BF0F9FC222061
:102F0000FEF72EFB944B93ED020A0020B8EEC00AA8
:102F1000FEF7CAFA8E4907A81BF02AFD002107A870
:102F2000FEF7ACF907A81BF0E3FC8A4907A81BF0E1
:102F30001FFD002107A8FEF7A1F907A81BF0D8FC88
:102F40002220FEF70DFB0020DDED1E7ADAE51821C8
:102F500082481AF0B1FE824B824819681BF08CFB44
:102F600080481BF039FB19217F481AF0A5FE1499FF
:102F70007C481BF081FB7B481BF02EFB18217B4813
:102F80001AF09AFE079C774821461BF075FB75489E
:102F90001BF022FB6D4903A81BF0EAFC002103A8EB
:102FA000FEF76CF903A81BF0A3FC2220FEF7D8FA69
:102FB000DDED0B7A0020B8EEE70AFEF775FA6449FA
:102FC00003A81BF0D5FC002103A8FEF757F903A8BE
:102FD0001BF08EFC642018F0BBFB5E4903A81BF0BD
:102FE000C7FC002103A8FEF749F903A81BF080FCE9
:102FF0002220FEF7B5FA07EE904AB8EEE70A002065
:10300000FEF752FA524903A81BF0B2FC03A80021B4
:10301000FEF734F903A81BF06BFCBBE44B4903A893
:103020001BF0A6FC002103A8FEF728F903A81BF05B
:103030005FFC2220FEF794FADDED0A7A0020B8EE5C
:10304000E70AFEF731FA424903A81BF091FC002180
:1030500003A8FEF713F903A81BF04AFC3D4903A897
:103060001BF086FC002103A8FEF708F903A81BF05B
:103070003FFC2220FEF774FADDED127A0020B8EE54
:10308000E70ABDE7314907A81BF072FC002107A839
:10309000FEF7F4F807A81BF02BFC2220FEF760FADD
:1030A000DDED157A0020B8EEE70AFEF7FDF92849B4
:1030B00007A81BF05DFC002107A8FEF7DFF807A8B2
:1030C0001BF016FC234907A81BF052FC002107A89F
:1030D000FEF7D4F807A81BF00BFC2220FEF740FAFD
:1030E0000020DDED1D7A0DE5184907A81BF040FC16
:1030F000002107A8FEF7C2F807A81BF0F9FB222061
:10310000FEF72EFADDED197AB8EEE70A0020FEF799
:10311000CBF90F4907A81BF02BFC002107A8FEF7ED
:10312000ADF807A81BF0E4FB0A4907A81BF020FC38
:10313000002107A8FEF7A2F807A81BF0D9FB222060
:10314000FEF70EFA0020DDED1A7ADBE46C51020086
:1031500074500200805102006414FF1F9451020059
:103160009818FF1FE407FF1FB0510200CC51020066
:103170008F4907A81BF0FCFB002107A8FEF77EF88B
:1031800007A81BF0B5FB2220FEF7EAF9DDED177A60
:103190000020B8EEE70AFEF787F9864907A81BF07A
:1031A000E7FB002107A8FEF769F807A81BF0A0FBC2
:1031B000814907A81BF0DCFB002107A8FEF75EF899
:1031C00007A81BF095FB2220FEF7CAF90020DDEDD1
:1031D000187A97E4764907A81BF0CAFB002107A8D4
:1031E000FEF74CF807A81BF083FB2220FEF7B8F986
:1031F000DDED157A0020B8EEE70AFEF755F96D49C6
:1032000007A81BF0B5FB002107A8FEF737F807A8B1
:103210001BF06EFB684907A81BF0AAFB002107A85A
:10322000FEF72CF807A81BF063FB2220FEF798F9A5
:103230000020DDED197A65E45D4907A81BF098FBD5
:10324000002107A8FEF71AF807A81BF051FB22205F
:10325000FEF786F9DDED167A0020B8EE670A56E72C
:10326000534907A81BF084FB002107A8FEF706F8C6
:1032700007A81BF03DFB2220FEF772F9DDED217A55
:103280000020B8EEE70AFEF70FF94A4907A81BF03D
:103290006FFB002107A8FDF7F1FF07A81BF028FB33
:1032A000454907A81BF064FB002107A8FDF7E6FFCE
:1032B00007A81BF01DFB2220FEF752F90020DDEDD0
:1032C000297A1FE43A4907A81BF052FB002107A8FE
:1032D000FDF7D4FF07A81BF00BFB2220FEF740F9F7
:1032E000DDED227A0020B8EEE70AFEF7DDF831497D
:1032F00007A81BF03DFB002107A8FDF7BFFF07A8AB
:103300001BF0F6FA2C4907A81BF032FB002107A896
:10331000FDF7B4FF07A81BF0EBFA2220FEF720F917
:103320000020DDED2A7AFFF7EDBB07A820491BF04E
:103330001FFB214607A8FDF7A1FF07A81BF0D8FA3D
:103340002220FEF70DF9DDED187A2046B8EEE70AE7
:10335000FEF7AAF807A817491BF00AFB214607A8A1
:10336000FDF78CFF07A81BF0C3FA07A812491BF052
:10337000FFFA214607A8FDF781FF07A81BF0B8FA5E
:103380002220FEF7EDF8DDED197A2046B8EE670A47
:10339000FEF78AF807A807491BF0EAFA07A82146B2
:1033A000FDF76CFF07A81BF0A3FAFFF7F3BA00BF05
:1033B0006C510200745002008051020070B5C64B7F
:1033C000AEB01D6805AC2D1B2EAE281918F012F8F2
:1033D00004F8010BB442F8D1C049C14CC14D01A859
:1033E0001BF0C6FA002101A8FDF748FF01A81BF059
:1033F0007FFA2220FEF7B4F8DDED057A0020B8EE62
:10340000670AFEF751F8B84901A81BF0B1FA00218C
:1034100001A8FDF733FF01A81BF06AFAB34901A820
:103420001BF0A6FA002101A8FDF728FF01A81BF058
:103430005FFA2220FEF794F8DDED067A0020B8EE60
:10344000670AFEF731F8A84901A81BF091FA00219C
:1034500001A8FDF713FF01A81BF04AFAA44901A82F
:103460001BF086FA002101A8FDF708FF01A81BF058
:103470003FFA2220FEF774F89DED070A0420FEF7BC
:1034800013F8994901A81BF073FA002101A8FDF770
:10349000F5FE01A81BF02CFA964901A81BF068FA6A
:1034A000002101A8FDF7EAFE01A81BF021FA222065
:1034B000FEF756F89DF8881001A8002914BF294688
:1034C00021461BF055FA002101A8FDF7D7FE01A8FF
:1034D0001BF00EFA844901A81BF04AFA002101A84A
:1034E000FDF7CCFE01A81BF003FA834901A81BF0ED
:1034F0003FFA002101A8FDF7C1FE01A81BF0F8F971
:103500002220FEF72DF8DDED267A0020B8EE670ABE
:10351000FDF7CAFF744901A81BF02AFA002101A88F
:10352000FDF7ACFE01A81BF0E3F9744901A81BF0FC
:103530001FFA002101A8FDF7A1FE01A81BF0D8F990
:103540002220FEF70DF8DDED277A0020B8EE670A9D
:10355000FDF7AAFF644901A81BF00AFA002101A89F
:10356000FDF78CFE01A81BF0C3F9654901A81BF00B
:10357000FFF9002101A8FDF781FE01A81BF0B8F9B1
:103580002220FDF7EDFFDDED087A0020B8EE670A96
:10359000FDF78AFF544901A81BF0EAF9002101A8B0
:1035A000FDF76CFE01A81BF0A3F9564901A81BF01A
:1035B000DFF9002101A8FDF761FE01A81BF098F9D1
:1035C0002220FDF7CDFFDDED097A0020B8EE670A75
:1035D000FDF76AFF444901A81BF0CAF9002101A8C0
:1035E000FDF74CFE01A81BF083F9474901A81BF029
:1035F000BFF9002101A8FDF741FE01A81BF078F9F1
:103600002220FDF7ADFF9DED0A0A0420FDF74CFFD7
:10361000354901A81BF0ACF9002101A8FDF72EFEE9
:1036200001A81BF065F9394901A81BF0A1F9002197
:1036300001A8FDF723FE01A81BF05AF92220FDF78F
:103640008FFF9DF8891001A8002914BF2946214643
:103650001BF08EF9002101A8FDF710FE01A81BF058
:1036600047F9214901A81BF083F9002101A8FDF7C2
:1036700005FE01A81BF03CF9254901A81BF078F9CB
:10368000002101A8FDF7FAFD01A81BF031F9222065
:10369000FDF766FFDDED0D7A0020B8EE670AFDF755
:1036A00003FF114901A81BF063F9002101A8FDF7F0
:1036B000E5FD01A81BF01CF9164901A81BF058F9FB
:1036C000002101A8FDF7DAFD01A81BF011F9222065
:1036D000FDF746FF20E000BFE413FF1F6052020029
:1036E00058520200545202007450020078520200F4
:1036F00090520200A8520200C0520200D4520200AE
:10370000EC520200FC5202000C5302001C53020057
:103710002C5302003C530200DDED0E7A0020B8EE7F
:10372000670AFDF7C1FEC34901A81BF021F900217A
:1037300001A8FDF7A3FD01A81BF0DAF8BE4901A816
:103740001BF016F9002101A8FDF798FD01A81BF058
:10375000CFF82220FDF704FF9DED0F0A0520FDF7AD
:10376000A3FEB44901A81BF003F9002101A8FDF74D
:1037700085FD01A81BF0BCF8B04901A81BF0F8F8C2
:10378000002101A8FDF77AFD01A81BF0B1F8222065
:10379000FDF7E6FE9DF88A1001A8002914BF29460E
:1037A00021461BF0E5F8002101A8FDF767FD01A8FF
:1037B0001BF09EF89F4901A81BF0DAF8002101A830
:1037C000FDF75CFD01A81BF093F89D4901A81BF0D3
:1037D000CFF8002101A8FDF751FD01A81BF088F8E2
:1037E0002220FDF7BDFEDDED2A7A0020B8EE670A43
:1037F000FDF75AFE8F4901A81BF0BAF8002101A875
:10380000FDF73CFD01A81BF073F88E4901A81BF0E1
:10381000AFF8002101A8FDF731FD01A81BF068F801
:103820002220FDF79DFEDDED2B7A0020B8EE670A21
:10383000FDF73AFE7F4901A81BF09AF8002101A884
:10384000FDF71CFD01A81BF053F87F4901A81BF0F0
:103850008FF8002101A8FDF711FD01A81BF048F821
:103860002220FDF77DFE9DED2C0A0520FDF71CFEB4
:10387000704901A81BF07CF8002101A8FDF7FEFCAF
:1038800001A81BF035F8714901A81BF071F800215F
:1038900001A8FDF7F3FC01A81BF02AF82220FDF790
:1038A0005FFE9DF8B41001A8002914BF29462146E7
:1038B0001BF05EF8002101A8FDF7E0FC01A81BF059
:1038C00017F85C4901A81BF053F8002101A8FDF787
:1038D000D5FC01A81BF00CF85D4901A81BF048F8C5
:1038E000002101A8FDF7CAFC01A81BF001F8222065
:1038F000FDF736FEDDED137A0020B8EE670AFDF71E
:10390000D3FD4C4901A81BF033F8002101A8FDF7B5
:10391000B5FC01A81AF0ECFF4E4901A81BF028F8ED
:10392000002101A8FDF7AAFC01A81AF0E1FF22205E
:10393000FDF716FEDDED147A0020B8EE670AFDF7FC
:10394000B3FD3C4901A81BF013F8002101A8FDF7C5
:1039500095FC01A81AF0CCFF3F4901A81BF008F81C
:10396000002101A8FDF78AFC01A81AF0C1FF22205E
:10397000FDF7F6FD9DED150A0420FDF795FD2D4997
:1039800001A81AF0F5FF002101A8FDF777FC01A8B6
:103990001AF0AEFF314901A81AF0EAFF002101A890
:1039A000FDF76CFC01A81AF0A3FF2220FDF7D8FD5B
:1039B0009DF88B1001A8002914BF294621461AF052
:1039C000D7FF002101A8FDF759FC01A81AF090FFCC
:1039D000184901A81AF0CCFF01A80021FDF74EFC00
:1039E00001A81AF085FF129C002C40F096801C491B
:1039F00001A81AF0BDFF214601A8FDF73FFC01A870
:103A00001AF076FF174901A81AF0B2FF214601A863
:103A1000FDF734FC01A81AF06BFF134901A81AF056
:103A2000A7FF214601A8FDF729FC01A81AF060FFB5
:103A30001CE000BF745002004C5302005C530200B3
:103A40006C530200845302009C530200B4530200E2
:103A5000CC530200DC530200EC530200FC53020082
:103A60002C540200604E02003C540200414901A85F
:103A70001AF07EFF01A82146FDF700FC01A81AF00C
:103A800037FF3D4901A81AF073FF002101A8FDF797
:103A9000F5FB01A81AF02CFF2220FDF761FD9DED3A
:103AA000160A0420FDF700FD344901A81AF060FF52
:103AB000002101A8FDF7E2FB01A81AF019FF304927
:103AC00001A81AF055FF002101A8FDF7D7FB01A8B6
:103AD0001AF00EFF274901A81AF04AFF002101A899
:103AE000FDF7CCFB01A81AF003FF264901A81AF044
:103AF0003FFF002101A8FDF7C1FB01A81AF0F8FE65
:103B00001C4901A81AF034FF002101A8FDF7B6FBFB
:103B100001A81AF0EDFE2EB070BD1B4901A81AF0E5
:103B200027FF002101A8FDF7A9FB01A81AF0E0FE7C
:103B3000104901A81AF01CFF002101A8FDF79EFB07
:103B400001A81AF0D5FE114901A81AF011FF0021B1
:103B500001A8FDF793FB01A81AF0CAFE054901A8C8
:103B60001AF006FF01A80021FDF788FB01A81AF052
:103B7000BFFE86E7604E02004C5402007450020003
:103B80005C540200745402000C5402001C540200E5
:103B900070B5C24BAEB01D6805AC2D1B2EAE2819FA
:103BA00017F028FC04F8010BA642F8D1BC49BD4C23
:103BB00001A81AF0DDFE002101A8FDF75FFB01A8B6
:103BC0001AF096FE2220FDF7CBFCD4ED067A0020F9
:103BD000B8EE670AFDF768FCB34901A81AF0C8FE01
:103BE000002101A8FDF74AFB01A81AF081FEAF49A8
:103BF00001A81AF0BDFE002101A8FDF73FFB01A8B6
:103C00001AF076FE2220FDF7ABFCD4ED077A0020F7
:103C1000B8EE670AFDF748FCA34901A81AF0A8FE10
:103C2000002101A8FDF72AFB01A81AF061FEA049B6
:103C300001A81AF09DFE002101A8FDF71FFB01A8B5
:103C40001AF056FE2220FDF78BFCD4ED1E7A0020E0
:103C5000B8EE670AFDF728FC934901A81AF088FE20
:103C6000002101A8FDF70AFB01A81AF041FE9149C5
:103C700001A81AF07DFE002101A8FDF7FFFA01A8B6
:103C80001AF036FE2220FDF76BFCD4ED0B7A0020F3
:103C9000B8EE670AFDF708FC834901A81AF068FE30
:103CA000002101A8FDF7EAFA01A81AF021FE8249D5
:103CB00001A81AF05DFE002101A8FDF7DFFA01A8B6
:103CC0001AF016FE2220FDF74BFCD4ED0C7A0020F2
:103CD000B8EE670AFDF7E8FB734901A81AF048FE41
:103CE000002101A8FDF7CAFA01A81AF001FE7349E4
:103CF00001A81AF03DFE002101A8FDF7BFFA01A8B6
:103D00001AF0F6FD2220FDF72BFCD4ED1F7A0020DF
:103D1000B8EE670AFDF7C8FB634901A81AF028FE50
:103D2000002101A8FDF7AAFA01A81AF0E1FD6449F3
:103D300001A81AF01DFE002101A8FDF79FFA01A8B5
:103D40001AF0D6FD2220FDF70BFCD4ED137A0020EB
:103D5000B8EE670AFDF7A8FB534901A81AF008FE60
:103D6000002101A8FDF78AFA01A81AF0C1FD554902
:103D700001A81AF0FDFD002101A8FDF77FFA01A8B6
:103D80001AF0B6FD2220FDF7EBFBD4ED147A0020EB
:103D9000B8EE670AFDF788FB434901A81AF0E8FD71
:103DA000002101A8FDF76AFA01A81AF0A1FD464911
:103DB00001A81AF0DDFD002101A8FDF75FFA01A8B6
:103DC0001AF096FD2220FDF7CBFBD4ED207A0020DF
:103DD000B8EE670AFDF768FB334901A81AF0C8FD81
:103DE000002101A8FDF74AFA01A81AF081FD0D2172
:103DF000364819F061FFD4F88C10354800230A22A8
:103E00001AF0FAFB32481AF0E7FBD4F88C40002C89
:103E100068D1304901A81AF0ABFD01A82146FDF791
:103E20002DFA01A81AF064FD2B4901A81AF0A0FD93
:103E3000002101A8FDF722FA01A81AF059FD27492F
:103E400001A81AF095FD002101A8FDF717FA01A8B5
:103E50001AF04EFD204901A81AF08AFD002101A8A0
:103E6000FDF70CFA01A81AF043FD1D4901A81AF04C
:103E70007FFD002101A8FDF701FA01A81AF038FD25
:103E8000154901A81AF074FD002101A8FDF7F6F903
:103E900001A81AF02DFD2EB070BD00BFE413FF1F66
:103EA00088540200DC17FF1F745002009C5402006B
:103EB000B0540200C4540200D8540200EC54020072
:103EC0000055020014550200285502003C5502001E
:103ED000E407FF1F60550200604E020074550200A7
:103EE00090550200054901A81AF042FD01A80021E1
:103EF000FDF7C4F901A81AF0FBFC95E74C55020048
:103F000070B59D4BAEB01D6805AC2D1B2EAE2819AB
:103F100017F070FA04F8010BB442F8D101A89749E0
:103F20001AF026FD002101A8FDF7A8F901A81AF052
:103F3000DFFC2220FDF714FBDDED1A7A0020B8EE3D
:103F4000E70AFDF7B1FA01A88D491AF011FD01A8A1
:103F50000021FDF793F901A81AF0CAFC01A88949CC
:103F60001AF006FD002101A8FDF788F901A81AF052
:103F7000BFFC2220FDF7F4FADDED1B7A0020B8EE3D
:103F8000670AFDF791FA01A87D491AF0F1FC01A832
:103F90000021FDF773F901A81AF0AAFC01A87A49DB
:103FA0001AF0E6FC002101A8FDF768F901A81AF053
:103FB0009FFC2220FDF7D4FADDED1C7A0020B8EE3C
:103FC000E70AFDF771FA01A86D491AF0D1FC01A8C2
:103FD0000021FDF753F901A81AF08AFC01A86B49EA
:103FE0001AF0C6FC002101A8FDF748F901A81AF053
:103FF0007FFC2220FDF7B4FADDED1D7A0020B8EE3B
:10400000670AFDF751FA01A85D491AF0B1FC01A851
:104010000021FDF733F901A81AF06AFC01A85C49F8
:104020001AF0A6FC002101A8FDF728F901A81AF052
:104030005FFC2220FDF794FADDED1E7A0020B8EE39
:10404000E70AFDF731FA01A84D491AF091FC01A8E1
:104050000021FDF713F901A81AF04AFC01A84D4907
:104060001AF086FC002101A8FDF708F901A81AF052
:104070003FFC2220FDF774FADDED1F7A0020B8EE38
:10408000670AFDF711FA01A83D491AF071FC01A871
:104090000021FDF7F3F801A81AF02AFC01A83E4917
:1040A0001AF066FC002101A8FDF7E8F801A81AF053
:1040B0001FFC2220FDF754FADDED207A0020B8EE37
:1040C000E70AFDF7F1F901A82D491AF051FC01A802
:1040D0000021FDF7D3F801A81AF00AFC01A82F4926
:1040E0001AF046FC002101A8FDF7C8F801A81AF053
:1040F000FFFB2220FDF734FADDED217A0020B8EE37
:10410000670AFDF7D1F901A81D491AF031FC01A891
:104110000021FDF7B3F801A81AF0EAFB01A8204935
:104120001AF026FC01A80021FDF7A8F801A81AF052
:10413000DFFB01A81B491AF01BFC01A80021FDF7B9
:104140009DF801A81AF0D4FB01A817491AF010FC39
:1041500001A80021FDF792F801A81AF0C9FB01A8F7
:1041600010491AF005FC01A80021FDF787F801A805
:104170001AF0BEFB2EB070BDE413FF1FA85502005D
:1041800074500200BC550200D0550200E4550200F4
:10419000F85502000C560200205602003456020068
:1041A0004C560200604E02006856020070B5DA4BB1
:1041B0001B6884B00A2B00F2AD81DFE813F05903CD
:1041C000AB0149045404C204AB01E9042B064B07BC
:1041D0000B00D101D149D24D68461AF0C9FB00212C
:1041E0006846FDF74BF868461AF082FB2220FDF77F
:1041F000B7F9D5ED0C7A0020B8EEE70AFDF754F9CF
:10420000C84968461AF0B4FB00216846FDF736F845
:1042100068461AF06DFBC44968461AF0A9FB0021F4
:104220006846FDF72BF868461AF062FB2220FDF77E
:1042300097F9D5ED147A0020B8EE670AFDF734F946
:10424000B84968461AF094FB00216846FDF716F855
:1042500068461AF04DFBB54968461AF089FB002103
:104260006846FDF70BF868461AF042FB2220FDF77E
:1042700077F9D5ED107A0020B8EEE70AFDF714F9CA
:10428000A84968461AF074FB00216846FCF7F6FF5F
:1042900068461AF02DFBA64968461AF069FB002112
:1042A0006846FCF7EBFF68461AF022FB2220FDF778
:1042B00057F9D5ED077A0020B8EEE70AFDF7F4F8D4
:1042C000984968461AF054FB00216846FCF7D6FF6F
:1042D00068461AF00DFB974968461AF049FB002121
:1042E0006846FCF7CBFF68461AF002FB2220FDF778
:1042F00037F995ED080A0020FDF7D6F88949684698
:104300001AF036FB00216846FCF7B8FF68461AF041
:10431000EFFA894968461AF02BFB00216846FCF742
:10432000ADFF68461AF0E4FA2220FDF719F995ED81
:104330000B0A0020FDF7B8F87A4968461AF018FB16
:1043400068460021FCF79AFF68461AF0D1FAAE6A77
:104350006C46002E02F0BB80012E23D177496846BF
:104360001AF006FB00216846FCF788FF68461AF041
:10437000BFFA2220FDF7F4F8714968461AF0F8FAFE
:1043800000216846FCF77AFF68461AF0B1FA6549E1
:1043900068461AF0EDFA68460021FCF76FFF6846A0
:1043A0001AF0A6FA6B6A022B02F08080032B23D14D
:1043B000644920461AF0DCFA00212046FCF75EFF33
:1043C00020461AF095FA2220FDF7CAF85E492046E9
:1043D0001AF0CEFA00212046FCF750FF20461AF0D2
:1043E00087FA504920461AF0C3FA20460021FCF70C
:1043F00045FF20461AF07CFA2B68494D012B00F04E
:10440000B387C0F01C87022B40F084804F492046C0
:104410001AF0AEFA00212046FCF730FF20461AF0D1
:1044200067FA2220FDF79CF8494920461AF0A0FAC5
:1044300000212046FCF722FF20461AF059FA39499C
:1044400020461AF095FA00212046FCF717FF204677
:104450001AF04EFA3F4920461AF08AFA0021204607
:10446000FCF70CFF20461AF043FA2220FDF778F8FB
:10447000D5ED0F7A0020B8EEE70AFDF715F82949C7
:1044800020461AF075FA00212046FCF7F7FE204678
:104490001AF02EFA304920461AF06AFA0021204616
:1044A000FCF7ECFE20461AF023FA2220FDF758F81C
:1044B000D5ED177A0020B8EE670AFCF7F5FF194929
:1044C00020461AF055FA00212046FCF7D7FE204678
:1044D0001AF00EFA214920461AF04AFA0021204625
:1044E000FCF7CCFE20461AF003FA2220FDF738F83C
:1044F00095ED130A0020B8EEC00AFCF7D5FF094974
:1045000020461AF035FA20460021FCF7B7FE204677
:104510001AF0EEF904B070BD4C07FF1F8056020080
:10452000F813FF1F7450020094560200A8560200B0
:104530000C570200205702006C5702009C570200E3
:10454000045A020080570200D4570200BC560200F1
:10455000785D0200D0560200E4560200F8560200D0
:10456000B549B64C68461AF003FA00216846FCF7D4
:1045700085FE68461AF0BCF92220FCF7F1FFD4ED65
:10458000007A0020B8EEE70AFCF78EFFAC496846D7
:104590001AF0EEF900216846FCF770FE68461AF042
:1045A000A7F9A84968461AF0E3F900216846FCF724
:1045B00065FE68461AF09CF92220FCF7D1FFD4ED85
:1045C000047A0020B8EE670AFCF76EFF9C49684643
:1045D0001AF0CEF900216846FCF750FE68461AF042
:1045E00087F9994968461AF0C3F900216846FCF733
:1045F00045FE68461AF07CF92220FCF7B1FFD4EDA5
:10460000087A0020B8EEE70AFCF74EFF8C496846AE
:104610001AF0AEF900216846FCF730FE68461AF041
:1046200067F98A4968461AF0A3F900216846FCF741
:1046300025FE68461AF05CF92220FCF791FFD4EDC4
:104640000C7A0020B8EEE70AFCF72EFF7C4968469A
:104650001AF08EF900216846FCF710FE68461AF041
:1046600047F97B4968461AF083F900216846FCF750
:1046700005FE68461AF03CF92220FCF771FFD4EDE4
:104680000D7A0020B8EEE70AFCF70EFF6C49684689
:104690001AF06EF968460021FCF7F0FD68461AF042
:1046A00027F9A36B012B02F03E83C2F08782022B15
:1046B0007FF430AF674968461AF05AF9002168461E
:1046C000FCF7DCFD68461AF013F92220FCF748FFDE
:1046D000614968461AF04CF900216846FCF7CEFDA6
:1046E00068461AF005F9564968461AF041F9002162
:1046F0006846FCF7C3FD68461AF0FAF85749684661
:104700001AF036F900216846FCF7B8FD68461AF041
:10471000EFF82220FCF724FFD4ED037A0020B8EE56
:10472000670AFCF7C1FE464968461AF021F90021E4
:104730006846FCF7A3FD68461AF0DAF8484968466F
:104740001AF016F900216846FCF798FD68461AF041
:10475000CFF82220FCF704FFD4ED077A0020B8EE52
:10476000670AFCF7A1FE364968461AF001F90021F4
:104770006846FCF783FD68461AF0BAF8394968467E
:104780001AF0F6F800216846FCF778FD68461AF042
:10479000AFF82220FCF7E4FED4ED0B7A0020B8EE4F
:1047A000E70AFCF781FE264968461AF0E1F8002185
:1047B0006846FCF763FD68461AF09AF82A4968468D
:1047C0001AF0D6F800216846FCF758FD68461AF042
:1047D0008FF82220FCF7C4FE94ED160A0020FCF7A7
:1047E00063FE174968461AF0C3F800216846FCF7D3
:1047F00045FD68461AF07CF81C4968461AF0B8F87E
:1048000000216846FCF73AFD68461AF071F822204C
:10481000FCF7A6FE94ED150A0020FCF745FE0849BA
:1048200068461AF0A5F800216846FCF727FD68469F
:104830001AF05EF804B070BD80560200D012FF1F5F
:104840007450020094560200A85602000C57020051
:1048500020570200BC560200785D0200D0560200CC
:10486000E4560200F85602006C5702009C57020002
:10487000BA49BB4C68461AF07BF800216846FCF741
:10488000FDFC68461AF034F82220FCF769FED4EDEE
:10489000017A0020B8EEE70AFCF706FEB149684647
:1048A0001AF066F800216846FCF7E8FC68461AF042
:1048B0001FF8AD4968461AF05BF800216846FCF71E
:1048C000DDFC68461AF014F82220FCF749FED4ED0E
:1048D000097A0020B8EEE70AFCF7E6FDA149684630
:1048E0001AF046F800216846FCF7C8FC684619F043
:1048F000FFFF9E4968461AF03BF800216846FCF726
:10490000BDFC684619F0F4FF2220FCF729FED4ED27
:10491000057A0020B8EEE70AFCF7C6FD9149684623
:104920001AF026F868460021FCF7A8FC684619F042
:10493000DFFF256B012D01F05086022D01F0C686A8
:10494000002D7FF4E7AD8A4968461AF011F8294630
:104950006846FCF793FC684619F0CAFF2220FCF772
:10496000FFFD844968461AF003F829466846FCF7BB
:1049700085FC684619F0BCFF7A49684619F0F8FFD3
:1049800029466846FCF77AFC684619F0B1FF7A4977
:10499000684619F0EDFF29466846FCF76FFC68464B
:1049A00019F0A6FF2220FCF7DBFDD4ED027A2846A1
:1049B000B8EEE70AFCF778FD6A49684619F0D8FFB7
:1049C00029466846FCF75AFC684619F091FF6B4986
:1049D000684619F0CDFF29466846FCF74FFC68464B
:1049E00019F086FF2220FCF7BBFDD4ED0A7A284699
:1049F000B8EEE70AFCF758FD5A49684619F0B8FFC7
:104A000029466846FCF73AFC684619F071FF5C4994
:104A1000684619F0ADFF29466846FCF72FFC68464A
:104A200019F066FF2220FCF79BFD94ED060A28464C
:104A3000B8EEC00AFCF738FD4A49684619F098FFFD
:104A400068462946FCF71AFC684619F051FF61E5F3
:104A50004C4C236B032B3FF65DADDFE813F00B07E7
:104A6000960621067C053D49474D684619F080FFB2
:104A700000216846FCF702FC684619F039FF222045
:104A8000FCF76EFDD5ED017A0020B8EEE70AFCF7E1
:104A90000BFD3449684619F06BFF00216846FCF7AE
:104AA000EDFB684619F024FF2F49684619F060FFB6
:104AB00000216846FCF7E2FB684619F019FF222046
:104AC000FCF74EFDD5ED037A0020B8EE670AFCF73F
:104AD000EBFC2449684619F04BFF00216846FCF7BF
:104AE000CDFB684619F004FF2049684619F040FFE5
:104AF00000216846FCF7C2FB684619F0F9FE222047
:104B0000FCF72EFDD5ED027A0020B8EEE70AFCF79F
:104B1000CBFC1449684619F02BFF68460021FCF7CE
:104B2000ADFB684619F0E4FE2B68013B6C46042B94
:104B30003FF6F0ACDFE813F0CD071307BC07AB0777
:104B40009A07124C2368052B3FF6E4ACDFE813F01C
:104B50008E081E0B740ADD094609F807805602000C
:104B60009818FF1F7450020094560200A8560200C5
:104B7000BC560200B05C0200D0560200E4560200AF
:104B8000F8560200AC13FF1F6C15FF1F9815FF1F8E
:104B90009449954D684619F0EBFE00216846FCF7F4
:104BA0006DFB684619F0A4FE2220FCF7D9FCD5ED78
:104BB000017A0020B8EEE70AFCF776FC8B496846DC
:104BC00019F0D6FE00216846FCF758FB684619F03C
:104BD0008FFE8749684619F0CBFE00216846FCF736
:104BE0004DFB684619F084FE2220FCF7B9FCD5ED98
:104BF000027A0020B8EE670AFCF756FC7B4968464B
:104C000019F0B6FE00216846FCF738FB684619F03B
:104C10006FFE7849684619F0ABFE00216846FCF744
:104C20002DFB684619F064FE2220FCF799FCD5EDB7
:104C3000097A0020B8EEE70AFCF736FC6B496846B3
:104C400019F096FE68460021FCF718FB684619F03B
:104C50004FFE6B6B012B6C4600F04C87C1F0158446
:104C6000302B01F01284312B00F0448762495E4EF4
:104C7000204619F07DFE00212046FCF7FFFA204671
:104C800019F036FE2220FCF76BFC95ED0F0A002090
:104C9000FCF70AFC5549204619F06AFE002120461F
:104CA000FCF7ECFA204619F023FE5449204619F08F
:104CB0005FFE00212046FCF7E1FA204619F018FEBD
:104CC0002220FCF74DFC95ED0E0A0020FCF7ECFBD2
:104CD0004649204619F04CFE00212046FCF7CEFA4A
:104CE000204619F005FE2B68012B01F0E386C1F088
:104CF0006B86022B7FF40EAC4149204619F038FE3A
:104D000000212046FCF7BAFA204619F0F1FD2220D6
:104D1000FCF726FC3B49204619F02AFE00212046DC
:104D2000FCF7ACFA204619F0E3FD3049204619F0B3
:104D30001FFE00212046FCF7A1FA204619F0D8FDFD
:104D40003149204619F014FE00212046FCF796FA5E
:104D5000204619F0CDFD2220FCF702FCD6ED077AA3
:104D60000020B8EEE70AFCF79FFB2049204619F027
:104D7000FFFD00212046FCF781FA204619F0B8FD1E
:104D80002249204619F0F4FD00212046FCF776FA6E
:104D9000204619F0ADFD2220FCF7E2FBD6ED087AA3
:104DA0000020B8EE670AFCF77FFB1049204619F097
:104DB000DFFD00212046FCF761FA204619F098FD3E
:104DC0001349204619F0D4FD00212046FCF756FA7D
:104DD000204619F08DFD2220FCF7C2FB96ED0C0A4F
:104DE000FFF788BB805602006C13FF1F745002004F
:104DF00094560200A8560200205702006C57020089
:104E0000BC560200785D0200D0560200E456020053
:104E1000F85602008449854D684619F0A9FD002125
:104E20006846FCF72BFA684619F062FD2220FCF771
:104E300097FBD5ED007A0020B8EEE70AFCF734FBCB
:104E40007B49684619F094FD00216846FCF716FA84
:104E5000684619F04DFD7749684619F089FD002133
:104E60006846FCF70BFA684619F042FD2220FCF771
:104E700077FBD5ED087A0020B8EE670AFCF714FB43
:104E80006B49684619F074FD00216846FCF7F6F995
:104E9000684619F02DFD6849684619F069FD002142
:104EA0006846FCF7EBF9684619F022FD2220FCF772
:104EB00057FBD5ED047A0020B8EEE70AFCF7F4FAC8
:104EC0005B49684619F054FD00216846FCF7D6F9A5
:104ED000684619F00DFD5949684619F049FD002151
:104EE0006846FCF7CBF9684619F002FD2220FCF772
:104EF00037FBD5ED147A0020B8EE670AFCF7D4FA38
:104F00004B49684619F034FD68460021FCF7B6F9B4
:104F1000684619F0EDFCEE6C6C46002E01F0338211
:104F2000012E00F09782AB6C404D012B01F0D6842E
:104F3000C1F04584022B7FF4EDAA4149204619F0C7
:104F400017FD00212046FCF799F9204619F0D0FC06
:104F50002220FCF705FB3B49204619F009FD002102
:104F60002046FCF78BF9204619F0C2FC3049204658
:104F700019F0FEFC00212046FCF780F9204619F0CC
:104F8000B7FC3149204619F0F3FC00212046FCF71C
:104F900075F9204619F0ACFC2220FCF7E1FAD5EDBA
:104FA000037A0020B8EEE70AFCF77EFA2049204693
:104FB00019F0DEFC00212046FCF760F9204619F0CC
:104FC00097FC2249204619F0D3FC00212046FCF72B
:104FD00055F9204619F08CFC2220FCF7C1FAD5EDDA
:104FE0000B7A0020B8EE670AFCF75EFA10492046FB
:104FF00019F0BEFC00212046FCF740F9204619F0CC
:1050000077FC1349204619F0B3FC00212046FCF739
:1050100035F9204619F06CFC2220FCF7A1FA95ED39
:10502000070AFFF767BA00BF805602006414FF1F2B
:105030007450020094560200A856020080570200E5
:10504000BC560200785D0200D0560200E456020011
:10505000F8560200B549B64D684619F089FC0021A2
:105060006846FCF70BF9684619F042FC2220FCF771
:1050700077FAD5ED0C7A0020B8EEE70AFCF714FABF
:10508000AC49684619F074FC00216846FCF7F6F854
:10509000684619F02DFCA849684619F069FC002102
:1050A0006846FCF7EBF8684619F022FC2220FCF772
:1050B00057FAD5ED147A0020B8EE670AFCF7F4F938
:1050C0009C49684619F054FC00216846FCF7D6F864
:1050D000684619F00DFC9949684619F049FC002111
:1050E0006846FCF7CBF8684619F002FC2220FCF772
:1050F00037FAD5ED107A0020B8EEE70AFCF7D4F9BC
:105100008C49684619F034FC00216846FCF7B6F873
:10511000684619F0EDFB8A49684619F029FC002120
:105120006846FCF7ABF8684619F0E2FB2220FCF772
:1051300017FAD5ED047A0020B8EEE70AFCF7B4F9C7
:105140007C49684619F014FC00216846FCF796F883
:10515000684619F0CDFB7B49684619F009FC00212F
:105160006846FCF78BF8684619F0C2FB2220FCF772
:10517000F7F995ED030A0020FCF796F96D496846AA
:1051800019F0F6FB00216846FCF778F8684619F03C
:10519000AFFB6D49684619F0EBFB00216846FCF750
:1051A0006DF8684619F0A4FB2220FCF7D9F995EDBB
:1051B000060A0020FCF778F95E49684619F0D8FB2A
:1051C00068460021FCF75AF8684619F091FB6E69B1
:1051D0006C46002E01F0CA81012E23D15B4968463E
:1051E00019F0C6FB00216846FCF748F8684619F03C
:1051F0007FFB2220FCF7B4F95549684619F0B8FB4B
:1052000000216846FCF73AF8684619F071FB4949F5
:10521000684619F0ADFB68460021FCF72FF8684698
:1052200019F066FBAB68023B052B3FF6E5A8DFE80B
:1052300013F0440888087708660855089908454916
:10524000204619F095FB00212046FCF717F8204670
:1052500019F04EFB2220FCF783F93F49204619F054
:1052600087FB00212046FCF709F8204619F040FB97
:105270003049204619F07CFB00212046FBF7FEFF59
:10528000204619F035FB3549204619F071FB002105
:105290002046FBF7F3FF204619F02AFB2220FCF7FB
:1052A0005FF9D5ED0D7A0020B8EEE70AFCF7FCF8BF
:1052B0002049204619F05CFB00212046FBF7DEFF69
:1052C000204619F015FB2649204619F051FB002114
:1052D0002046FBF7D3FF204619F00AFB2220FCF7FB
:1052E0003FF9D5ED157A0020B8EE670AFCF7DCF837
:1052F0001049204619F03CFB00212046FBF7BEFF79
:10530000204619F0F5FA1749204619F031FB002123
:105310002046FBF7B3FF204619F0EAFA2220FCF7FB
:105320001FF995ED110AFFF7E5B800BF805602009E
:10533000F813FF1F7450020094560200A856020092
:105340000C570200205702006C5702009C570200C5
:10535000045A0200BC560200B05C0200D0560200A3
:10536000E4560200F8560200BE49204619F000FB40
:1053700000212046FBF782FF204619F0B9FA2220CF
:10538000FCF7EEF8B849204619F0F2FA0021204661
:10539000FBF774FF204619F0ABFAB449204619F028
:1053A000E7FA00212046FBF769FF204619F0A0FA32
:1053B000AF49204619F0DCFA00212046FBF75EFFDA
:1053C000204619F095FA2220FCF7CAF8D5ED0E7A9E
:1053D0000020B8EEE70AFCF767F8A449204619F068
:1053E000C7FA00212046FBF749FF204619F080FA52
:1053F000A049204619F0BCFA00212046FBF73EFFE9
:10540000204619F075FA2220FCF7AAF8D5ED167A95
:105410000020B8EE670AFCF747F89449204619F0D7
:10542000A7FA00212046FBF729FF204619F060FA71
:105430009149204619F09CFA00212046FBF71EFFF7
:10544000204619F055FA2220FCF78AF895ED120A49
:10545000FFF750B88949684619F08AFA0021684672
:10546000FBF70CFF684619F043FA2220FCF778F8A6
:105470008349684619F07CFA00216846FBF7FEFE76
:10548000684619F035FA7949684619F071FA002131
:105490006846FBF7F3FE684619F02AFA7949684630
:1054A00019F066FA00216846FBF7E8FE684619F035
:1054B0001FFA2220FCF754F8D5ED0C7A0020B8EE44
:1054C000E70AFBF7F1FF6949684619F051FA002134
:1054D0006846FBF7D3FE684619F00AFA6A4968463F
:1054E00019F046FA00216846FBF7C8FE684619F035
:1054F000FFF92220FCF734F895ED0F0A0020FBF7A6
:10550000D3FF5A49684619F033FA00216846FBF781
:10551000B5FE684619F0ECF95C49684619F028FABE
:1055200000216846FBF7AAFE684619F0E1F922203F
:10553000FCF716F895ED0E0A0020FBF7B5FF4B4976
:10554000684619F015FA68460021FBF797FE684691
:1055500019F0CEF9E7E44349684619F009FA002149
:105560006846FBF78BFE684619F0C2F92220FBF76C
:10557000F7FF4749684619F0FBF900216846FBF739
:105580007DFE684619F0B4F93849684619F0F0F91B
:1055900000216846FBF772FE684619F0A9F93D49FB
:1055A000684619F0E5F900216846FBF767FE684692
:1055B00019F09EF92220FBF7D3FFD4ED017A0020E9
:1055C000B8EEE70AFBF770FF2849684619F0D0F9F2
:1055D00000216846FBF752FE684619F089F92E490A
:1055E000684619F0C5F900216846FBF747FE684692
:1055F00019F07EF92220FBF7B3FFD4ED097A0020E1
:10560000B8EEE70AFBF750FF1849684619F0B0F901
:1056100000216846FBF732FE684619F069F91F4918
:10562000684619F0A5F900216846FBF727FE684691
:1056300019F05EF92220FBF793FF94ED050AB8EE0E
:10564000C00A0020FBF730FF6846084919F090F9BE
:1056500068460021FBF712FE684619F049F904B0CC
:1056600070BD00BFBC560200787E0200745002007C
:10567000D0560200E4560200F85602000C57020011
:10568000045A0200205702006C5702009C57020087
:10569000445C02008056020094560200A8560200A4
:1056A000E549684619F064F900216846FBF7E6FD14
:1056B000684619F01DF92220FBF752FFDF496846C2
:1056C00019F056F900216846FBF7D8FD684619F035
:1056D0000FF9DB49684619F04BF900216846FBF7E2
:1056E000CDFD684619F004F9D649684619F040F92D
:1056F00000216846FBF7C2FD684619F0F9F8222040
:10570000FBF72EFFD4ED047A0020B8EEE70AFBF792
:10571000CBFECB49684619F02BF900216846FBF710
:10572000ADFD684619F0E4F8C749684619F020F95C
:1057300000216846FBF7A2FD684619F0D9F822203F
:10574000FBF70EFFD4ED007A0020B8EEE70AFBF776
:10575000ABFEBB49684619F00BF900216846FBF720
:105760008DFD684619F0C4F8B849684619F000F98B
:1057700000216846FBF782FD684619F0B9F822203F
:10578000FBF7EEFE94ED080A59E7AB49684619F0BD
:10579000EFF800216846FBF771FD684619F0A8F89C
:1057A0002220FBF7DDFEAA49684619F0E1F8002146
:1057B0006846FBF763FD684619F09AF8A049684609
:1057C00019F0D6F800216846FBF758FD684619F035
:1057D0008FF89C49684619F0CBF800216846FBF722
:1057E0004DFD684619F084F82220FBF7B9FED4ED90
:1057F000037A0020B8EEE70AFBF756FE90496846A8
:1058000019F0B6F800216846FBF738FD684619F034
:105810006FF88D49684619F0ABF800216846FBF730
:105820002DFD684619F064F82220FBF799FED4EDAF
:105830000B7A0020B8EEE70AFBF736FE804968468F
:1058400019F096F800216846FBF718FD684619F034
:105850004FF87E49684619F08BF800216846FBF73F
:105860000DFD684619F044F82220FBF779FE94ED0F
:10587000070AE4E67049684619F07AF8002168469C
:10588000FBF7FCFC684619F033F82220FBF768FEB2
:105890007049684619F06CF800216846FBF7EEFC89
:1058A000684619F025F86649684619F061F8002144
:1058B0006846FBF7E3FC684619F01AF86149684648
:1058C00019F056F800216846FBF7D8FC684619F035
:1058D0000FF82220FBF744FED4ED027A0020B8EE48
:1058E000E70AFBF7E1FD5649684619F041F8002147
:1058F0006846FBF7C3FC684618F0FAFF5249684651
:1059000019F036F800216846FBF7B8FC684618F035
:10591000EFFF2220FBF724FED4ED0A7A0020B8EE38
:10592000E70AFBF7C1FD4649684619F021F8002156
:105930006846FBF7A3FC684618F0DAFF434968465F
:1059400019F016F800216846FBF798FC684618F035
:10595000CFFF2220FBF704FE94ED060A6FE63649DE
:105960003D4D684619F004F800216846FBF786FCB7
:10597000684618F0BDFF2220FBF7F2FD37492046AC
:1059800018F0F6FF00212046FBF778FC204618F0BF
:10599000AFFF2B49204618F0EBFF00212046FBF714
:1059A0006DFC204618F0A4FF2D49204618F0E0FFBA
:1059B00000212046FBF762FC204618F099FF2220C8
:1059C000FBF7CEFDD5E904011BF0D0F900EE100A7B
:1059D0000020FBF769FD1A49204618F0C9FF002195
:1059E0002046FBF74BFC204618F082FF6B68012B2A
:1059F00007D0C0F0E185302B00F0DE85312B7EF43E
:105A000089AD1849204618F0B3FF00212046FBF766
:105A100035FC204618F06CFF2220FBF7A1FD12494F
:105A2000204618F0A5FF20460021FBF727FC204662
:105A300018F05EFFFEF763BDBC560200785D020001
:105A400074500200D0560200E4560200F8560200DC
:105A5000787E0200B05C02003816FF1F745B020003
:105A60000C570200205702003C570200CA49CB4D98
:105A7000684618F07DFF00216846FBF7FFFB68468B
:105A800018F036FF2220FBF76BFDC54977E7C249C6
:105A9000C44D684618F06CFF00216846FBF7EEFB2A
:105AA000684618F025FF2220FBF75AFDBE4966E73D
:105AB000B949BE4D684618F05BFF00216846FBF708
:105AC000DDFB684618F014FF2220FBF749FDB849BA
:105AD00055E7B149B74D684618F04AFF00216846BE
:105AE000FBF7CCFB684618F003FF2220FBF738FDDC
:105AF000B14944E7B149204618F03AFF0021204659
:105B0000FBF7BCFB204618F0F3FE2220FBF728FD34
:105B1000AB49204618F02CFF00212046FBF7AEFBD6
:105B2000204618F0E5FEA749204618F021FF204640
:105B30000021FBF7A3FB204618F0DAFEFFF796B82A
:105B40009549684618F014FF00216846FBF796FB5C
:105B5000684618F0CDFE2220FBF702FD9A49684600
:105B600018F006FF00216846FBF788FB684618F02E
:105B7000BFFE9449684618F0FBFE00216846FBF71B
:105B80007DFB684618F0B4FE9049684618F0F0FEB8
:105B900000216846FBF772FB684618F0A9FE222038
:105BA000FBF7DEFCD4ED077A0020B8EEE70AFBF73E
:105BB0007BFC8449684618F0DBFE00216846FBF751
:105BC0005DFB684618F094FE8149684618F0D0FEE7
:105BD00000216846FBF752FB684618F089FE222038
:105BE000FBF7BEFCD4ED087A0020B8EE670AFBF79D
:105BF0005BFC7449684618F0BBFE00216846FBF761
:105C00003DFB684618F074FE7249684618F0B0FE15
:105C100000216846FBF732FB684618F069FE222037
:105C2000FBF79EFCD4ED097A0020B8EEE70AFBF7FB
:105C30003BFC6449684618F09BFE00216846FBF770
:105C40001DFB684618F054FE5C49684618F090FE4B
:105C500000216846FBF712FB684618F049FE222037
:105C6000FBF77EFC002094ED0F0AEBE44A496846FE
:105C700018F07EFE00216846FBF700FB684618F02E
:105C800037FE2220FBF76CFC5349684618F070FE83
:105C900000216846FBF7F2FA684618F029FE4949E8
:105CA000684618F065FE00216846FBF7E7FA68468B
:105CB00018F01EFE4549684618F05AFE0021684655
:105CC000FBF7DCFA684618F013FE2220FBF748FCCD
:105CD000D4ED017A0020B8EEE70AFBF7E5FB39497D
:105CE000684618F045FE00216846FBF7C7FA68468B
:105CF00018F0FEFD3649684618F03AFE0021684665
:105D0000FBF7BCFA684618F0F3FD2220FBF728FCED
:105D1000D4ED027A0020B8EE670AFBF7C5FB2949EB
:105D2000684618F025FE00216846FBF7A7FA68468A
:105D300018F0DEFD2749684618F01AFE0021684673
:105D4000FBF79CFA684618F0D3FD2220FBF708FC0D
:105D5000D4ED037A0020B8EEE70AFBF7A5FB19495A
:105D6000684618F005FE00216846FBF787FA68468A
:105D700018F0BEFD1149684618F0FAFD002168468A
:105D8000FBF77CFA684618F0B3FD2220FBF7E8FB2E
:105D9000002094ED0A0A55E4BC5602008016FF1F4D
:105DA000045C02006816FF1F645602005016FF1FB5
:105DB000A45B0200B814FF1F587502000C570200C4
:105DC000645702007450020058570200D056020077
:105DD000E4560200F856020044570200E2496846C1
:105DE00018F0C6FD00216846FBF748FA684618F02F
:105DF0007FFD2220FBF7B4FBDC49684618F0B8FDB4
:105E000000216846FBF73AFA684618F071FDD84958
:105E1000684618F0ADFD00216846FBF72FFA68468A
:105E200018F066FDD349684618F0A2FD00216846C7
:105E3000FBF724FA684618F05BFD2220FBF790FB85
:105E4000D4ED077A0020B8EEE70AFBF72DFBC8492E
:105E5000684618F08DFD00216846FBF70FFA68468A
:105E600018F046FDC449684618F082FD00216846D6
:105E7000FBF704FA684618F03BFD2220FBF770FBA5
:105E8000D4ED087A0020B8EE670AFBF70DFBB8499D
:105E9000684618F06DFD00216846FBF7EFF968468B
:105EA00018F026FDB549684618F062FD00216846E5
:105EB000FBF7E4F9684618F01BFD2220FBF750FBC6
:105EC000D4ED097A0020B8EEE70AFBF7EDFAA8490D
:105ED000684618F04DFD00216846FBF7CFF968468B
:105EE00018F006FDA649684618F042FD00216846F4
:105EF000FBF7C4F9684618F0FBFC2220FBF730FBE7
:105F0000002094ED0C0AFFF79DBB9749684618F0F6
:105F10002FFD00216846FBF7B1F9684618F0E8FC50
:105F20002220FBF71DFB9749684618F021FD002150
:105F30006846FBF7A3F9684618F0DAFC8C49684616
:105F400018F016FD00216846FBF798F9684618F02E
:105F5000CFFC8849684618F00BFD00216846FBF726
:105F60008DF9684618F0C4FC2220FBF7F9FAD4ED4D
:105F7000047A0020B8EEE70AFBF796FA7C496846F7
:105F800018F0F6FC00216846FBF778F9684618F02F
:105F9000AFFC7949684618F0EBFC00216846FBF736
:105FA0006DF9684618F0A4FC2220FBF7D9FAD4ED6D
:105FB000057A0020B8EE670AFBF776FA6C49684666
:105FC00018F0D6FC00216846FBF758F9684618F02F
:105FD0008FFC6A49684618F0CBFC00216846FBF745
:105FE0004DF9684618F084FC2220FBF7B9FAD4ED8D
:105FF000067A0020B8EEE70AFBF756FA5C496846D5
:1060000018F0B6FC00216846FBF738F9684618F02E
:106010006FFC5B49684618F0ABFC00216846FBF753
:106020002DF9684618F064FC2220FBF799FA00204D
:1060300094ED0E0AFFF706BB4B49684618F098FC32
:1060400000216846FBF71AF9684618F051FC222037
:10605000FBF786FA4C49684618F08AFC002168462E
:10606000FBF70CF9684618F043FC4149684618F004
:106070007FFC00216846FBF701F9684618F038FC00
:106080003C49684618F074FC00216846FBF7F6F8B6
:10609000684618F02DFC2220FBF762FAD4ED047A52
:1060A0000020B8EEE70AFBF7FFF93149684618F01F
:1060B0005FFC00216846FBF7E1F8684618F018FC21
:1060C0002D49684618F054FC00216846FBF7D6F8C5
:1060D000684618F00DFC2220FBF742FAD4ED057A51
:1060E0000020B8EE670AFBF7DFF92149684618F08F
:1060F0003FFC00216846FBF7C1F8684618F0F8FB42
:106100001E49684618F034FC00216846FBF7B6F8D3
:10611000684618F0EDFB2220FBF722FAD4ED067A50
:106120000020B8EEE70AFBF7BFF91149684618F0FE
:106130001FFC00216846FBF7A1F8684618F0D8FB61
:106140000F49684618F014FC00216846FBF796F8E2
:10615000684618F0CDFB2220FBF702FA002094EDF0
:106160000B0AFFF76FBA00BFBC560200545702007B
:1061700074500200D0560200E4560200F8560200A5
:106180000C570200505702004C570200E349684682
:1061900018F0EEFB00216846FBF770F8684618F02F
:1061A000A7FB2220FBF7DCF9DD49684618F0E0FB8D
:1061B00000216846FBF762F8684618F099FBD94958
:1061C000684618F0D5FB00216846FBF757F868468B
:1061D00018F08EFBD449684618F0CAFB00216846C7
:1061E000FBF74CF8684618F083FB2220FBF7B8F960
:1061F000D4ED017A0020B8EEE70AFBF755F9C9495A
:10620000684618F0B5FB00216846FBF737F868468A
:1062100018F06EFBC549684618F0AAFB00216846D5
:10622000FBF72CF8684618F063FB2220FBF798F97F
:10623000D4ED027A0020B8EE670AFBF735F9B949C8
:10624000684618F095FB00216846FBF717F868468A
:1062500018F04EFBB649684618F08AFB00216846E4
:10626000FBF70CF8684618F043FB2220FBF778F99F
:10627000D4ED037A0020B8EEE70AFBF715F9A94937
:10628000684618F075FB00216846FAF7F7FF684684
:1062900018F02EFBA749684618F06AFB00216846F3
:1062A000FAF7ECFF684618F023FB2220FBF758F9B9
:1062B000002094ED0D0AFFF7C5B99F49204618F05C
:1062C00057FB00212046FAF7D9FF204618F010FBB3
:1062D0002220FBF745F99949FEF779B896492046FF
:1062E00018F046FB00212046FAF7C8FF204618F0B8
:1062F000FFFA2220FBF734F99149FEF768B88E497E
:10630000204618F035FB00212046FAF7B7FF20465B
:1063100018F0EEFA2220FBF723F98A49FEF757B866
:106320008549204618F024FB00212046FAF7A6FFF5
:10633000204618F0DDFA2220FBF712F98249FEF719
:1063400046B87D49204618F013FB00212046FAF795
:1063500095FF204618F0CCFA2220FBF701F97B4983
:10636000FEF735B87449204618F002FB002120469C
:10637000FAF784FF204618F0BBFA2220FBF7F0F86A
:106380007349FEF724B86B49684618F0F1FA3146B4
:106390006846FAF773FF684618F0AAFA2220FBF75E
:1063A000DFF86C49684618F0E3FA31466846FAF7B8
:1063B00065FF684618F09CFA5A49684618F0D8FA02
:1063C00031466846FAF75AFF684618F091FA624972
:1063D000684618F0CDFA31466846FAF74FFF68462E
:1063E00018F086FA2220FBF7BBF8D5ED0D7A30467F
:1063F000B8EEE70AFBF758F84A49684618F0B8FAC9
:1064000031466846FAF73AFF684618F071FA534980
:10641000684618F0ADFA31466846FAF72FFF68462D
:1064200018F066FA2220FBF79BF895ED110A30462A
:10643000FBF73AF83B49684618F09AFA3146684645
:10644000FAF71CFF684618F053FA4549684618F0F9
:106450008FFA31466846FAF711FF684618F048FA95
:106460002220FBF77DF895ED100A3046FBF71CF86B
:106470002C49684618F07CFA68463146FAF7FEFE69
:10648000684618F035FAFEF74EBD2A49204618F046
:106490006FFA00212046FAF7F1FE204618F028FA9C
:1064A0002220FBF75DF82F49FFF733BB2249204636
:1064B00018F05EFA00212046FAF7E0FE204618F0B8
:1064C00017FA2220FBF74CF82749FDF780BF244933
:1064D000684618F04DFA31466846FAF7CFFE68462E
:1064E00018F006FA2220FBF73BF81A49684618F024
:1064F0003FFA31466846FAF7C1FE684618F0F8F9E7
:106500000849684618F034FA68463146FAF7B6FE8C
:10651000684618F0EDF9FDF745BF00BFBC56020014
:106520004857020074500200D0560200E4560200A0
:10653000F85602000C57020080570200B0570200C4
:10654000C0570200BC570200B8570200B4570200FF
:10655000C457020094570200205702006C570200F3
:106560009C5702005C570200C8570200CF4968469A
:1065700018F0FEF931466846FAF780FE684618F0D2
:10658000B7F92220FAF7ECFFC949684618F0F0F98C
:1065900031466846FAF772FE684618F0A9F9C5490F
:1065A000684618F0E5F968463146FAF767FE68462E
:1065B00018F09EF9FEF736BEBF49204618F0D8F90C
:1065C00000212046FAF75AFE204618F091F92220C1
:1065D000FAF7C6FFB949FFF723BAB949684618F078
:1065E000C7F900216846FAF749FE684618F080F9B5
:1065F0002220FAF7B5FFB349684618F0B9F900212F
:106600006846FAF73BFE684618F072F9A9496846F1
:1066100018F0AEF900216846FAF730FE684618F027
:1066200067F9A949684618F0A3F900216846FAF706
:1066300025FE684618F05CF92220FAF791FFD4EDA8
:10664000037A0020B8EEE70AFAF72EFF9949684668
:1066500018F08EF900216846FAF710FE684618F027
:1066600047F99A49684618F083F900216846FAF715
:1066700005FE684618F03CF92220FAF771FFD4EDC8
:106680000B7A0020B8EEE70AFAF70EFF8949684650
:1066900018F06EF900216846FAF7F0FD684618F028
:1066A00027F98B49684618F063F900216846FAF724
:1066B000E5FD684618F01CF92220FAF751FF94ED29
:1066C000070A0020B8EEC00AFEF7A7B87C49684662
:1066D00018F04EF900216846FAF7D0FD684618F028
:1066E00007F92220FAF73CFF7A49684618F040F98A
:1066F00000216846FAF7C2FD684618F0F9F86D49BE
:10670000684618F035F900216846FAF7B7FD684683
:1067100018F0EEF86C49684618F02AF9002168462E
:10672000FAF7ACFD684618F0E3F82220FAF718FFF4
:10673000D4ED047A0020B8EEE70AFAF7B5FE5D4919
:10674000684618F015F900216846FAF797FD684683
:1067500018F0CEF85D49684618F00AF9002168463D
:10676000FAF78CFD684618F0C3F82220FAF7F8FE15
:10677000D4ED007A0020B8EEE70AFAF795FE4D490D
:10678000684618F0F5F800216846FAF777FD684684
:1067900018F0AEF84E49684618F0EAF8002168464D
:1067A000FAF76CFD684618F0A3F82220FAF7D8FE35
:1067B00094ED080A0020B8EEC00AFEF72EB8404952
:1067C000204618F0D5F800212046FAF757FD20465C
:1067D00018F08EF82220FAF7C3FE3F49204618F041
:1067E000C7F800212046FAF749FD204618F080F846
:1067F0003049204618F0BCF800212046FAF73EFD4B
:10680000204618F075F83049204618F0B1F80021FC
:106810002046FAF733FD204618F06AF82220FAF7EE
:106820009FFED5ED017A0020B8EEE70AFAF73CFEAC
:106830002049204618F09CF800212046FAF71EFD5A
:10684000204618F055F82149204618F091F800210B
:106850002046FAF713FD204618F04AF82220FAF7EE
:106860007FFED5ED097A0020B8EE670AFAF71CFE24
:106870001049204618F07CF800212046FAF7FEFC6B
:10688000204618F035F81249204618F071F800211A
:106890002046FAF7F3FC204618F02AF82220FAF7EF
:1068A0005FFE95ED050AFDF725BE00BF9C5702006F
:1068B000945702007450020020570200345702001F
:1068C000BC560200787E0200D0560200E456020058
:1068D000F8560200785D0200B05C0200B049204624
:1068E00018F046F800212046FAF7C8FC204617F0B9
:1068F000FFFF2220FAF734FEAA49204618F038F8A4
:1069000000212046FAF7BAFC204617F0F1FFA6490D
:10691000204618F02DF800212046FAF7AFFC20465B
:1069200017F0E6FFA149204618F022F80021204682
:10693000FAF7A4FC204617F0DBFF2220FAF710FE3E
:10694000D5ED027A0020B8EEE70AFAF7ADFD9649D8
:10695000204618F00DF800212046FAF78FFC20465B
:1069600017F0C6FF9249204618F002F80021204691
:10697000FAF784FC204617F0BBFF2220FAF7F0FD5F
:10698000D5ED0A7A0020B8EE670AFAF78DFD864940
:10699000204617F0EDFF00212046FAF76FFC204655
:1069A00017F0A6FF8349204617F0E2FF002120469A
:1069B000FAF764FC204617F09BFF2220FAF7D0FD7F
:1069C00095ED060AFDF796BD7549204617F0D0FFF4
:1069D00000212046FAF752FC204617F089FF2220BA
:1069E000FAF7BEFD7449204617F0C2FF0021204689
:1069F000FAF744FC204617F07BFF6B49204617F05E
:106A0000B7FF00212046FAF739FC204617F070FF47
:106A10006649204617F0ACFF00212046FAF72EFC0D
:106A2000204617F065FF2220FAF79AFDD6ED037A8B
:106A30000020B8EEE70AFAF737FD5B49204617F069
:106A400097FF00212046FAF719FC204617F050FF67
:106A50005749204617F08CFF00212046FAF70EFC1C
:106A6000204617F045FF2220FAF77AFDD6ED047A8A
:106A70000020B8EE670AFAF717FD4B49204617F0D9
:106A800077FF00212046FAF7F9FB204617F030FF88
:106A90004849204617F06CFF00212046FAF7EEFB2C
:106AA000204617F025FF2220FAF75AFD96ED0A0A34
:106AB000FDF720BD3A49204617F05AFF0021204635
:106AC000FAF7DCFB204617F013FF2220FAF748FD07
:106AD0003449204617F04CFF00212046FAF7CEFB40
:106AE000204617F005FF3049204617F041FF0021EE
:106AF0002046FAF7C3FB204617F0FAFE2B49204642
:106B000017F036FF00212046FAF7B8FB204617F0B1
:106B1000EFFE2220FAF724FDD6ED057A0020B8EE2C
:106B2000E70AFAF7C1FC2049204617F021FF0021AF
:106B30002046FAF7A3FB204617F0DAFE1C49204650
:106B400017F016FF00212046FAF798FB204617F0B1
:106B5000CFFE2220FAF704FDD6ED067A0020B8EE2B
:106B6000670AFAF7A1FC1049204617F001FF00213F
:106B70002046FAF783FB204617F0BAFE0D4920465F
:106B800017F0F6FE00212046FAF778FB204617F0B2
:106B9000AFFE2220FAF7E4FC96ED0B0AFDF7AABC43
:106BA000BC560200787E020074500200D0560200EB
:106BB000E4560200F8560200B05C0200B449684690
:106BC00017F0D6FE00216846FAF758FB684617F022
:106BD0008FFE2220FAF7C4FCAE49684617F0C8FEC3
:106BE00000216846FAF74AFB684617F081FEAA4979
:106BF000684617F0BDFE00216846FAF73FFB68467D
:106C000017F076FEA549684617F0B2FE00216846E7
:106C1000FAF734FB684617F06BFE2220FAF7A0FC67
:106C2000D4ED017A0020B8EEE70AFAF73DFC9A4964
:106C3000684617F09DFE00216846FAF71FFB68467C
:106C400017F056FE9649684617F092FE00216846F6
:106C5000FAF714FB684617F04BFE2220FAF780FC87
:106C6000D4ED057A0020B8EE670AFAF71DFC8A49D0
:106C7000684617F07DFE00216846FAF7FFFA68467D
:106C800017F036FE8749684617F072FE0021684605
:106C9000FAF7F4FA684617F02BFE2220FAF760FCA8
:106CA000D4ED097A0020B8EEE70AFAF7FDFB7A493D
:106CB000684617F05DFE00216846FAF7DFFA68467D
:106CC00017F016FE7849684617F052FE0021684614
:106CD000FAF7D4FA684617F00BFE2220FAF740FCC8
:106CE00094ED160A0020FAF7DFFB6B49684617F0AF
:106CF0003FFE00216846FAF7C1FA684617F0F8FD32
:106D00006A49684617F034FE00216846FAF7B6FA79
:106D1000684617F0EDFD2220FAF722FC002094EDE2
:106D2000130AFDF77ABD5A49684617F021FE002183
:106D30006846FAF7A3FA684617F0DAFD2220FAF758
:106D40000FFC5B49684617F013FE00216846FAF70E
:106D500095FA684617F0CCFD4F49684617F008FED3
:106D600000216846FAF78AFA684617F0C1FD4B49D8
:106D7000684617F0FDFD00216846FAF77FFA68467D
:106D800017F0B6FD2220FAF7EBFBD4ED027A0020D3
:106D9000B8EE670AFAF788FB3F49684617F0E8FD46
:106DA00000216846FAF76AFA684617F0A1FD3C49E7
:106DB000684617F0DDFD00216846FAF75FFA68467D
:106DC00017F096FD2220FAF7CBFBD4ED067A0020CF
:106DD000B8EE670AFAF768FB2F49684617F0C8FD56
:106DE00000216846FAF74AFA684617F081FD2D49F6
:106DF000684617F0BDFD00216846FAF73FFA68467D
:106E000017F076FD2220FAF7ABFBD4ED0A7A0020CA
:106E1000B8EEE70AFAF748FB1F49684617F0A8FDE5
:106E200000216846FAF72AFA684617F061FD1E4904
:106E3000684617F09DFD00216846FAF71FFA68467C
:106E400017F056FD2220FAF78BFB94ED160A00206E
:106E5000FAF72AFB1049684617F08AFD00216846B8
:106E6000FAF70CFA684617F043FD1049684617F028
:106E70007FFD00216846FAF701FA684617F038FDF1
:106E80002220FAF76DFB002094ED140AFDF7C5BC33
:106E9000BC560200B05C020074500200D0560200E2
:106EA000E4560200F85602006C5702009C5702009C
:106EB000787E02002DE9F043B34DB44CD5F800E0E4
:106EC0002468BEF1010F2DED028B1F4604BFB04BAD
:106ED0001C68ADB006460D46904608A80023012266
:106EE000214613F099FF0FA811F050FD002840F043
:106EF000FF8018A89DF83A30A64908AA11F0FAFDBB
:106F00001A9A9DF86C309DF8641011928DF84830F3
:106F10008DF840101BAA0DF149030DF1560012F82F
:106F2000011F03F8011B8342F9D11F9B169318A878
:106F300011F0FEFC0FA811F029FD8146002836D182
:106F40000123092194488DF83B3016F0B5FE204608
:106F50001BF0D6FA0146204616F0AEFE0F218F48F0
:106F60009FED8F8A16F0A8FE8E4817F035FB8E49EC
:106F700018A817F0FDFC494618A8FAF77FF918A8D9
:106F800017F0B6FC894918A817F0F2FC18A8494672
:106F9000FAF774F918A817F0ABFC08A813F05AFF19
:106FA000B0EE480A2DB0BDEC028BBDE8F0830024A2
:106FB000502218A908A88DF83B4013F0A9FF00281B
:106FC00000F08480502300932A4618AB314608A86D
:106FD00014F00EF9002800F08F8018A81BF090FA2A
:106FE000014618A816F068FE6E4817F0F5FA7049C9
:106FF00004A817F0BDFC04A82146FAF73FF904A83D
:1070000017F076FC002F00F0AB802220FAF7A8FAE8
:1070100018A904A817F0ACFC214604A8FAF72EF929
:1070200004A817F065FC2220FAF79AFA614904A82F
:1070300017F09EFC002104A8FAF720F904A817F025
:1070400057FC07EE908A0020B8EEE70AFAF72CFA10
:10705000564904A817F08CFC002104A8FAF70EF991
:1070600004A817F045FC30461BF04AFA01463046AA
:1070700016F022FE4B4817F0AFFA28461BF040FAF4
:107080000146284616F018FE464817F0A5FA0521D5
:10709000474816F011FE002F6ED0222016F090FE09
:1070A00018A81BF02DFA014618A816F005FE22209C
:1070B00016F086FE01213F4816F0FEFD4146394894
:1070C00017F0DAFA374817F087FA35E009213A481D
:1070D0009FED338A16F0F0FD08A81BF011FA014667
:1070E00008A816F0E9FD0C21344816F0E5FD54E738
:1070F0000FA811F03DFCFCE61021314816F0DCFD34
:10710000284817F069FA04212E4816F0D5FD3046BC
:107110001BF0F6F90146304616F0CEFD03212A4851
:1071200016F0CAFD28461BF0EBF90146284616F07A
:10713000C3FD1C4817F050FA244A136804930499BD
:1071400013680393039B5B1A632BF9D918A81AF0F1
:1071500035F951EC100B19F009FE08EE100A1CE786
:1071600018A904A817F004FC04A83946FAF786F811
:1071700004A817F0BDFB59E718A81BF0C1F9014698
:1071800018A816F099FD95E7E416FF1F3007FF1FBA
:107190004407FF1FD018FF1FDC570200E85702000A
:1071A00000000000E407FF1FF8570200604E0200D5
:1071B000205802002858020004580200105802000B
:1071C000FC7002002C58020034580200841BFF1F80
:1071D00038B5854D8549864C284600234FF43C72CE
:1071E000FFF768FEBDEEC00A28460023C822814989
:1071F00084ED000AFFF75EFEBDEEC00A28460023BC
:107200004FF449727C4984ED010AFFF753FEBDEE4D
:10721000C00A284600234FF44A72784984ED0C0ACC
:10722000FFF748FEBDEEC00A284600233C22744901
:1072300084ED140AFFF73EFEBDEEC00A2846002387
:107240004FF458726F4984ED100AFFF733FEBDEE1C
:10725000C00A284600234FF457726B4984ED0D0A8B
:10726000FFF728FEBDEEC00A2846002340226749EA
:1072700084ED150AFFF71EFEBDEEC00A2846002366
:107280004FF45572624984ED110AFFF713FEBDEE0B
:10729000C00A284600234FF456725E4984ED0E0A58
:1072A000FFF708FEBDEEC00A2846002344225A49D3
:1072B00084ED160AFFF7FEFDBDEEC00A2846002346
:1072C0004FF44C72554984ED120AFFF7F3FDBDEE01
:1072D000C00A284600234FF44B72514984ED0F0A2F
:1072E000FFF7E8FDBDEEC00A284600231C224D49E9
:1072F00084ED170AFFF7DEFDBDEEC00A2846002325
:107300004FF4D872484984ED130AFFF7D3FDBDEE60
:10731000C00A284600234FF42E72444984ED050A22
:10732000FFF7C8FDBDEEC00A284601234FF4BA722C
:107330003F4984ED020AFFF7BDFDBDEEC00A2846B5
:10734000B8EEC00A00234FF4F8723A4984ED030AFC
:10735000FFF7B0FDBDEEC00A284601234FF41B72B3
:10736000354984ED040AFFF7A5FDBDEEC00A2846A5
:10737000B8EEC00A00234FF4DA72304984ED060AF1
:10738000FFF798FDBDEEC00A284601234FF41F7297
:107390002B4984ED0A0AFFF78DFDBDEEC00A284691
:1073A000B8EEC00A00234FF43D72264984ED080A66
:1073B000FFF780FDBDEEC00A284601234FF4967208
:1073C000214984ED070AFFF775FDBDEEC00A1F4B8A
:1073D000B8EEC00A2046196884ED0B0A6022BDE8A9
:1073E000384014F049B800BF405802003858020035
:1073F000F813FF1F44580200545802006858020056
:1074000078580200905802009C580200A4580200CC
:10741000B8580200C4580200CC580200E0580200DC
:10742000EC580200F45802000859020020590200EA
:107430002C590200445902005C59020074590200A0
:10744000885902009C590200B05902001407FF1F1E
:1074500038B54A4D4A494B4C284600234FF4EC724C
:10746000FFF728FDBDEEC00A284600234FF46172E5
:10747000454984ED0C0AFFF71DFDBDEEC00A284604
:1074800000234FF46B72414984ED010AFFF712FDAE
:10749000BDEEC00A2846002314223D4984ED090AA6
:1074A000FFF708FDBDEEC00A284600234FF45372D3
:1074B000384984ED050AFFF7FDFCBDEEC00A2846F9
:1074C00000234FF45472344984ED020AFFF7F2FCB2
:1074D000BDEEC00A284600233822304984ED0A0A4E
:1074E000FFF7E8FCBDEEC00A284600234FF4767291
:1074F0002B4984ED060AFFF7DDFCBDEEC00A2846E5
:1075000000234FF45172274984ED030AFFF7D2FCA0
:10751000BDEEC00A284600235422234984ED0B0AFD
:10752000FFF7C8FCBDEEC00A284600234FF4527294
:107530001E4984ED070AFFF7BDFCBDEEC00A2846D0
:1075400000234FF446721A4984ED040AFFF7B2FC97
:10755000BDEEC00A284600236C22164984ED000ABD
:10756000FFF7A8FC144BBDEEC00A2046196884ED55
:10757000080A3422BDE8384013F07EBFC459020027
:1075800038580200AC13FF1F54580200685802001C
:1075900078580200905802009C580200A45802003B
:1075A000B8580200C4580200CC580200E05802004B
:1075B000EC580200F45802005007FF1F38B54A4D3E
:1075C0004A494B4C284600234FF40E72FFF772FCD9
:1075D000BDEEC00A284600234FF45A72454984ED97
:1075E0000C0AFFF767FCBDEEC00A284600234FF4E3
:1075F0006472414984ED010AFFF75CFC0023BDEE93
:10760000C00A28461A463D4984ED090AFFF752FC94
:10761000BDEEC00A284600234FF46E72384984ED4F
:10762000050AFFF747FCBDEEC00A284600234FF4C9
:107630007372344984ED020AFFF73CFCBDEEC00AC8
:10764000284600231022304984ED0A0AFFF732FC55
:10765000BDEEC00A284600234FF478722B4984ED12
:10766000060AFFF727FCBDEEC00A284600234FF4A8
:107670007B72274984ED030AFFF71CFCBDEEC00AAC
:10768000284600230822234984ED0B0AFFF712FC49
:10769000BDEEC00A284600234FF47E721E4984EDD9
:1076A000070AFFF707FCBDEEC00A284600234FF487
:1076B0007F721A4984ED040AFFF7FCFBBDEEC00A95
:1076C000284600230C22164984ED000AFFF7F2FB3E
:1076D000144BBDEEC00A2046196884ED080A342216
:1076E000BDE8384013F0C8BEC8590200385802003F
:1076F0009818FF1F5458020068580200785802007A
:10770000905802009C580200A4580200B858020089
:10771000C4580200CC580200E0580200EC580200A5
:10772000F45802002C07FF1F38B5594D59495A4CDF
:10773000284600234FF41872FFF7BCFBBDEEC00AC9
:10774000284600234FF4D272544984ED000AFFF713
:10775000B1FBBDEEC00A284601234FF4197250490F
:1077600084ED0D0AFFF7A6FB284601234FF41D7296
:107770004C4984ED0F0AFFF79DFB284600234FF488
:107780005D72494984ED0E0AFFF794FBBDEEC00A15
:10779000284600234FF46772444984ED010AFFF73D
:1077A00089FBBDEEC00A284600234C22404984EDE7
:1077B000020AFFF77FFBBDEEC00A284600234FF404
:1077C0006F723C4984ED090AFFF774FBBDEEC00AF5
:1077D000284600234FF47472374984ED030AFFF7FB
:1077E00069FBBDEEC00A284600234822334984EDD8
:1077F000040AFFF75FFBBDEEC00A284600234FF4E2
:1078000079722F4984ED0A0AFFF754FBBDEEC00AD6
:10781000284600234FF47C722A4984ED050AFFF7BD
:1078200049FBBDEEC00A284600231822264984EDF4
:10783000060AFFF73FFBBDEEC00A284600234FF4BF
:107840006872224984ED0B0AFFF734FBBDEEC00AD3
:10785000284600234FF463721D4984ED070AFFF7A1
:1078600029FBBDEEC00A284600235022194984EDA9
:10787000080AFFF71FFB184BBDEEC00A2046196827
:1078800084ED0C0A4022BDE8384013F0F5BD00BF7E
:10789000D0590200385802006C13FF1FD85902005B
:1078A000E4590200445A0200545802006858020089
:1078B00078580200905802009C580200A458020018
:1078C000B8580200C4580200CC580200E058020028
:1078D000EC580200F45802000407FF1F38B5724D3F
:1078E0007249734C284600234FF4E872FFF7E2FA1E
:1078F000BDEEC00A284600234FF40D726D4984ED99
:10790000120AFFF7D7FABDEEC00A284600234FF44B
:107910000C72694984ED140AFFF7CCFABDEEC00A77
:10792000284600234FF46072644984ED130AFFF780
:10793000C1FABDEEC00A284600234FF46A726049BE
:1079400084ED000AFFF7B6FABDEEC00A2846002310
:1079500004225C4984ED080AFFF7ACFABDEEC00AC8
:10796000284600234FF47172574984ED040AFFF74B
:10797000A1FABDEEC00A284600234FF469725349AC
:1079800084ED010AFFF796FABDEEC00A28460023EF
:1079900058224F4984ED090AFFF78CFABDEEC00A60
:1079A000284600234FF470724A4984ED050AFFF718
:1079B00081FABDEEC00A284600234FF4757246498D
:1079C00084ED020AFFF776FABDEEC00A28460023CE
:1079D0006022424984ED0A0AFFF76CFABDEEC00A44
:1079E000284600234FF447723D4984ED060AFFF70D
:1079F00061FABDEEC00A284600234FF448723949A7
:107A000084ED030AFFF756FABDEEC00A28460023AC
:107A10003022354984ED0B0AFFF74CFABDEEC00A5F
:107A2000284600234FF40B72304984ED070AFFF714
:107A300041FABDEEC00A284601234FF49A722C4940
:107A400084ED0D0AFFF736FA28460123E82229497A
:107A500084ED100AFFF72EFA284600234FF43972FE
:107A6000254984ED100AFFF725FABDEEC00A284625
:107A700001234FF43A72214984ED0C0AFFF71AFAF8
:107A8000284601234FF4A2721D4984ED0F0AFFF727
:107A900011FA1C4B84ED0E0A204619685422BDE8E9
:107AA000384013F0E9BC00BFF0590200385802001A
:107AB0006414FF1FF4590200FC59020054580200DC
:107AC0006858020078580200905802009C58020042
:107AD000A4580200B8580200C4580200CC58020052
:107AE000E0580200EC580200F45802000C5A020060
:107AF0001C5A0200385A0200505A02005C5A020016
:107B0000745A02000007FF1F38B5864D8649874C1E
:107B100028460023A422FFF7CDF9BDEEC00A28466F
:107B20000023D022824984ED0E0AFFF7C3F9BDEE8F
:107B3000C00A28460023F0227E4984ED0C0AFFF794
:107B4000B9F9BDEEC00A284600234FF4E2727A4923
:107B500084ED0F0AFFF7AEF9BDEEC00A28460023F8
:107B60004FF42E72754984ED0D0AFFF7A3F9BDEEAF
:107B7000C00A2846B8EEC00A00234FF44F7270497D
:107B800084ED160AFFF796F9BDEEC00A28460023D9
:107B90004FF450726B4984ED000AFFF78BF9BDEE8C
:107BA000C00A284600236422674984ED040AFFF7CF
:107BB00081F9BDEEC00A284600234FF45C72634988
:107BC00084ED080AFFF776F9BDEEC00A28460023C7
:107BD0004FF46D725E4984ED010AFFF76BF9BDEE5B
:107BE000C00A2846002334225A4984ED050AFFF7CB
:107BF00061F9BDEEC00A284601234FF48A72564946
:107C000084ED090AFFF756F9BDEEC00A2846B8EE22
:107C1000C00A01234FF49272504984ED130AFFF712
:107C200049F9BDEEC00A2846B8EEC00A00234FF459
:107C30005B724B4984ED100AFFF73CF9BDEEC00AB8
:107C4000284600234FF45972464984ED020AFFF793
:107C500031F9BDEEC00A284600232C22424984EDAA
:107C6000060AFFF727F9BDEEC00A284601234FF4A4
:107C70008E723E4984ED0A0AFFF71CF9BDEEC00A78
:107C80002846B8EEC00A0123E022394984ED140ADF
:107C9000FFF710F9BDEEC00A2846B8EEC00A00236F
:107CA0004FF44E72334984ED110AFFF703F9BDEE2C
:107CB000C00A284600234FF44D722F4984ED030A71
:107CC000FFF7F8F8BDEEC00A2846002320222B4912
:107CD00084ED070AFFF7EEF8BDEEC00A284601233F
:107CE0004FF40272264984ED0B0AFFF7E3F8BDEE6C
:107CF000C00A2846B8EEC00A01234FF40472214995
:107D000084ED150AFFF7D6F8BDEEC00A1E4BB8EE9B
:107D1000C00A2046196884ED120A5C22BDE838408A
:107D200013F0AABB8C5A020038580200D012FF1F71
:107D3000905A0200FC590200985A0200A05A020010
:107D40005458020068580200785802009058020007
:107D50009C580200A4580200B45A0200C85A0200FB
:107D6000B8580200C4580200CC580200DC5A020085
:107D7000F05A0200E0580200EC580200F4580200E9
:107D8000045B0200185B0200FC06FF1F2DE9F047B0
:107D9000794C7A497A4DDFF844A2DFF84482794F72
:107DA000794EDFF84092204600234FF4B872FFF777
:107DB00081F8BDEEC00A204600234FF46272734979
:107DC00085ED000AFFF776F8BDEEC00A20460023D5
:107DD0004FF46C726E4985ED010AFFF76BF8BDEE4A
:107DE000C00A2046002368226A4985ED030AFFF78E
:107DF00061F8BDEEC00A204651460023C02285ED41
:107E0000020AFFF757F8BDEEC00A204600234FF4E0
:107E10000F72614988ED000AFFF74CF8BDEEC00A09
:107E2000204601234FF4B0725C4988ED010AFFF748
:107E300041F8BDEEC00A514620460023A02288ED3D
:107E4000020AFFF737F8BDEEC00A204600234FF4C0
:107E50003172534987ED000AFFF72CF8BDEEC00AD6
:107E6000204601234FF4B4724E4987ED010AFFF713
:107E700021F8BDEEC00A2046002398224A4987ED2A
:107E8000020AFFF717F8BDEEC00A204600234FF4A0
:107E90001472464986ED000AFFF70CF8BDEEC00AE1
:107EA000204601234FF41172414986ED010AFFF784
:107EB00001F8BDEEC00A204600234FF4D6723D49BA
:107EC00086ED020AFEF7F6FFBDEEC00A204600234B
:107ED0004FF41372384989ED000AFEF7EBFFBDEE4F
:107EE000C00A204601234FF42872344989ED010A63
:107EF000FEF7E0FFBDEEC00A204600234FF4DC721F
:107F00002F4989ED020AFEF7D5FFDFF8DC902D49F5
:107F1000BDEEC00A204600234FF4067289ED000A28
:107F2000FEF7C8FFBDEEC00A204601234FF42A72B7
:107F3000254989ED010AFEF7BDFF244BBDEEC00ABD
:107F40002846196889ED020A102213F095FA204B91
:107F500040461968182213F08FFA1E4B38461968EC
:107F6000182213F089FA1C4B304619681822BDE814
:107F7000F04713F081BA00BF345B02002C5B0200B3
:107F80006C15FF1F3816FF1F5016FF1F54580200B4
:107F90006858020078580200505B0200605B0200E3
:107FA000685B0200785B0200805B0200985B020065
:107FB000A85B0200B05B0200C85B0200D85B020055
:107FC000E05B0200F85B0200085C02005807FF1F3C
:107FD0001807FF1F1C07FF1F3407FF1F385B020035
:107FE000B814FF1F6816FF1F8016FF1F38B5B42294
:107FF000002397499748984C974DFEF75BFF002365
:10800000D42296499348FEF755FFBDEEC00A0023DF
:10801000F42293498F4884ED000AFEF74BFFBDEE32
:10802000C00A01234FF486728E498A4884ED010A02
:10803000FEF740FF0023F8228B49864884ED020AB0
:10804000FEF738FFF7EE007AB4EEE70AF1EE10FA29
:10805000ACBF0123002384F87430D8220123834964
:108060007C48FEF727FFBCEEC00A0123DC228049D2
:10807000784884ED210AFEF71DFFBCEEC00A0023FC
:108080004FF4EA727B49734884ED220AFEF712FF2F
:10809000BDEEC00A00234FF4E67277496D4884EDC7
:1080A000040AFEF707FFBDEEC00A01234FF4007279
:1080B0007249684884ED030AFEF7FCFE0023FC22A7
:1080C0006F49644884ED050AFEF7F4FEF7EE007A86
:1080D000B4EEE70AF1EE10FAACBF0123002385F8F5
:1080E00075304FF4F272002366495A485A4DFEF734
:1080F000E1FEBDEEC00A00234FF4F072624955481C
:1081000084ED090AFEF7D6FEBDEEC00A01234FF446
:10811000F4725E494F4884ED080AFEF7CBFE002357
:108120004FF480725A494B4884ED0A0AFEF7C2FEAA
:10813000F7EE007AB4EEE70AF1EE10FAACBF0123D5
:10814000002385F87630CC22002352494148424D25
:10815000FEF7B0FEBDEEC00A0023C4224E493D48E2
:1081600084ED260AFEF7A6FEBDEEC00A0123D82242
:108170004A49384884ED250AFEF79CFE00234FF457
:1081800065724749334884ED270AFEF793FEF7EE00
:10819000007AB4EEE70AF1EE10FAACBF0123002337
:1081A00085F8A0304FF4087200233E4929482A4D33
:1081B000FEF780FEBDEEC00A00234FF407723A4975
:1081C000244884ED0F0AFEF775FEBDEEC00A0123B8
:1081D0004FF4097235491F4884ED0E0AFEF76AFE16
:1081E00000234FF4827232491A4884ED100AFEF7D8
:1081F00061FEF7EE007AB4EEE70AF1EE10FAACBFDA
:108200000123002385F877304FF4CC7201232949EC
:108210001048FEF74FFE0023942227490D4884EDB5
:10822000110AFEF747FEBCEEC00A01234FF42C7280
:108230002249084884ED0D0AFEF73CFE204B84EDF0
:10824000120A19680448A422BDE8384013F014B992
:10825000105C02001C5C0200DC17FF1F245C0200A3
:10826000385C02004C5C0200605C0200745C02003E
:10827000885C0200A45C0200B45C0200C45C0200E2
:10828000D85C0200E45C0200F45C0200045D0200C1
:10829000185D0200245D0200385D0200485D0200A6
:1082A0005C5D02006C5D02007C5D02008C5D020082
:1082B000985D0200A45D0200B85D0200C85D020086
:1082C000E413FF1F38B53A4D3A493B4C284600238A
:1082D0004FF4EE72FEF7EEFDBDEEC00A2846002315
:1082E0004FF4C472354984ED130AFEF7E3FDBDEE89
:1082F000C00A28460023B022314984ED140AFEF753
:10830000D9FDBDEEC00A284600234FF4D4722D4992
:1083100084ED200AFEF7CEFDBDEEC00A28460023FC
:108320004FF43072284984ED060AFEF7C3FDBDEE16
:10833000C00A284600238C22244984ED070AFEF750
:10834000B9FDBDEEC00A284600234FF4157220493E
:1083500084ED1E0AFEF7AEFDBDEEC00A28460023DE
:108360004FF410721B4984ED0B0AFEF7A3FDBDEE1E
:10837000C00A28460023B022174984ED0C0AFEF7F4
:1083800099FDBDEEC00A28460023B822134984EDAA
:108390001F0AFEF78FFD124BBDEEC00A204619687A
:1083A00084ED1F0AA422BDE8384013F065B800BF71
:1083B000D85D0200D05D0200DC17FF1FE05D020007
:1083C000E85D0200F05D0200F85D0200005E020060
:1083D000085E0200105E0200185E0200205E0200CD
:1083E000E413FF1F38B5314D3149324C2846002384
:1083F0004FF43E72FEF75EFDBDEEC00A2846002334
:108400004FF43F722C4984ED150AFEF753FDBDEE83
:10841000C00A284600234FF44072284984ED160A0A
:10842000FEF748FDBDEEC00A284600234FF4417216
:10843000234984ED170AFEF73DFDBDEEC00A28462C
:1084400000234FF444721F4984ED180AFEF732FDF1
:10845000BDEEC00A284600234FF445721A4984ED48
:10846000190AFEF727FDBDEEC00A284600234FF487
:108470004272164984ED1A0AFEF71CFDBDEEC00AD1
:10848000284600234FF44372114984ED1B0AFEF77E
:1084900011FD104BBDEEC00A2046196884ED1C0A80
:1084A000A422BDE8384012F0E7BF00BF2C5E0200F6
:1084B00054580200DC17FF1F68580200345E0200A7
:1084C000445E0200545E0200645E0200745E0200BC
:1084D000845E0200E413FF1F70B5574D5749584C96
:1084E000584E284600234FF4E472FEF7E3FCBDEE3D
:1084F000C00A284600234FF47272534984ED000AE3
:10850000FEF7D8FCBDEEC00A284600234FF4777270
:108510004E4984ED010AFEF7CDFCBDEEC00A2846A7
:10852000002328224A4984ED020AFEF7C3FCBDEE6F
:10853000C00A28460123A822464984ED030AFEF713
:10854000B9FC284601234FF4C672434984ED0A0A58
:10855000FEF7B0FC284600234FF47A723F4984EDC1
:108560000D0AFEF7A7FCBDEEC00A284600234FF413
:108570007D723B4984ED040AFEF79CFCBDEEC00A07
:10858000284600232422374984ED050AFEF792FC91
:10859000BDEEC00A284601234FF4AA72324984ED89
:1085A000060AFEF787FC284601234FF49E722F49E6
:1085B00084ED0B0AFEF77EFC284600234FF45E7222
:1085C0002B4984ED0E0AFEF775FCBDEEC00A284665
:1085D00000234FF45F72274984ED070AFEF76AFC17
:1085E000BDEEC00A284600235C22234984ED080A18
:1085F000FEF760FCBDEEC00A284601234FF4A672C8
:108600001E4984ED090AFEF755FC2046316884EDC9
:108610000C0A402212F030FF28464FF4FA72184933
:108620000123FEF747FC316884ED0F0A2046402203
:10863000BDE8704012F020BF945E0200385802007E
:108640009815FF1F3807FF1F905802009C58020022
:10865000A4580200985E0200A45E0200B85802000E
:10866000C4580200CC580200B05E0200BC5E02009A
:10867000E0580200EC580200F4580200C85E020004
:10868000D45E0200804B814A1B68116810B5012B33
:1086900008BF7F4B9AB008BF19680AA800230122BF
:1086A00012F0BAFB11A810F071F9002840F0E88030
:1086B00002A89DF8423077490AAA10F01BFA049AE2
:1086C0009DF814309DF80C1013928DF850308DF8F1
:1086D000481005AA0DF151030DF15E0012F8011FBB
:1086E00003F8011B8342F9D1099B189302A810F0EB
:1086F0001FF911A810F04AF90446002850D10123AF
:10870000182165488DF8433015F0D6FA634815F006
:1087100063FF634902A816F02BF9214602A8F8F777
:10872000ADFD02A816F0E4F85E4902A816F020F9A3
:10873000214602A8F8F7A2FD02A816F0D9F85A4976
:1087400002A816F015F9214602A8F8F797FD02A82D
:1087500016F0CEF8534902A816F00AF9214602A8ED
:10876000F8F78CFD02A816F0C3F8504902A816F0DD
:10877000FFF8214602A8F8F781FD02A816F0B8F824
:10878000484902A816F0F4F8214602A8F8F776FD49
:1087900002A816F0ADF80AA812F05CFB1AB010BDE2
:1087A0000023142142488DF8433015F085FA3B48E8
:1087B00015F012FF11A810F0E9F800285CD1FFF7BE
:1087C00015FCFFF70FFEFFF77DFDFEF7F7FEFEF746
:1087D0003FFEFFF7DBFAFFF77FFEFEF7A5FFFFF78F
:1087E0007DF8FEF7F5FCFFF78FF92D4902A816F08A
:1087F000BFF8002102A8F8F741FD02A816F078F8AA
:10880000284902A816F0B4F8002102A8F8F736FDAE
:1088100002A816F06DF8274A1368019301991368AE
:108820000093009B5B1A0E2BF9D91F4902A816F082
:108830009FF8002102A8F8F721FD02A816F058F8C9
:10884000184902A816F094F8002102A8F8F716FDBE
:1088500002A816F04DF8184902A816F089F8002170
:1088600002A8F8F70BFD02A816F042F80D4902A87D
:1088700016F07EF8002188E711A810F079F89EE73D
:1088800011A810F075F813E7E416FF1F3007FF1F5B
:108890004407FF1FD018FF1FF85E0200E407FF1F08
:1088A000145F0200604E0200806A0200F857020066
:1088B000E05E0200841BFF1F245F020090F89030EE
:1088C00010B504461BB906E0012012F041FFA36871
:1088D000002BF9D110BDF7F757FEF8E78368E3B135
:1088E000816D826F4B68D21A30B482EAE273D0F89D
:1088F000AC40A3EBE273A34210DBD0F8B02093426C
:1089000014DA1A190025C2672346C0F8B05030BCEB
:108910004A68086800FB0323CB60704700225C00B4
:10892000C0F8B020C0F8AC20C467F0E7C26FD31A1B
:10893000EDE700BF10B50446FFF7D0FFA3682BB1E9
:10894000012012F005FFA368002BF9D110BD00BF74
:1089500007EE901AF8EE676A07EE902A9FED1C7AF0
:10896000DFED1C5A9FED1C6A4167F8EE677A66EEF0
:10897000876A67EE877A66EEA56A27EEA57AF6EE35
:10898000007AF0EE675AE6EE865AF0B4E7EE067A21
:108990000346124F5861FDEEE56AFDEEE77A104E90
:1089A0000267802500220124076046600574C466C2
:1089B000C0ED066AC0ED077A8260C26080F82820A8
:1089C000C265026680F864208266F0BC704700BF12
:1089D000BD378635C0E1644C0000003DCC4A020042
:1089E000C04A020038B590F86430114A026004466B
:1089F00000F10C0553B1284615F05CFD0023206AF8
:108A0000A36012F0CFF9606A12F0CCF9094B6360F1
:108A1000284615F04FFD0023A360206A12F0C2F92A
:108A2000606A12F0BFF9284615F044FD204638BDB3
:108A3000CC4A0200C04A020010B5034B0360044652
:108A4000FFF7D0FF204610BD044B020010B5054BC8
:108A500003600446FFF7C6FF2046B82115F07EFDEF
:108A6000204610BD044B020010B5034B03600446C2
:108A7000FFF7B8FF204610BDE84A020010B5054BCD
:108A800003600446FFF7AEFF2046942115F066FD13
:108A9000204610BDE84A020010B50446FFF7A2FFC9
:108AA0002046782115F05AFD204610BD884231D06D
:108AB0002DE9F04700F10408414516468A468146F3
:108AC00017D0D9F80010D8F80000B04798B9D8F8F6
:108AD0000050444601E0236863602746284654F866
:108AE000041DB0470028F6D13D6008F10408C245D6
:108AF000E7D1BDE8F087C9EB08029308D8F8004039
:108B000005D0C2F104004044494618F0BFFFC9F83F
:108B10000040EAE7704700BF2DE9F8430B1A432BEA
:108B20001CDD00F14008894641461746FFF7BEFFAD
:108B3000C14515D0D8F80050444601E02368636071
:108B40002646284654F8041DB8470028F6D108F1F7
:108B50000408C1453560EDD1BDE8F883FFF7A6FFF5
:108B6000BDE8F8832DE9F04F561E06EBD67683B0AC
:108B70007610B14201928846054699460C9F5CDA10
:108B80008A4600E0DA460AF101034FEA430B0BF193
:108B90008041013955F8330055F8211005EBC30425
:108BA000B84718B10BF1FF3B05EB8B04236845F880
:108BB0002A30B345E6DB019BDA0707D4019BA3F11A
:108BC000020A0AEBDA7ABBEB6A0F06D0C34514DC63
:108BD000C4F8009003B0BDE8F08F0BF1010B4FEA31
:108BE0004B0B0BF18043013B0BF1FF3B55F823305E
:108BF0002360C34505EB8B04EADD0BF1FF3606EB82
:108C0000D6767610494655F82600B847731E03EB12
:108C1000D37305EB86045B1030B905EB8B04C4F805
:108C2000009003B0BDE8F08F55F8262045F82B20C2
:108C3000B045CDDAB3461E46E4E7019BDB0700EB07
:108C40008104C5D48B46B9E72DE9F04F0C1A432CAB
:108C500085B040F389800546894692461E46002A23
:108C600061D0031D0393E410686855F82410B047E1
:108C70000AF1FF3A59F8041C002834D055F82400B2
:108C8000B047002837D02B6855F824202A6045F8D3
:108C9000243068682968039FCB46B846B04780B93E
:108CA000ABF1040421682868A346043CB0470028BF
:108CB000F8D15F4509D23A68DBF800103960CBF88B
:108CC000002057F8040F2968E7E749463346524623
:108CD00038467C1BFFF7B8FF432C45DDBAF1000F87
:108CE00022D0B946BFE76868B04798B195E803005D
:108CF00029606860CFE759F8041C6868B04700280D
:108D0000F4D02B6859F8042C2A6049F8043C6868B0
:108D10002968C0E759F8041C55F82400B0472B68AF
:108D20000028B1D0EEE78846A410A71E7F1005EBFF
:108D3000870900E0013F59F8043900962246394678
:108D40002846FFF70FFF002FF4D158F8043D2A689A
:108D50000096C5EB0804C8F800200021A2102846A0
:108D6000FFF700FF072CF0DC05B0BDE8F08F00BF77
:108D7000836833B1614B1B6813B10121022018478E
:108D800070472DE9F04700F12C064FEA810906EB08
:108D90000905AE422DED028B10EE107A884604468E
:108DA00010D04FEAA902B2FA82F2C2F11F025200B9
:108DB00029463046524BFFF747FF514A2946304675
:108DC000FFF7AAFEE16AA1658A69002A00F08E8099
:108DD00082EAE273A3EBE273B8F1010F4FF00002F5
:108DE0000B618A6012DD09F1280EA644304650F866
:108DF000042F936983EAE37CACEBE37CC2F810C0F8
:108E00000B697045C3EB4C035361F0D1AE4271D096
:108E10004A6A04F1300306E01968496A8A4203F19C
:108E2000040328BF0A469D42F6D108EE102A00230B
:108E3000251D84F8903084F82830284611F09EFFD4
:108E40002062284611F09AFF606211F06BFF04F176
:108E50000800616911F01CFFA36DD4ED1C6A93ED4D
:108E6000067A9FED286A5B68F8EE487AF8EE666A43
:108E7000B8EEC77A67EEA67A84ED207A87EE867A16
:108E80000022E26784ED217A72B6D4F88430C4F807
:108E9000883062B672B694ED200AD4ED1F7A07EEE0
:108EA000107A27EE000AB4EEE70AD4ED227A84EDB8
:108EB0001E0AF1EE10FAD8BFF1EE677AC4ED237AFC
:108EC00062B6114A236AE06900211160DB00516833
:108ED00003F1804303F5603301440D2019611060F4
:108EE000DA68502122F08002DA60D960BDEC028B92
:108EF000BDE8F087E36A93ED098A98E74C1BFF1FF2
:108F00007D04000000247449008003402DE9F04FE7
:108F10002DED028BD3B041F28832052106462DA8F3
:108F2000FFF716FD9E489F4B2D93002303609E4D37
:108F30009E489F4F03602A6B9E48D7F81C908DF87F
:108F4000443101210360D7F818A04891032A00F2A8
:108F50006283DFE802F0CCB39A02D5ED057A9FED8B
:108F6000968A6B68D5F824800193F8EEE77A07EECD
:108F7000106A67EE887AB8EEC78A022227EE888ADE
:108F800003210DF1740B584611F08CFD8B4C00221F
:108F90001E9222680692069823680593059B874ACD
:108FA0001B1A042BF8D901990092584611F0BCFD08
:108FB000414611F0ADFD824911F0DAFD0121286B27
:108FC000F7F76CFD479952AB01F10B0E03EB8100F3
:108FD00003EB8E0E002340F868BCB7EE000A4EF893
:108FE000903C01212DA84793FFF7C2FE009A136819
:108FF0000493049A23680393039B9B1A042BF9D9C7
:1090000000238DF8443172B6DDED4D7A9DED4C7A3A
:1090100068EE277AB4EEE77ACDED4B7ADDED4F7A44
:10902000F1EE10FA58BFF1EE677ACDED507A62B6E4
:10903000DFF89481DFF894B1DFED5F8A2F9B002B7E
:1090400000F0E580F8F736FE002840F39080D8F86D
:109050000000F8F71FFEC0B253288BF8000000F0A4
:10906000D581662840F08380D8F80000F7F700FE2D
:1090700051EC100B17F032FE2B6B032B59D8DFE8A5
:1090800013F0B902AB029D024B00D5ED087A9FEDBB
:109090004A8A2B690193F8EEE77A07EE106A67EEC9
:1090A000887AB8EEC78AD7F85090D7F84CA0D5F890
:1090B0000080172227EE888A102162E7D5ED077A13
:1090C0009FED3D8AEB680193F8EEE77A07EE106AB0
:1090D00067EE887AB8EEC78AD7F83090D7F82CA018
:1090E000D5F82C80142227EE888A152149E7D5ED82
:1090F000067A9FED318AAB680193F8EEE77A07EEC6
:10910000106A67EE887AB8EEC78AD5F828800522FB
:1091100027EE888A062134E707EE900AB8EEE78A40
:1091200007EE906A28EE288AF8EEE77A686128EE62
:10913000278A244B1C481968342212F09DF9002319
:109140008DF8443172B6DDED4D7A9DED4C7A68EEC6
:10915000277AF4EEC77ACDED4B7ADDED4F7AF1EE5A
:1091600010FAD8BFF1EE677ACDED507A62B65FFAA9
:1091700089F012F0D9FA08B9012E2BD05FFA8AF0E3
:1091800012F0D2FA08B9731C24D023680C930C9AFD
:1091900023680B930B9B9B1A092BF9D94EE700BF51
:1091A000B812FF1FE84A0200AC13FF1F4017FF1F51
:1091B000DC17FF1F7412FF1F0AD7233C841BFF1FFD
:1091C000C09EF87F5007FF1F1007FF1FE816FF1F04
:1091D000000000008DF8440172B65FED036ADDED1A
:1091E0004D7A9DED4C7A67EEA67AF4EEC77AF1EEF1
:1091F00010FACDED4B7A00F30B82DDED4F7AF1EEF4
:10920000677ACDED507A62B62DA8FFF757FB286B31
:10921000032800F02F811E9B704A714F136007EEE8
:10922000903A4FF00009B8EEE70AC7F80090F7F758
:1092300043FD19AEDFF8CC816A4988ED000A30465B
:1092400015F096FB49463046F8F718F8304615F009
:109250004FFB2220F8F784F998ED000A4846F8F70A
:1092600023F92220F8F77CF9FF20F8F779F9FF209D
:10927000F8F776F9FF20F8F773F92368189318992F
:1092800023681793179B584A5B1A042BF8D9554942
:109290000092304615F06CFB00213046F7F7EEFFE8
:1092A000304615F025FB2220F8F75AF998ED000A10
:1092B0000020F8F7F9F82220F8F752F9FF20F8F724
:1092C0004FF9FF20F8F74CF9FF20F8F749F9009A19
:1092D00013681693169923681593159B424A5B1AD7
:1092E000042BF8D941490092304615F041FB00218A
:1092F0003046F7F7C3FF304615F0FAFA2220F8F7A8
:109300002FF997ED000A0020B8EEC00AF8F7CCF864
:109310002220F8F725F9FF20F8F722F9FF20F8F7C7
:109320001FF9FF20F8F71CF9009A13681493149A98
:1093300023681393139B9B1A042BF9D9286B0021E4
:10934000F7F7ACFB2A49304615F012FB00213046F6
:10935000F7F794FF304615F0CBFA2649304615F062
:1093600007FB00213046F7F789FF304615F0C0FAB9
:109370002149304615F0FCFA00213046F7F77EFF10
:10938000304615F0B5FA1B49304615F0F1FA0021C8
:109390003046F7F773FF304615F0AAFA1749304602
:1093A00015F0E6FA00213046F7F768FF304615F071
:1093B0009FFA1049304615F0DBFA00213046F7F7E6
:1093C0005DFF304615F094FA0D4B2D932DA8FFF755
:1093D00009FB53B0BDEC028BBDE8F08F7412FF1F88
:1093E0006815FF1F405F0200841BFF1F305F0200F3
:1093F000505F0200604E0200685F0200845F02005E
:10940000E84A02009015FF1F0000000000238DF8BD
:10941000443172B65FED046ADDED4D7A9DED4C7A14
:1094200067EEA67AF4EEC77ACDED4B7ADDED4F7A92
:10943000F1EE10FAD8BFF1EE677ACDED507A62B650
:1094400023680A930A9A23680993099B764E9B1A0C
:10945000042BF8D92DA8FFF731FA33680893089A3E
:1094600023680793079B9B1A632BF9D9286B032862
:109470007FF4D1AE79683B681E9A97ED027ADFEDF2
:109480006B6A6B486B4F026003FB01F307EE903A87
:1094900006EE102AF8EE677AB8EEC66A67EE877AAB
:1094A000654B66491A6086EE277A654B19AE4FF018
:1094B00000083046C3F8008067EE267AC7ED007AD0
:1094C00015F056FA41463046F7F7D8FE304615F00B
:1094D0000FFA2220F8F744F897ED000A4046F7F714
:1094E000E3FF2220F8F73CF8FF20F8F739F8FF20D7
:1094F000F8F736F8FF20F8F733F82368129312993B
:1095000023681193119B484A5B1A042BF8D94B49E5
:109510000092304615F02CFA00213046F7F7AEFEE7
:10952000304615F0E5F92220F8F71AF897ED000A11
:109530000020F7F7B9FF2220F8F712F8FF20F8F71C
:109540000FF8FF20F8F70CF8FF20F8F709F8009A59
:1095500013681093109A23680F930F9B324F9B1A36
:10956000042BF8D93749304615F002FA002130466D
:10957000F7F784FE304615F0BBF92220F7F7F0FF2D
:109580002F4B93ED000A0020B8EEC00AF7F78CFFCE
:109590002220F7F7E5FFFF20F7F7E2FFFF20F7F7BC
:1095A000DFFFFF20F7F7DCFF3B680E930E9A23687E
:1095B0000D930D9B9B1A042BF9D9BFE607EE900A79
:1095C000B8EEE78A07EE906A28EE288AF8EEE77A86
:1095D000286228EE278AACE507EE900AB8EEE78A03
:1095E00007EE906A28EE288AF8EEE77AE86128EE1E
:1095F000278A9EE507EE900AB8EEE78A07EE906AA2
:1096000028EE288AF8EEE77AA86128EE278A90E506
:10961000DDED4F7AF5E54FF000089FED0B8ACDF8B0
:10962000048005220621ACE4841BFF1F0000B44324
:109630004017FF1F3016FF1F6815FF1F305F020025
:109640007412FF1F405F0200000000002DE9F04F80
:109650002DED048BADF54B7D1446804641F28832EA
:109660008A4680A80521FFF773F94FF00009634B84
:10967000634E8093012541F288320521A5A89B9570
:109680008DF89092FFF764F902225C4BC09503219C
:1096900040A8A5938DF8249311F004FAB3695948B2
:1096A00001931021D6F81CB0574F14F005FB21464A
:1096B000564814F0E1FF554814F08EFF032C4FF08C
:1096C00005024FF0060150A8BABF4D4601244C4692
:1096D00011F0E8F91422152160A811F0E3F970A83F
:1096E0001722102111F0DEF93B6B012B00F0BE8731
:1096F000022B00F08F87002B00F00C85CDF800B016
:10970000DFED438ADFF82CB1D7F824900023419392
:10971000DBF800300C937B6903930C9A7B6802930F
:10972000DBF800300B930B9B9B1A042BF8D9029BA0
:1097300040A80AFB03F111F0F7F9494611F0E8F9E6
:10974000344911F015FA0821334814F0B5FA0A210A
:10975000324814F0B1FA02992C4814F08DFF2B48CE
:1097600014F03AFF08212C4814F0A6FA07212C48DF
:1097700014F0A2FA4946254814F07EFF234814F05D
:109780002BFF0821244814F097FA1121254814F0E2
:1097900093FA20491D4814F06FFF1C4814F01CFF79
:1097A000E4B1D7F83090B9F1010F01F04480B9F17C
:1097B000020F00F0FC87B9F1000F00F09D87052132
:1097C000194814F079FA0421184814F075FA0121A7
:1097D0000E4814F051FF0D4814F0FEFE002D40F02D
:1097E0007C869FED0B8ADFF85090DFF850A09FED4C
:1097F000109A2CBB002D00F05F8521E0E84A0200A2
:10980000DC17FF1F985F02009818FF1FE407FF1F77
:1098100000000000C09EF87FAC5F0200B85F02004D
:1098200004520200C45F0200D85F0200E05F020041
:109830000AD7233C841BFF1F1007FF1FE816FF1FDA
:10984000DBF8002018921899DBF800301793179B6B
:109850005B1A042BF8D9F8F72DFA0028C0F289809A
:10986000D9F80000F8F716FAC0B2A0F153028AF84E
:109870000000722A7DD8DFE812F0C1037C007C0072
:109880007C007C007C007C00000473037C007C0076
:109890007C007C007C007C007C0026037C007C003B
:1098A0007C007C007C007C007C00DC0278027C0078
:1098B000490203027C007C007C007C007C007C0070
:1098C0007C007C007C007C007C007C007C007C00B8
:1098D0007C007C007C007C007C007C007C007C00A8
:1098E0007C007C007C007C007C007C007C007C0098
:1098F0007C007C007C007C007C007C007C007C0088
:109900007C007C007C007C007C007C007C007C0077
:109910007C007C007C007C007C007C007C00AD0135
:1099200061017C007C007C007C00FA0095007C00DA
:109930007C007C007C007C007C007C007C007C0047
:109940007C007C007C007C007C007C007C007C0037
:109950007C007C007C007C007C007C007C00730030
:10996000F8F7BCF9C24A38631168C248342211F0D2
:1099700083FD002C00F0BD819DF8000011F0D4FEA5
:1099800018B9B8F1010F00F0F1830124DBF80020D1
:1099900034923499DBF800303393339B5B1A042BF9
:1099A000F8D926E7A79A002AE3D1D7ED087A3969D2
:1099B000039270A8F8EEE78A11F0B6F8AE4911F0FC
:1099C000D7F801210220F7F769F8BF99039ABF92EF
:1099D000CAAB03EB8100044670AB40F8683CB7EEBD
:1099E000000A44F8642C0121A5A8FFF7C1F9039AE5
:1099F0008DF8242368EE898A72B6DDEDC57A9DED77
:109A0000C47A67EE887AF4EEC77ACDEDC37ADDEDDD
:109A1000C77AF1EE10FAD8BFF1EE677ACDEDC87AC9
:109A200062B6DBF800202E922E99DBF800302D93E1
:109A30002D9B5B1A042BF8D900228DF8242372B6D3
:109A4000DDEDC57A9DEDC47A68EEA77AF4EEC77AAB
:109A5000CDEDC37ADDEDC77AF1EE10FAD8BFF1EEA5
:109A6000677ACDEDC87A62B64FF0010884E7A79A0D
:109A7000002A7FF47EAF3969D7ED087A0392494214
:109A800070A8F8EEE78A11F04FF87C4911F070F8F1
:109A900001210220F7F702F8BF99039ABF92CAABDF
:109AA00003EB8100044670AB40F8683CB7EE000A57
:109AB00044F8642C0121A5A8FFF75AF9039A8DF800
:109AC000242368EE898A72B6DDEDC57A9DEDC47AED
:109AD00067EE887AF4EEC77ACDEDC37ADDEDC77A0A
:109AE000F1EE10FAD8BFF1EE677ACDEDC87A62B622
:109AF000DBF800202C922C99DBF800302B932B9B69
:109B00005B1A042BF8D900228DF8242372B6DDED00
:109B1000C57A9DEDC47A68EEA77AF4EEC77ACDEDEA
:109B2000C37ADDEDC77AF1EE10FAD8BFF1EE677AAD
:109B3000CDEDC87A62B64FF0FF381DE7A79A002A2C
:109B40007FF417AFD7ED077AF968039260A8F8EEB3
:109B5000E78A10F0E9FF484911F00AF801210846A8
:109B6000F6F79CFFBF99039ABF92CAAB03EB810043
:109B7000044660AB40F8683CB7EE000A44F8642C39
:109B80000121A5A8FFF7F4F8039A8DF8242368EEC5
:109B9000898A72B6DDEDC57A9DEDC47A67EE887A62
:109BA000F4EEC77ACDEDC37ADDEDC77AF1EE10FAA7
:109BB000D8BFF1EE677ACDEDC87A62B6DBF8002047
:109BC0002A922A99DBF800302993299B5B1A042BEF
:109BD000F8D931E7A79A002A7FF4CBAEF968D7ED20
:109BE000077A0392494260A8F8EEE78A10F09CFFDA
:109BF000224910F0BDFF01210846F6F74FFFBF993B
:109C0000039ABF92CAAB03EB8100044660AB40F8F5
:109C1000683CB7EE000A44F8642C0121A5A8FFF7C0
:109C2000A7F8039A8DF8242368EE898A72B6DDEDD1
:109C3000C57A9DEDC47A67EE887AF4EEC77ACDEDE9
:109C4000C37ADDEDC77AF1EE10FAD8BFF1EE677A8C
:109C5000CDEDC87A62B6DBF8002028922899DBF8AF
:109C600000302793279B5B1A042BF8D94BE700BFE2
:109C70002C07FF1F9818FF1FC09EF87F40610780C8
:109C8000D9F80000F6F7F4FF51EC100B17F026F8A6
:109C90003A6BB049012A00F02685022A00F01A85A5
:109CA00032B907EE900AF8EEE78A886168EE898A91
:109CB000A94AA8481168342211F0DEFB00228DF871
:109CC000242372B6DDEDC57A9DEDC47A68EEA77ADD
:109CD000F4EEC77ACDEDC37ADDEDC77AF1EE10FA76
:109CE000D8BFF1EE677ACDEDC87A62B6002C7FF46A
:109CF00043AE9DF8040011F017FD002840F02781C5
:109D0000B8F1FF3F00F07E8204463FE6D9F800003C
:109D1000F6F7AEFF51EC100B16F0E0FF8E4A09EE9D
:109D2000900A11688B48C7ED059A342211F0A4FB04
:109D300000228DF8902272B6B8EEE97ADDEDA07AB5
:109D4000DDED9F6A27EE097A67EE277AF4EEE67A70
:109D5000CDED9E7ADDEDA27AF1EE10FAD8BFF1EEEC
:109D6000677ACDEDA37A62B603E6829A002A7FF481
:109D700000AED7ED057A029B0392F8EEE77A5942DE
:109D800040A867EE899A10F0CFFE744910F0F0FEFB
:109D900001210320F6F782FE9A99039A9A9280ABEA
:109DA00003EB8100054640ABC362B7EE000A2A63AD
:109DB000012180A8FEF7DCFF039A8DF8902272B68D
:109DC000DDEDA07A9DED9F7A67EE887AF4EEC77A92
:109DD000CDED9E7ADDEDA27AF1EE10FAD8BFF1EE6C
:109DE000677ACDEDA37A62B6DBF800202692269939
:109DF000DBF800302593259B5B1A042BF8D9002251
:109E00008DF8902272B6DDEDA07A9DED9F7A69EE15
:109E1000A77AF4EEC77ACDED9E7ADDEDA27AF1EE67
:109E200010FAD8BFF1EE677ACDEDA37A62B60125BC
:109E30009FE5829A002A7FF49CADD7ED057A0299BE
:109E40000392F8EEE77A40A867EE899A10F06CFE6C
:109E5000424910F08DFE01210320F6F71FFE9A996A
:109E6000039A9A9280AB03EB8100054640ABC36234
:109E7000B7EE000A2A63012180A8FEF779FF039A52
:109E80008DF8902272B6DDEDA07A9DED9F7A67EE97
:109E9000887AF4EEC77ACDED9E7ADDEDA27AF1EE06
:109EA00010FAD8BFF1EE677ACDEDA37A62B6DBF88F
:109EB000002024922499DBF800302393239B5B1A23
:109EC000042BF8D99BE700228DF8242372B6DDED30
:109ED000C57A9DEDC47A67EE887AF4EEC77ACDED47
:109EE000C37ADDEDC77AF1EE10FAD8BFF1EE677AEA
:109EF000CDEDC87A62B6DBF8002020922099DBF81D
:109F000000301F931F9B5B1A042BF8D9A5A8FEF7FE
:109F1000D5FC386B012800F0DC82022800F0D982E1
:109F200010B90146F6F7BAFDDBF80020229222991B
:109F3000DBF800302193219B5B1AB3F57A7FF7D3CE
:109F40009DF8040011F0F0FB00283FF4D9AE002486
:109F50001CE500BF9818FF1F2C07FF1FC09EF87F4D
:109F6000A79A002A7FF405ADB968D7ED067A039267
:109F7000494250A8F8EEE78A10F0D6FDC74910F024
:109F8000F7FD039A01211046F6F788FDBF99039A61
:109F9000BF92CAAB03EB8100044650AB40F8683C6B
:109FA000B7EE000A44F8642C0121A5A8FEF7E0FEF4
:109FB000039A8DF8242368EE898A72B6DDEDC57A9E
:109FC0009DEDC47A67EE887AF4EEC77ACDEDC37A58
:109FD000DDEDC77AF1EE10FAD8BFF1EE677ACDED7C
:109FE000C87A62B6DBF800201E921E99DBF80030BA
:109FF0001D931D9B5B1A042BF8D984E50821A84802
:10A0000013F05AFE0621A74813F056FE00228DF8E1
:10A01000902272B6DDEDA07A9DED9F7A67EE887A88
:10A02000F4EEC77ACDED9E7ADDEDA27AF1EE10FA6C
:10A03000D8BFF1EE677ACDEDA37A62B6DBF80020E7
:10A040001A921A99DBF800301993199B5B1A042BAA
:10A05000F8D980A8FEF732FC0821914813F02CFEB5
:10A060000721914813F028FE904814F0B5FA00211A
:10A070000320F6F713FD00257BE4A79A002A7FF45E
:10A0800078ACD7ED067AB968039250A8F8EEE78A63
:10A0900010F04AFD864910F06BFD039A012110462D
:10A0A000F6F7FCFCBF99039ABF92CAAB03EB8100A1
:10A0B000044650AB40F8683CB7EE000A44F8642C04
:10A0C0000121A5A8FEF754FE039A8DF8242368EE1B
:10A0D000898A72B6DDEDC57A9DEDC47A67EE887A1D
:10A0E000F4EEC77ACDEDC37ADDEDC77AF1EE10FA62
:10A0F000D8BFF1EE677ACDEDC87A62B6DBF8002002
:10A100001C921C99DBF800301B931B9B5B1A042BE1
:10A11000F8D991E4B968D7ED067AD7F82890519329
:10A120000293F369009301FB08F1B369019350A80E
:10A13000F8EEE78A10F0F8FC494610F0E9FC029BC3
:10A14000DFF870B1194610F02DFDDBF800300693F2
:10A15000069ADBF800300593059B9B1A042BF8D96F
:10A16000534950A810F01EFDFFF7CEBA8DF8240316
:10A1700072B6DDEDC57A9DEDC47A67EE887AF4EEAD
:10A18000C77AF1EE10FACDEDC37A40F38180DDEDB0
:10A19000C77ACDEDC87A62B6A5A8FEF78FFBD6F8D0
:10A1A0008C40002C3FF4F2AB00228DF8902272B666
:10A1B000DDEDA07A9DED9F7A67EE887AF4EEC77A9E
:10A1C000CDED9E7ADDEDA27AF1EE10FAD8BFF1EE78
:10A1D000677ACDEDA37A62B6DBF800203092309931
:10A1E000DBF800302F932F9B5B1A042BF8D980A843
:10A1F000FEF764FB00210D460320F6F74FFC2C46CA
:10A20000FFF7C4BB8DF8240372B6DDEDC57A9DED72
:10A21000C47A67EE887AF4EEC77AF1EE10FACDEDE3
:10A22000C37A30DDDDEDC77ACDEDC87A62B6A5A878
:10A23000FEF744FBD6F88C40002C3FF4A7AB00227D
:10A240008DF8902272B6DDEDA07A9DED9F7A67EED3
:10A25000887AF4EEC77ACDED9E7ADDEDA27AF1EE42
:10A2600010FAD8BFF1EE677ACDEDA37A62B6DBF8CB
:10A27000002032923299DBF800303193319B5B1A27
:10A28000042BF8D9B3E7DDEDC77AF1EE677ACBE7B7
:10A29000DDEDC77AF1EE677A7BE700BF40610780AA
:10A2A000AC5F0200E85F0200F05F0200E407FF1FFE
:10A2B000C09EF87F841BFF1F0821C548C54C13F0C2
:10A2C000FBFC0521C44813F0F7FC0721C34813F039
:10A2D000F3FCC34814F080F93B6B012B00F0F681CE
:10A2E000022B00F0EF8113B9519B236051957068E8
:10A2F0003368419A96ED027ADFEDBA6ABA49BB4DEE
:10A300000A6003FB00F307EE903A06EE102AF8EE1F
:10A31000677AB8EEC66A67EE877AB54986EE277A1D
:10A320003CA867EE267AC5ED007A14F021FB0021E7
:10A330003CA8F6F7A3FF3CA814F0DAFA2220F7F7BE
:10A340000FF995ED000A0020F7F7AEF82220F7F795
:10A3500007F9FF20F7F704F9FF20F7F701F9FF20CD
:10A36000F7F7FEF8DBF800303B933B9ADBF8003060
:10A370003A933A9B9F4E9B1A042BF7D99C493CA8D1
:10A3800014F0F6FA00213CA8F6F778FF3CA814F088
:10A39000AFFA2220F7F7E4F895ED000A0020F7F76E
:10A3A00083F82220F7F7DCF8FF20F7F7D9F8FF2031
:10A3B000F7F7D6F8FF20F7F7D3F833683993399ACF
:10A3C000DBF800303893389B8A4E9B1A042BF7D960
:10A3D00094ED000A386B884DB8EEC00AF6F76CFCB5
:10A3E000864985ED000A3CA814F0C2FA00213CA879
:10A3F000F6F744FF3CA814F07BFA2220F7F7B0F8F8
:10A4000095ED000A0020F7F74FF82220F7F7A8F89B
:10A41000FF20F7F7A5F8FF20F7F7A2F8FF20F7F7DE
:10A420009FF833683793379ADBF800303693369BC2
:10A43000704C9B1A042BF7D970493CA814F098FA79
:10A4400000213CA8F6F71AFF3CA814F051FA22208C
:10A45000F7F786F895ED000A0020F7F725F8222097
:10A46000F7F77EF8FF20F7F77BF8FF20F7F778F88B
:10A47000FF20F7F775F823683C933C9ADBF800302F
:10A480003593359B9B1A042BF8D900245C4B4194DF
:10A49000214603201C60F6F701FB21462046F6F713
:10A4A000FDFA21460120F6F7F9FA21460220F6F7D7
:10A4B000F5FA544BA593A5A8FEF794FA514B809357
:10A4C00080A8FEF78FFA0DF54B7DBDEC048BBDE83F
:10A4D000F08F0021F6F7E2FA26E501210320F6F7D6
:10A4E000DDFADBF800301693169ADBF8003015938E
:10A4F000159B9B1A042BF8D99A9B80A903F10B0298
:10A5000001EB820201EB83034FF0000940A8D862FF
:10A51000B7EE000A012180A8C2F80490CDF8689235
:10A52000FEF726FC8DF8909272B6DFED376ADDED0E
:10A53000A07A9DED9F7A67EEA67AF4EEC77ACDED0C
:10A540009E7ADDEDA27AF1EE10FAD8BFF1EE677ACD
:10A55000CDEDA37A62B6DBF800301493149ADBF8E1
:10A5600000301393139B9B1A092BF8D900238DF805
:10A57000903272B69DED037ADFED247A9DEDA06AEC
:10A58000DDED9F6AB8EEC77A67EE277A67EE867AC6
:10A59000F4EEE67ACDED9E7ADDEDA27AF1EE10FAD8
:10A5A000D8BFF1EE677ACDEDA37A62B608210848EC
:10A5B00013F082FB0421164813F07EFB01210848AA
:10A5C00014F05AF8064814F007F8FFF70AB900BF6C
:10A5D000AC5F02007412FF1FD85F0200F05F020040
:10A5E000E407FF1F0000B4436815FF1F3016FF1F6C
:10A5F000305F0200841BFF1F9015FF1F405F0200A9
:10A60000B812FF1FE84A0200000000000AD7233CEE
:10A61000E05F02003B683969D7ED087A0293336D39
:10A62000009301FB08F1F36C019370A8F8EEE78A40
:10A63000CDF8C49110F078FA029BDFF890B2194679
:10A6400010F066FA494610F0ADFADBF800300A93D4
:10A650000A9ADBF800300993099B9B1A042BF8D95E
:10A66000974970A810F09EFAFFF74EB8FB6AF96898
:10A67000D7ED077A0293336B009301FB08F1F36A7D
:10A68000019360A8F8EEE78ACDF8849110F04CFAB7
:10A69000029BDFF838B2194610F03AFA494610F03A
:10A6A00081FADBF800300893089ADBF80030079352
:10A6B000079B9B1A042BF8D9814960A810F072FA05
:10A6C000FFF722B8719B2360719510E6619B2360B0
:10A6D00061950CE607EE900AF8EEE78A086268EEEC
:10A6E000898AFFF7E5BA07EE900AF8EEE78AC861B3
:10A6F00068EE898AFFF7DCBA48460121F6F7CEF901
:10A70000BF9BCDF8FC92CAAA02EB830250A842F884
:10A71000680CB7EE000A0121A5A842F8649CFEF778
:10A7200027FB8DF8249372B6DFED666ADDEDC57AFE
:10A730009DEDC47A67EEA67AF4EEC77ACDEDC37AC2
:10A74000DDEDC77AF1EE10FAD8BFF1EE677ACDED04
:10A75000C87A62B6DBF800300E930E9ADBF8003050
:10A760000D930D9B9B1A092BF8D99FED577AD7EDC6
:10A77000067AF8EEE77A002367EE877A8DF82433BD
:10A7800072B6DDEDC56A9DEDC47A67EEA67AF4EE89
:10A79000C77ACDEDC37ADDEDC77AF1EE10FAD8BFF6
:10A7A000F1EE677ACDEDC87A62B6FFF708B8484691
:10A7B0000121F6F773F9BF9BCAA903F10B0201EB64
:10A7C000820201EB83034FF0000970A843F8680C84
:10A7D000B7EE000A0121A5A842F8909CCDF8FC92A2
:10A7E000FEF7C6FA8DF8249372B6DFED366ADDED1A
:10A7F000C57A9DEDC47A67EEA67AF4EEC77ACDED00
:10A80000C37ADDEDC77AF1EE10FAD8BFF1EE677AC0
:10A81000CDEDC87A62B6DBF800301293129ADBF8FD
:10A8200000301193119B9B1A092BF8D99FED267AC2
:10A83000D7ED087A9DE749464846F6F72FF90023F9
:10A840008DF8243372B6DFED1F6ADDEDC57A9DED1C
:10A85000C47A67EEA67AF4EEC77ACDEDC37ADDED61
:10A86000C77AF1EE10FAD8BFF1EE677ACDEDC87A6B
:10A8700062B6BF9BCAA903F10B0201EB820201EB96
:10A8800083034FF0000E60A943F8681CB7EE000A7E
:10A8900042F890ECA5A80121CDF8FCE2FEF768FA99
:10A8A000DBF800301093109ADBF800300F930F9B09
:10A8B0009B1A092BF8D99FED047AD7ED077A58E750
:10A8C000C09EF87F000000000AD7233C841BFF1FB6
:10A8D0002DE9F04F8B002DED028B00F12C0808EBD9
:10A8E0000305A84585B004460F46B0EE408A00F047
:10A8F00006819A10B2FA82F2C2F11F025200B64BE0
:10A9000029464046FEF7A0F9B34A29464046FEF7DD
:10A9100003F9E66AA665012F40F30B813069C6464C
:10A9200001225EF8041F0B690132C0EB430397421A
:10A930004B61F6DCA84500F02681D4F82C8004F1A8
:10A940003002D8F8183011460DE00F68BF6983EA6D
:10A95000E37E87EAE77CAEEBE37EACEBE77C043199
:10A96000F445B8BF3B468D42EFD1002BB8BF5B42E8
:10A9700007EE903AF8EEE77AD8F82430D6F81C8043
:10A98000366A67EE887AFCEEE77A17EE907A06E090
:10A990001168496A8B4202F1040228BF0B469542B6
:10A9A000F6D11D4600B127B905B0BDEC028BBDE85C
:10A9B000F08F4FF0000304F1040984F82830484672
:10A9C00010F0DCF92062484610F0D8F9606210F00F
:10A9D000A9F9616904F1080010F05AF9A36D5A68E9
:10A9E000DB68A267C2EB0309B9F1000FB8BFC9F178
:10A9F000000908FB08F306FB06F09B4607FB07F27D
:10AA0000CDF804904FF0000C00219146019BE367C4
:10AA1000B0EB0B0261EB0C03C4E926016D0010469C
:10AA200019465A4663464FF0000AC4E92423C4F885
:10AA30008870C4F884602A460023C4F8A850C4F87B
:10AA40008080C4E9289ACDE902BC16F0EDFA019A9B
:10AA5000801841EBE271CB0FC01841F100014F109B
:10AA60004FEA3006002E43DBB24241DBDDE902BC97
:10AA7000B9EB0B096AEB0C0A2A46002348465146FB
:10AA800016F0D2FA864240F38780C0EB4606C4F83F
:10AA9000B060C4F8AC00A368B8F1000F76D0002B0A
:10AAA0007FD01A684D498A4245D84D4AB2FBF8F228
:10AAB0001A60226A4B49E469002003250126DE6002
:10AAC000AA4098609D60086002F180434A6803F5DF
:10AAD000603322440D201A610860DA68502122F0A8
:10AAE0008002DA60D96005B0BDEC028BBDE8F08F62
:10AAF000192010F02DFE192010F02AFEF8E7C66A82
:10AB0000866501293FF70AAF30693246B369756A35
:10AB1000D2F81C80166A002BB8BF5B4207EE903A51
:10AB2000B8EEE77A67EE087AFCEEE77A17EE907AED
:10AB300038E7306901E758682949B1FBF8F1121A82
:10AB4000914209D38A1A0026012503209E60DD6008
:10AB50001A6098601960ACE76069026800270125F7
:10AB600003269F601268DD6019609E609047A368AD
:10AB7000002B9ED11C4A1268002A9AD02846022136
:10AB80009047A36895E73246E66ABFE7DBB19A686B
:10AB900022F002029A608CE7C4F8B060C4F8AC609E
:10ABA00079E7114A0E4D1268B5FBF8F51AB102218A
:10ABB00001209047A3680020012103229860D960FA
:10ABC0001D609A6075E7084B1B687BB1022101206C
:10ABD0009847A368DBE700BF6D0400007FA903006E
:10ABE00000879303008003404C1BFF1F4346CEE7C2
:10ABF0002DE9F04F2DED028BEBB0044641F2883287
:10AC000088463CA80521FDF7A3FE174B3C9305227F
:10AC1000002306210CA857930FF044FF142215219E
:10AC20001CA80FF03FFF114E172210212CA80FF087
:10AC300039FF35210E48356813F03EF80D4813F002
:10AC4000CBFC21460B4813F017FD0A4813F0C4FC57
:10AC5000052C00F2E780DFE814F0C502C903D50433
:10AC60005706D5060F0000BF044B02007412FF1FE9
:10AC7000F85F0200E407FF1FDFF880A3DFF880938E
:10AC8000DAF8343099ED0F0A002B40F02B87F6F7F5
:10AC900045F810EE100A15F01DFDCDE90001D9F8B8
:10ACA0002420D9F81C309FEDC27A03FB02F308EE92
:10ACB000103AF8EEC87A002727EE878A2CA8FDEE16
:10ACC000C87A2D9717EE901A0FF02EFFD9F82010A2
:10ACD0000FF01EFF8346404615F0EAFCDDE9002335
:10ACE00015F04CFD15F0FAFF014658460FF05AFFDB
:10ACF0000D21B04812F0E0FFDAF8440015F0EAFC4C
:10AD000041EC100B0221AC4813F0BEFCAA4813F032
:10AD100063FC0A21A94812F0CFFF3B460A22DAF869
:10AD20003C10A54813F068FCA34813F055FC0B2118
:10AD3000A34812F0C1FF3B46DAF838109E480A22B9
:10AD400013F05AFC9C4813F047FC09219D4812F06F
:10AD5000B3FFD9F83C0015F0BDFC41EC100B042109
:10AD6000954813F091FC944813F036FC0621964860
:10AD700012F0A2FF9DED000B02218F4813F084FC1E
:10AD80008D4813F029FC0A21904812F095FFD9F85C
:10AD90001C10894813F070FC874813F01DFC0E212D
:10ADA0008B4812F089FFD9F82410834813F064FC13
:10ADB000814813F011FC0B21864812F07DFF18EE3C
:10ADC000100A15F087FC41EC100B02217A4813F0B1
:10ADD0005BFC794813F000FC06217F4812F06CFF01
:10ADE0003B460A22D9F82010734813F005FC72483C
:10ADF00013F0F2FB01210220F5F750FE569B569707
:10AE000003F10B026AA901EB820E01EB83032CAA6A
:10AE100043F88C2CB7EE000A01213CA84EF8B47C14
:10AE2000FFF756FD3E9B002B41D0DFF8D8B1DFF88D
:10AE3000D8A1DFF8D891DFF8D8810027F6F73AFFDC
:10AE4000002809DBDAF80000F6F724FFC0B2532827
:10AE500089F8000000F0A180DBF800300493049A28
:10AE6000DBF800300393039B9B1A092BF8D988FB6E
:10AE70000723FA17C2EB2313322202FB137393B991
:10AE8000012C00F09380022C00F08E8004B90D9DFF
:10AE90005248092112F010FF2946474813F0ECFBF5
:10AEA000454813F099FB3E9B0137002BC6D14C4916
:10AEB00008A813F05DFD002108A8F6F7DFF908A83F
:10AEC00013F016FD474908A813F052FD002108A809
:10AED000F6F7D4F908A813F00BFD434908A813F0BE
:10AEE00047FD002108A8F6F7C9F908A813F000FDEE
:10AEF0003C4908A813F03CFD002108A8F6F7BEF96C
:10AF000008A813F0F5FC394908A813F031FD002119
:10AF100008A8F6F7B3F908A813F0EAFC314908A825
:10AF200013F026FD002108A8F6F7A8F908A813F0E9
:10AF3000DFFC2F4908A813F01BFD002108A8F6F735
:10AF40009DF908A813F0D4FC264908A813F010FDB9
:10AF500008A80021F6F792F908A813F0C9FC012C03
:10AF600000F00B81022C00F0F480002C52D0002164
:10AF70000846F5F793FD00210120F5F78FFD00212C
:10AF80000220F5F78BFD1B4B3C933CA8FDF72AFDF7
:10AF90006BB0BDEC028BBDE8F08F3CA8FDF7CAFC9E
:10AFA000154B01221A7057E72D9D71E71D9D6FE724
:10AFB0000AD7233C30600200E407FF1F4060020014
:10AFC0004C600200586002001C62020064600200D3
:10AFD0005473020070600200B0610200F060020071
:10AFE000A0600200604E0200B4600200C86002006F
:10AFF000DC600200044B0200A016FF1FDC17FF1FDD
:10B000009815FF1F841BFF1F1007FF1FE816FF1F67
:10B010001F85EB5169496A4DDFF8C0B108A813F0EC
:10B02000A7FC214608A8F6F729F908A813F060FC48
:10B030002220F6F795FA634B204693ED000AF6F7C7
:10B0400033FA614908A813F093FC214608A8F6F7E3
:10B0500015F908A813F04CFC32680D9B5B481344AB
:10B060000921336012F028FE3168594813F004FBBF
:10B07000574813F0B1FA574A96ED007A1069D36831
:10B08000D2ED056A544903FB00F307EE903AB8EE9F
:10B09000C77AF8EE677A27EE267A08A8C7EE276AFD
:10B0A000C5ED006A13F064FC214608A8F6F7E6F83F
:10B0B00008A813F01DFC2220F6F752FA95ED000ABD
:10B0C0002046F6F7F1F92220F6F74AFAFF20F6F7C4
:10B0D00047FAFF20F6F744FAFF20F6F741FADBF8CB
:10B0E00000300793079ADBF800300693069B3B4C31
:10B0F0009B1A042BF7D9384908A813F039FC002112
:10B1000008A8F6F7BBF808A813F0F2FB2220F6F720
:10B1100027FA95ED000A0020F6F7C6F92220F6F787
:10B120001FFAFF20F6F71CFAFF20F6F719FAFF20A6
:10B13000F6F716FA23680893089ADBF800300593AF
:10B14000059B9B1A042BF8D900210846F5F7A6FCAD
:10B150000DE72D9B32681D4813440921336012F01E
:10B16000ABFD31681A4813F087FA194813F034FA26
:10B1700020460021F5F792FCF9E6104908A813F0E3
:10B18000F7FB002108A8F6F779F808A813F0B0FB40
:10B190002220F6F7E5F9124B002093ED000AF6F7AE
:10B1A00083F9094908A813F0E3FB002108A8F6F782
:10B1B00065F808A813F09CFB1D9BCBE7FC60020020
:10B1C0009015FF1F9418FF1F74500200F0600200DA
:10B1D000E407FF1FDC17FF1F405F0200841BFF1FF7
:10B1E0009018FF1F734FDFF800A2D7ED0A6ADAED5F
:10B1F000057ADAF81020DAF80C3086EEA77A03FB2D
:10B2000002F307EE903AF8EE677A67EE877A17EE68
:10B21000900A15F05FFAFA687B689FED677A03FB86
:10B2200002F308EE103AF8EEC87A0CAB27EE878AE4
:10B23000CDE90001FDEEC87A184617EE901A0FF01E
:10B2400073FCB9680FF064FC8346404615F030FA91
:10B25000DDE9008942464B4615F090FA15F03EFDB7
:10B26000014658460FF09EFC3521544812F024FD4B
:10B27000534813F0B1F90021514813F0FDF950483B
:10B2800013F0AAF90D214F4812F016FDDAF8140058
:10B2900015F020FA41EC100B0221494813F0F4F9A3
:10B2A000474813F099F90A21474812F005FDDAF8EA
:10B2B0001010434800230A2213F09EF9404813F06F
:10B2C0008BF90B21414812F0F7FC00230A22DAF82F
:10B2D0000C103B4813F090F9394813F07DF909211F
:10B2E0003B4812F0E9FCB86A15F0F4F941EC100B98
:10B2F0000221334813F0C8F9314813F06DF90621E3
:10B30000344812F0D9FC49EC108B02212C4813F080
:10B31000BBF92B4813F060F90A212F4812F0CCFC3E
:10B320007968274813F0A8F9254813F055F90E213C
:10B330002A4812F0C1FCF968214813F09DF9204811
:10B3400013F04AF90B21264812F0B6FC18EE100A49
:10B3500015F0C0F941EC100B0221194813F094F9D3
:10B36000174813F039F906211E4812F0A5FCB968F8
:10B37000134800230A2213F03FF9114813F02CF967
:10B3800001210020F5F78AFB569B6AA903F10B0205
:10B3900001EB820E01EB830300270CAA43F88C2CEF
:10B3A000B7EE000A01213CA84EF8B47C5697FFF78F
:10B3B0008FFA37E59815FF1F0AD7233CF85F020084
:10B3C000E407FF1F30600200406002004C60020092
:10B3D000586002001C6202006460020054730200A4
:10B3E00070600200B0610200DC17FF1FDFF80C92F2
:10B3F000DFF80CB2D9ED0D6ADBED057ADBF8102031
:10B40000DBF80C3086EEA77A03FB02F300270D97DA
:10B4100007EE903AF8EE677A67EE877A17EE900AB1
:10B4200015F058F9D9F80C20D9F804309FED677A57
:10B4300003FB02F308EE103AF8EEC87A0CAB27EEE5
:10B44000878ACDE90001FDEEC87A184617EE901AFA
:10B450000FF06AFBD9F808100FF05AFB82464046FD
:10B4600015F026F9DDE9002315F088F915F036FC12
:10B47000014650460FF096FB3521554812F01CFC52
:10B48000544813F0A9F80121524813F0F5F8514837
:10B4900013F0A2F80D21504812F00EFCDBF8140056
:10B4A00015F018F941EC100B02214A4813F0ECF8A2
:10B4B000484813F091F80A21484812F0FDFB3B463A
:10B4C000DBF8101043480A2213F096F8414813F0B5
:10B4D00083F80B21424812F0EFFB3B460A22DBF8CF
:10B4E0000C103C4813F088F83A4813F075F809211D
:10B4F0003C4812F0E1FBD9F8340015F0EBF841ECD0
:10B50000100B0221334813F0BFF8324813F064F8EF
:10B510000621354812F0D0FB9DED000B02212D488D
:10B5200013F0B2F82B4813F057F80A212F4812F005
:10B53000C3FBD9F80410274813F09EF8254813F0F0
:10B540004BF80E212A4812F0B7FBD9F80C1021480D
:10B5500013F092F81F4813F03FF80B21254812F022
:10B56000ABFB18EE100A15F0B5F841EC100B0221F8
:10B57000184813F089F8174813F02EF806211E48D2
:10B5800012F09AFB3B46D9F8081012480A2213F031
:10B5900033F8104813F020F838460121F5F77EFA09
:10B5A000569B56976AA903F10B0201EB820E01EB41
:10B5B00083030CAA43F88C2CB7EE000A01213CA8A7
:10B5C0004EF8B47CFFF784F92CE400BF0AD7233C83
:10B5D000F85F0200E407FF1F3060020040600200D5
:10B5E0004C600200586002001C62020064600200AD
:10B5F0005473020070600200B06102009815FF1FD2
:10B60000DC17FF1FDFF8F8A2B148DFF8F892072136
:10B6100012F052FBDAF89010AE4800230A2212F022
:10B62000EBFFAC4812F0D8FFDAF89070002F40F032
:10B630006C82D9ED0B6ADAED0A7ADAF82420DAF8AE
:10B64000203086EEA77A03FB02F307EE903AF8EE7D
:10B65000677A67EE877A17EE900A15F03BF8CDE926
:10B6600000010D219C4812F027FBDAF8280015F0A4
:10B6700031F841EC100B0221964813F005F895487B
:10B6800012F0AAFF0A21954812F016FB3B460A2247
:10B69000DAF824108F4812F0AFFF8E4812F09CFFAA
:10B6A0000B218F4812F008FB3B460A22DAF82010E3
:10B6B000884812F0A1FF874812F08EFF09218948BF
:10B6C00012F0FAFAD9F82C0015F004F841EC100B3E
:10B6D0000221804812F0D8FF7E4812F07DFF06213B
:10B6E000814812F0E9FA9DED000B0221794812F031
:10B6F000CBFF784812F070FF0A217C4812F0DCFA88
:10B70000D9F81010734812F0B7FF724812F064FFB6
:10B710000E21774812F0D0FAD9F818106D4812F0BF
:10B72000ABFF6C4812F058FF0621724812F0C4FAC1
:10B730003B46D9F8141067480A2212F05DFF6548AD
:10B7400012F04AFFD9F81820D9F810309FED6A7A24
:10B7500003FB02F308EE103AF8EEC87A002727EE52
:10B76000878A1CA8FDEEC87A1D9717EE901A0FF075
:10B77000DBF9D9F814100FF0CBF98346404614F0EA
:10B7800097FFDDE9002314F0F9FF15F0A7FA014651
:10B7900058460FF007FA0D214F4812F08DFADAF8EB
:10B7A000280014F097FF41EC100B0221494812F0D9
:10B7B0006BFF484812F010FF0A21484812F07CFA4B
:10B7C0003B460A22DAF82410424812F015FF41489D
:10B7D00012F002FF0B21424812F06EFA3B46DAF8F3
:10B7E00020103C480A2212F007FF3A4812F0F4FEFB
:10B7F00009213C4812F060FAD9F82C0014F06AFFD5
:10B8000041EC100B0221334812F03EFF314812F098
:10B81000E3FE0621344812F04FFA9DED000B0221A1
:10B820002C4812F031FF2B4812F0D6FE0A212F4887
:10B8300012F042FAD9F81010264812F01DFF2548E0
:10B8400012F0CAFE0E212A4812F036FAD9F8181062
:10B85000204812F011FF1F4812F0BEFE0B212748AE
:10B8600012F02AFA18EE100A14F034FF41EC100B13
:10B870000221184812F008FF164812F0ADFE06210A
:10B880001C4812F019FA3B46D9F8141011480A2244
:10B8900012F0B2FE0F4812F09FFE01210846F5F7A4
:10B8A000FDF8569B56976AA903F10B0201EB820E35
:10B8B00001EB83031CAA43F88C2CB7EE000A01218C
:10B8C0003CA84EF8B47CFFF703F8FFF7ABBA00BF13
:10B8D0007C600200E407FF1F30600200406002004D
:10B8E0004C600200586002001C62020064600200AA
:10B8F00054730200B06102000AD7233C706002005A
:10B90000DC17FF1F9815FF1FDFF8E8A2DFF8E892A9
:10B91000DAF89030002B40F05681DAED0A7AD9ED52
:10B920000E6ADAF82420DAF8203086EEA77A03FBD4
:10B9300002F3002707EE903AF8EE677A67EE877A0F
:10B9400017EE900A14F0C6FED9F81820D9F8103076
:10B950009FEDA17A1D9703FB02F308EE103AF8EE73
:10B96000C87ACDE9000127EE878A1CA8FDEEC87AC7
:10B9700017EE901A0FF0D8F8D9F814100FF0C8F895
:10B980008346404614F094FEDDE9002314F0F6FEF1
:10B9900015F0A4F9014658460FF004F90D218F481F
:10B9A00012F08AF9DAF8280014F094FE41EC100B3A
:10B9B00002218B4812F068FE894812F00DFE0A2120
:10B9C000884812F079F93B460A22DAF824108448B4
:10B9D00012F012FE824812F0FFFD0B21824812F095
:10B9E0006BF93B46DAF820107D480A2212F004FE7B
:10B9F0007B4812F0F1FD09217C4812F05DF9D9F87D
:10BA00003800FBE6DFF8ECA1DFF8EC91DAF834302F
:10BA100099ED0C0A002B6FD1F5F780F910EE100AA2
:10BA200014F058FECDE90001D9F82420D9F81C30D3
:10BA30009FED697A03FB02F308EE103AF8EEC87A3C
:10BA4000002727EE878A2CA8FDEEC87A2D9717EEDF
:10BA5000901A0FF069F8D9F820100FF059F88346C2
:10BA6000404614F025FEDDE9002314F087FE15F0B2
:10BA700035F9014658460FF095F80D21574812F058
:10BA80001BF9DAF8440014F025FE41EC100B0221FA
:10BA9000534812F0F9FD524812F09EFD0A21514818
:10BAA00012F00AF93B460A22DAF83C104C4812F030
:10BAB000A3FD4B4812F090FD0B214B4812F0FCF80F
:10BAC0003B46DAF8381046480A2212F095FD444801
:10BAD00012F082FD0921454812F0EEF8D9F8300045
:10BAE000FFF739B9F5F7B4F910EE100A14F0F2FDCA
:10BAF000CDE90001FFF7D3B8F5F7AAF910EE100A67
:10BB000014F0E8FDCDE900018EE7D9ED0B6ADAED1E
:10BB1000277ADAF89820DAF8943086EEA77A03FBD1
:10BB200002F307EE903AF8EE677A67EE877A17EE3F
:10BB3000900A14F0CFFDCDE9000118212C4812F035
:10BB4000BBF8274812F048FD0D21244812F0B4F844
:10BB5000DAF89C0014F0BEFD41EC100B02212048E5
:10BB600012F092FD1E4812F037FD0A211D4812F016
:10BB7000A3F800230A22DAF89810194812F03CFDC5
:10BB8000174812F029FD0B21174812F095F80023F1
:10BB90000A22DAF89410124812F02EFD104812F022
:10BBA0001BFD0921114812F087F8D9F82C0014F078
:10BBB00091FD41EC100B0221094812F065FD084887
:10BBC00012F00AFDBEE5DAED277AD9ED0E6ADAF851
:10BBD0009820DAF89430A8E60AD7233C30600200B7
:10BBE000E407FF1F406002004C6002005860020042
:10BBF00084600200DC17FF1F9815FF1F2DE9F04F2E
:10BC0000CE4DCF4AAB6C2DED028BE3B00026012B5D
:10BC10000190166000F01685C0F0BE84022B00F083
:10BC2000068334460396B1463746B346B24614AE51
:10BC300041F28832052134A8FCF78AFE4FF0000853
:10BC4000C04B3493022203213046CDF83C810EF0E4
:10BC500029FF51465A4624A80EF024FF2A682B6972
:10BC60009FEDB97ADFF8D4A203FB02F307EE903A16
:10BC7000F8EEE77A304667EE877AFDEEE77A17EE60
:10BC8000901A0EF051FF296A0EF042FFEB6CC6F8D5
:10BC90000480002B00F00484012B40F073849AEDA3
:10BCA0000F6A9FEDAA7ADFF8F4B2DAF84800DBED0C
:10BCB000027A9AED0E0ADAF83080C6EE076A9BE83F
:10BCC0000C0003FB02F308F104084FEA480807EEF2
:10BCD000103AB8EE477A9DED016A67EE277AB8EE22
:10BCE000C68A67EEA67A67EE887AFDEEE77ACDED32
:10BCF000017AF5F7DDF8DAF830305B0007EE903ABC
:10BD0000F8EEE77A80EE270A20EE088AFDEEC87A80
:10BD1000CDED027A3B218E48DFF820A211F0CCFF56
:10BD20008C4812F059FC0D218B4811F0C5FF019988
:10BD3000884812F0A1FC874812F04EFC1121874878
:10BD400011F0BAFF864B8348196812F095FC8148C0
:10BD500012F042FC0A21834811F0AEFF02997D489F
:10BD600012F08AFC7B4812F037FC3B21784811F036
:10BD7000A3FF784812F030FC039924A80EF0D4FEFB
:10BD800021460EF0C5FE00240E217748259411F0BF
:10BD900093FF29686F4812F06FFC6E4812F01CFC8C
:10BDA0001421724811F088FF29696A4812F064FC76
:10BDB000684812F011FC0D216D4811F07DFF2346FB
:10BDC0000A22296A634812F017FC624812F004FC48
:10BDD0001321684811F070FF23460A22DBF8001097
:10BDE0005C4812F009FC5B4812F0F6FB1121624836
:10BDF00011F062FF23460A22DBF80410554812F0C6
:10BE0000FBFB544812F0E8FB12215C4811F054FF90
:10BE1000DBF8080014F05EFC41EC100B02214D48E9
:10BE200012F032FC4B4812F0D7FBEB6C002B00F009
:10BE30007A83012B2DD11021514811F03DFFDAF802
:10BE40003C0014F047FC41EC100B0221414812F079
:10BE50001BFC404812F0C0FB0F214A4811F02CFF98
:10BE6000DAF8380014F036FC41EC100B02213948A6
:10BE700012F00AFC374812F0AFFB0C21424811F0D7
:10BE80001BFFDAF83010334812F0F6FB314812F09D
:10BE9000A3FB0D21304811F00FFF01992D4812F03E
:10BEA000EBFB2C4812F098FB0A212E4811F004FFFE
:10BEB0000299284812F0E0FB264812F08DFB0B2176
:10BEC000324811F0F9FE0399224812F0D5FB2148BF
:10BED00012F082FB11212E4811F0EEFE49461D485A
:10BEE00012F0CAFB1B4812F077FB0A21294811F017
:10BEF000E3FE3946174812F0BFFB164812F06CFB00
:10BF000001210320F4F7CAFDA96C012900F0DB83AD
:10BF1000C0F0D48302290AD108460121F4F7BEFDFE
:10BF200023211D4811F0C8FE0A4812F055FBB8F154
:10BF3000040F40F38580DFF868A033E06414FF1F2E
:10BF4000B812FF1F044B02000AD7233C0000B44381
:10BF5000B8610200E407FF1FF461020004620200FE
:10BF60007412FF1F18620200246202003462020091
:10BF70004C6202005C620200706202008462020095
:10BF8000D8620200EC620200FC62020084610200DE
:10BF900094610200AC6102000C630200DC17FF1F19
:10BFA0001007FF1FDFF85C93042404F0030705214A
:10BFB000BC4811F081FE3946BB4812F05DFBBA481F
:10BFC00012F00AFB022F00F0E181032F00F0B48190
:10BFD000012F00F0B181EF6C002F00F00182012FE2
:10BFE00028D1019930460EF0DDFD4E9A62AB02F188
:10BFF0000B0E03EB8E0E03EB8202002342F88C6CD7
:10C0000039464EF8B43CB7EE000A34A84E93FEF71A
:10C010005FFCA64B1A68079207991A680692069A5F
:10C02000521A042AF9D9369B3BB1F5F743FE002892
:10C0300000F36A81369B002BF7D101344445B4D11B
:10C04000DBF80400DBF80030259972689BED027A7A
:10C05000DFED976A974C984F984D226003FB00F3F1
:10C0600007EE903A06EE102AF8EE677AB8EEC66A46
:10C0700067EE877A07EE101AB8EEC70A86EE277ABF
:10C0800029608F4D67EE267AC7ED007AF4F760FAE3
:10C0900010A88C4985ED000A12F06AFC002110A856
:10C0A000F5F7ECF810A812F023FC2220F5F758FA67
:10C0B00097ED000A0020F5F7F7F910A8824912F071
:10C0C00057FC10A80021F5F7D9F810A812F010FCC1
:10C0D00010A87E4912F04CFC002110A8F5F7CEF80C
:10C0E00010A812F005FC2220F5F73AFA95ED000AA7
:10C0F0000020F5F7D9F910A8734912F039FC10A8FF
:10C100000021F5F7BBF810A812F0F2FB10A8704957
:10C1100012F02EFC10A80021F5F7B0F810A812F0CC
:10C12000E7FB10A86B4912F023FC10A80021F5F7DB
:10C13000A5F810A812F0DCFB10A8674912F018FC53
:10C1400010A80021F5F79AF810A812F0D1FB10A85A
:10C15000604912F00DFC10A80021F5F78FF810A827
:10C1600012F0C6FB10A85D4912F002FC10A80021D5
:10C17000F5F784F810A812F0BBFB10A8554912F08F
:10C18000F7FB10A80021F5F779F810A812F0B0FB22
:10C1900010A8534912F0ECFB10A80021F5F76EF837
:10C1A00010A812F0A5FB10A84A4912F0E1FB10A854
:10C1B0000021F5F763F810A812F09AFB259B72682E
:10C1C00022603E4A47481360082111F075FD21683E
:10C1D000354812F051FA344812F0FEF90521424870
:10C1E00011F06AFD354B3048196812F045FA2E48B7
:10C1F00012F0F2F93D4B22681A6000210320F4F797
:10C200004DFC00210846F4F749FC00210120F4F719
:10C2100045FC00210220F4F741FC354B349334A84F
:10C22000FCF7E0FB63B0BDEC028BBDE8F08FD5F806
:10C230001C90EB689FED2F7A2F48EC6A03FB09F303
:10C2400007EE903AF8EEE77A0F2167EE877A2746F5
:10C25000FDEEE77A4FF0170BCDED037A11F02CFDD0
:10C26000E968114812F008FA0F4812F0B5F91521E3
:10C27000224811F021FDE9690B4812F0FDF90A4846
:10C2800012F0AAF90E211E4811F016FD33460A22BB
:10C29000E96A054812F0B0F9034812F09DF94FF031
:10C2A000100AC4E430630200E407FF1F841BFF1F71
:10C2B0000000B4434017FF1F3016FF1F7412FF1F0A
:10C2C0009015FF1F305F020074500200405F0200B3
:10C2D00054630200604E0200686302007C63020047
:10C2E000906302009C650200106202006815FF1F47
:10C2F000044B02000AD7233C8061020090610200D7
:10C30000A8610200E816FF1FDAF80000F5F7C2FC8A
:10C31000C0B2532889F800007FF48CAE1A21BC48C3
:10C3200011F0CAFCBB4812F057F934A8FCF702FB25
:10C33000B94B01221A7083E6EF6C002F70D0012FE9
:10C340007FF478AE029924A80EF02CFC4E9A62ABD2
:10C3500002F10B0E03EB8E0E03EB820224A80023E6
:10C3600042F88C0C39464EF8B43CB7EE000A34A8BB
:10C370004E93FEF7ADFAA94B1A680B920B991A6807
:10C380000A920A9A521A042AF9D953E6EF6C002F3E
:10C3900065D0012F7FF44EAE019B304659420EF01E
:10C3A00001FC4E9A62AB02F10B0E03EB8E0E03EB17
:10C3B0008202002342F88C6C39464EF8B43CB7EE4A
:10C3C000000A34A84E93FEF783FA944B1A680F9232
:10C3D0000F991A680E920E9A521A042AF9D929E670
:10C3E000029924A80EF0DEFB4E9A4E9762AB03EB47
:10C3F0008200024624AB40F88C3C012142F8887C44
:10C40000B7EE000A34A8FEF763FA844B1A68059267
:10C4100005991A680492049A521A042AF9D909E66D
:10C42000019930460EF0BEFB4E9A4E9762AB03EB7D
:10C430008200024640F88C6C012142F8887CB7EEFD
:10C44000000A34A8FEF744FA744B1A680992099955
:10C450001A680892089A521A042AF9D9EAE5029B46
:10C4600024A859420EF09EFB4E9A4E9762AB03EB06
:10C470008200024624AB40F88C3C012142F8887CC3
:10C48000B7EE000A34A8FEF723FA644B1A680D923F
:10C490000D991A680C920C9A521A042AF9D9C9E516
:10C4A000DAF834309AED117ADFED5D5ADFF88CB1AD
:10C4B0004FEA430807EE908AF8EEE77A9BE80C0013
:10C4C00087EE275A03FB02F308F1080807EE903ABB
:10C4D000C5EE256A9BED026AB8EE677A67EE067ACA
:10C4E0009DED017A67EEA67AB8EEC78A67EE887A84
:10C4F00017EE900A14F0EEF841EC100B12F02CFE3F
:10C5000051EC100B14F0EAFB9AED100A0190DAF8E6
:10C510004800F4F7CDFC28EE000AFDEEC07ACDED20
:10C52000027AFFF7F7BB0F213E4811F0C5FBDAF89E
:10C53000440014F0CFF841EC100B0221354812F002
:10C54000A3F8344812F048F81C21374811F0B4FB26
:10C55000DAF8400014F0BEF841EC100B02212D482F
:10C5600012F092F82B4812F037F80D212F4811F0F5
:10C57000A3FBDAF83410274812F07EF8254812F0B1
:10C580002BF886E4CDF80880CDF80480DFF8ACB055
:10C590004FF00808FFF7BEBBD5F814906B689FED0D
:10C5A000287A23486C6A03FB09F307EE903AF8EE09
:10C5B000E77A0F2167EE877A2746FDEEE77A4FF09C
:10C5C000050BCDED037A11F077FB6968114812F085
:10C5D00053F8104812F000F81521164811F06CFBC2
:10C5E00069690C4812F048F80A4811F0F5FF0E216D
:10C5F000114811F061FB33460A22696A054811F0BF
:10C60000FBFF044811F0E8FF4FF0060AFFF70FBBED
:10C6100038630200E407FF1FA016FF1F841BFF1FE3
:10C620000000B44398620200A8620200C8620200DF
:10C63000106102002061020038610200DC17FF1F58
:10C640000AD7233CD5F81890AB681FED037A204831
:10C65000AC6A03FB09F307EE903AF8EEE77A0F2194
:10C6600067EE877A2746FDEEE77A4FF0140BCDEDA3
:10C67000037A11F021FBA968164811F0FDFF154857
:10C6800011F0AAFF1521144811F016FBA9691148F1
:10C6900011F0F2FF0F4811F09FFF0E210F4811F02B
:10C6A0000BFB33460A22A96A0A4811F0A5FF094884
:10C6B00011F092FF4FF0150AFFF7B9BA01210020DF
:10C6C000F4F7ECF933E40846F4F7E8F92FE400BF97
:10C6D00048610200E407FF1F586102007061020018
:10C6E0002DE9F04F2DED068BC9B0C44D01900E46DB
:10C6F00006A8C349B0EE408AF0EE608A12F038F91D
:10C700002C683EB9012C00F03482C0F0CB81022CA1
:10C7100000F0C8813021BB4811F0CEFA2146BA485A
:10C7200011F0AAFFB84811F057FF1721B74811F0D0
:10C73000C3FA18EE100A13F0CDFF41EC1A0B0221D8
:10C74000B0EE4A0AF0EE6A0AAF4811F09DFFAE481B
:10C7500011F042FF1521AE4811F0AEFA18EE900A22
:10C7600013F0B8FF41EC190B0221B0EE490AF0EECC
:10C77000690AA54811F088FFA34811F02DFF19217F
:10C78000A44811F099FA31469F4811F075FF9E4870
:10C7900011F022FF012C00F0CD81022C00F0AB81C2
:10C7A000002C00F0608100270097BB4602973B46B3
:10C7B000BA463D460DF1280841F2883205211AA8F3
:10C7C0000393FCF7C5F85246934B1A93294640460B
:10C7D000002535950EF066F9DDED017ADFF87892E7
:10C7E00028EE288AF8EEE77A68EE277A17EE900AA4
:10C7F00013F070FF41EC100B12F0AEFC51EC100B7B
:10C8000014F06CFA0099824640460EF08DF93946D4
:10C810000EF07EF951460EF0C5F903217F480B95C5
:10C8200011F04AFA06A9784811F0B0FE19217C48A7
:10C8300011F042FA06A9744811F0A8FE03217748C6
:10C8400011F03AFA704811F0C7FE0E21754811F048
:10C8500033FAB0EE4A0AF0EE6A0A02216A4811F091
:10C8600013FF694811F0B8FE0C216F4811F024FA4B
:10C87000B0EE490AF0EE690A0221634811F004FFA4
:10C88000614811F0A9FE0B21684811F015FA0199D1
:10C890005D4811F0F1FE5C4811F09EFE0D216448E8
:10C8A00011F00AFA5146584811F0E6FE564811F0C8
:10C8B00093FE0D215F4811F0FFF90099524811F0E5
:10C8C000DBFE514811F088FE0A215B4811F0F4F9B3
:10C8D000039B4D48194611F0CFFE4B4811F07CFEEA
:10C8E0000E21564811F0E8F90299474811F0C4FEAC
:10C8F000454811F071FE1121514811F0DDF95946FA
:10C90000414811F0B9FE404811F066FE03214D4840
:10C9100011F0D2F906A93C4811F038FE192140481F
:10C9200011F0CAF906A9384811F030FE0321454834
:10C9300011F0C2F9344811F04FFE349B349548AAE7
:10C9400003F10B0702EB870702EB83031AA843F8F6
:10C950008C8CB7EE000A012147F8B45CFDF7B8FFF4
:10C960001C9890B1F5F7DCF9002840F0A880D9F8C0
:10C9700000300593059AD9F800300493049B9B1A64
:10C98000042BF8D91C980028ECD105462E4F2F48CF
:10C99000112111F091F939681B4811F06DFE1A4808
:10C9A00011F01AFE1EB13A680B9B13443B60112133
:10C9B000264811F081F93968134811F05DFE1248DC
:10C9C00011F00AFE1A21224811F076F921460E488C
:10C9D00011F052FE0C4811F0FFFD17211D4811F017
:10C9E0006BF9094811F0F8FD0B4B1A931AA8FBF7E5
:10C9F000F9FF06A811F07CFF28462FE0F813FF1F6F
:10CA0000B4630200CC630200E407FF1F006402006D
:10CA10001864020030640200044B0200F06102005E
:10CA20004C640200686402007864020088640200BA
:10CA300094640200A4640200B85F0200B4640200BF
:10CA4000C4640200306C02007412FF1F0462020012
:10CA5000F06402000C650200841BFF1F49B0BDECAE
:10CA6000068BBDE8F08F494906A812F009F80121AC
:10CA70002046F4F713F86B6BD5F844B09FED447A79
:10CA80006F6D02970BFB03F207EE902AF8EEE77A40
:10CA90004FF0050A67EE877A0625FDEEE77ACDEDC1
:10CAA000007A87E610213B4811F006F901213A4847
:10CAB00011F0E2FD384811F08FFD01242AE617211C
:10CAC000364811F0F9F8344811F086FD1AA8FBF742
:10CAD00031FF00210320F3F7E1FF00210846F3F7BF
:10CAE000DDFF00210120F3F7D9FF00210220F3F739
:10CAF000D5FF01254AE72A4906A811F0C1FF012107
:10CB00002046F3F7CBFFEB6BD5F84CB09FED207AC6
:10CB1000EF6D02970BFB03F207EE902AF8EEE77A2F
:10CB20004FF0170A67EE877A1025FDEEE77ACDED14
:10CB3000007A3FE61B4906A811F0A2FF21462046D5
:10CB4000F3F7ACFFAB6BD5F848B09FED117AAF6D42
:10CB500002970BFB03F207EE902AF8EEE77A4FF00C
:10CB6000140A67EE877A1525FDEEE77ACDED007A97
:10CB700020E610210C4811F09FF83146064811F0CC
:10CB80007BFD054811F028FD3446C3E5B05C02008A
:10CB90000AD7233CA4630200E407FF1FD864020005
:10CBA000785D0200787E0200B86302002DE9F04350
:10CBB0002DED048BC3B0322101908A488A4EDFF8F4
:10CBC0005C829FED8A9A8A4FF0EE408AB0EE608ACE
:10CBD00011F072F8874811F0FFFC01210320F3F7F0
:10CBE0005DFF04AC41F28832052114A8FBF7B0FECA
:10CBF0000025204602220321CDF850802F950DF00C
:10CC000051FF326B336C03FB02F307EE903AF8EE00
:10CC1000E77A204667EE897AFDEEE77A17EE901AFA
:10CC20000DF082FF316D0DF073FF326B336C724E7D
:10CC300003FB02F307EE903AF8EEE77A204667EE40
:10CC4000897AFDEEE77A17EE901A0DF06DFF9DEDF3
:10CC5000017A6A480595B8EEC77A68EE887A0C21A1
:10CC600067EE877AFDEEE77ACDED007A11F024F8D1
:10CC70000099604811F000FD5E4811F0ADFC00988D
:10CC800013F016FD41EC100B12F066FA51EC100B8C
:10CC900014F024F80C218146584811F00DF849464B
:10CCA000544811F0E9FC534811F096FC0F21544808
:10CCB00011F002F818EE900A13F00CFD41EC100B85
:10CCC00002214C4811F0E0FC4A4811F085FC0B2190
:10CCD0004C4810F0F1FF18EE100A13F0FBFC41EC89
:10CCE000100B0221434811F0CFFC424811F074FCB4
:10CCF0000A21454810F0E0FF01993E4811F0BCFCC4
:10CD00003C4811F069FC204649460DF04BFF2E9B34
:10CD10002E9542AA02EB830242A90B3301EB830357
:10CD200042F88C4CB7EE000A43F8B45C14A8012119
:10CD3000FDF7CEFD169B354CB3B1F4F7BBFF0028D1
:10CD400006DB3868F4F7A6FFC0B25328307038D03D
:10CD500023680393039A23680293029B9B1A042B74
:10CD6000F9D9169B002BE8D1294C2A48142110F040
:10CD7000A3FF21681F4811F07FFC1E4811F02CFC16
:10CD80002268059B234813441421236010F094FF6C
:10CD90002168184811F070FC164811F01DFC312173
:10CDA0001D4810F089FF134811F016FC14A8CDF8A7
:10CDB0005080FBF717FE284643B0BDEC048BBDE85E
:10CDC000F08314A8FBF7B6FD00210320F3F766FEFD
:10CDD00000210846F3F762FE00210120F3F75EFE12
:10CDE0000125B5E724650200F813FF1F0AD7233C8D
:10CDF0001007FF1FE407FF1FE816FF1F586502001A
:10CE0000686502007865020084650200841BFF1FCC
:10CE10004017FF1F90650200A8650200044B020046
:10CE20002DE9F04FDFF82483D8F81430012B14BF1C
:10CE30000820042083B0F4F7D7F8D8F81030002B7E
:10CE400040F37881BE4CBF4EBF4DA146B24601278C
:10CE5000D8F81430002B00F07B81012B40F0648166
:10CE6000D5ED007A20680093B8EEE70AF0EE080AE4
:10CE7000FFF79CFE8346F4F753FF002840F05A81E9
:10CE8000009BBBF1000F40F05581D6ED007AD9F838
:10CE9000000000931946B8EEE70AF0EE000A40429F
:10CEA000FFF71EFC8346F4F73BFF009B002840F091
:10CEB0004181BBF1000F40F03D810193A24BD9F8B5
:10CEC00000001B68009307EE903AF7EE000AB8EEF8
:10CED000E70A4042FFF76AFE8346F4F721FF019B11
:10CEE000002840F02781BBF1000F40F02381DAEDEC
:10CEF000007AD9F800001946B8EEE70AF7EE000A02
:10CF0000FFF7EEFB8346F4F70BFF002840F0128199
:10CF1000BBF1000F40F00E812068D5ED007A404251
:10CF2000B8EEE70AF7EE000AFFF740FE8346F4F793
:10CF3000F7FE002840F0FE80BBF1000F40F0FA80C1
:10CF40002068D6ED007A4042B8EEE70A0121F0EE03
:10CF5000000AFFF7C5FB8346F4F7E2FE002840F025
:10CF6000E980BBF1000F40F0E580D5ED007A206844
:10CF7000B8EEE70AF0EE080AFFF718FE8346F4F76A
:10CF8000CFFE002840F0D680BBF1000F40F0D280E9
:10CF9000D6ED007A2068B8EEE70A0121F1EE000A2A
:10CFA000FFF79EFB8346F4F7BBFE002840F0C280EB
:10CFB000BBF1000F40F0BE802068D6ED007A404201
:10CFC000B8EEE70A0121F2EE000AFFF789FB83467B
:10CFD000F4F7A6FE002840F0AD80BBF1000F40F052
:10CFE000A9802068D5ED007A4042B8EEE70AF0EE5D
:10CFF000080AFFF7DBFD8346F4F792FE002840F0B5
:10D000009980BBF1000F40F09580D6ED007A206842
:10D01000B8EEE70A0121F0EE000AFFF761FB834654
:10D02000F4F77EFE002840F08580BBF1000F40F051
:10D030008180D5ED007A2068B8EEE70AF7EE000AA5
:10D04000FFF7B4FD8346F4F76BFE002872D1BBF105
:10D05000000F6FD12068D6ED007A4042B8EEE70AA3
:10D060000121F7EE000AFFF73BFB8346F4F758FE79
:10D0700000285FD1BBF1000F5CD1D5ED007A2068AC
:10D08000B8EEE70AF7EE000AFFF790FD8346F4F7E3
:10D0900047FE00284ED1BBF1000F4BD1D6ED007AF0
:10D0A0002068B8EEE70A0121F0EE000AFFF718FB4E
:10D0B0008346F4F735FE00283CD1BBF1000F39D18F
:10D0C0002068D5ED007A4042B8EEE70AF0EE080A93
:10D0D000FFF76CFD8346F4F723FE58BBBBF1000F4E
:10D0E00028D1D6ED007A2068B8EEE70A0121F1EEEA
:10D0F000000AFFF7F5FA8346F4F712FED0B9BBF148
:10D10000000F17D12068D6ED007A4042B8EEE70A4A
:10D110000121F2EE000AFFF7E3FA8346F4F700FE7E
:10D1200040B9BBF1000F05D1D8F810300137BB4230
:10D13000BFF68EAE03B0BDE8F04FF4F7C3B800BF42
:10D140000807FF1FCC12FF1F6014FF1FF813FF1FFB
:10D15000D6ED007A2068B8EEE70A0121F0EE080A61
:10D16000FFF7BEFA8346F4F7DBFD0028E2D1BBF1FE
:10D17000000FDFD1D9F80000D5ED007A4042B8EEBB
:10D18000E70AF0EE000AFFF711FD8346F4F7C8FD49
:10D190000028CFD1BBF1000FCCD1D9F80000DAEDD7
:10D1A000007A4042B8EEE70A0121F7EE000AFFF7E5
:10D1B00097FA8346F4F7B4FD0028BBD1BBF1000F0A
:10D1C000B8D1934BD9F800001B68009307EE903A52
:10D1D000F7EE000AB8EEE70AFFF7E8FC8346F4F73B
:10D1E0009FFD0028A6D1BBF1000FA3D1D9F8000004
:10D1F000DAED007A4042B8EEE70A0121F7EE000AC4
:10D20000FFF76EFA8346F4F78BFD002892D1BBF14D
:10D21000000F8FD12068D5ED007A4042B8EEE70AC2
:10D22000F0EE000AFFF7C2FC8346F4F779FD002810
:10D2300080D1BBF1000F7FF47DAFD6ED007A20687E
:10D24000B8EEE70A0121F0EE080AFFF749FA834633
:10D25000F4F766FD00287FF46DAFBBF1000F7FF49B
:10D2600069AFD5ED007A2068B8EEE70AF1EE000A62
:10D27000FFF79CFC8346F4F753FD00287FF45AAF78
:10D28000BBF1000F7FF456AF2068D5ED007A404225
:10D29000B8EEE70AF2EE000AFFF788FC8346F4F7DF
:10D2A0003FFD00287FF446AFBBF1000F7FF442AF93
:10D2B0002068D6ED007A4042B8EEE70A0121F0EE90
:10D2C000080AFFF70DFA8346F4F72AFD00287FF4D9
:10D2D00031AFBBF1000F7FF42DAFD5ED007A2068A0
:10D2E000B8EEE70AF0EE000AFFF760FC8346F4F7B9
:10D2F00017FD00287FF41EAFBBF1000F7FF41AAFBB
:10D30000D6ED007A2068B8EEE70A0121F7EE000AB0
:10D31000FFF7E6F98346F4F703FD00287FF40AAF30
:10D32000BBF1000F7FF406AF2068D5ED007A4042D4
:10D33000B8EEE70AF7EE000AFFF738FC8346F4F789
:10D34000EFFC00287FF4F6AEBBF1000F7FF4F2AEE5
:10D35000D6ED007A2068B8EEE70A0121F7EE000A60
:10D36000FFF7BEF98346F4F7DBFC00287FF4E2AE5A
:10D37000BBF1000F7FF4DEAED5ED007A2068B8EE89
:10D38000E70AF0EE000AFFF711FC8346F4F7C8FC49
:10D3900000287FF4CFAEBBF1000F7FF4CBAE206846
:10D3A000D6ED007A4042B8EEE70A0121F0EE080A15
:10D3B000FFF796F98346F4F7B3FC00287FF4BAAE82
:10D3C000BBF1000F7FF4B6AED5ED007A2068B8EE61
:10D3D000E70AF1EE000AFFF7E9FB8346F4F7A0FC49
:10D3E00000287FF4A7AEBBF1000F7FF4A3AE206846
:10D3F000D5ED007A4042B8EEE70AF2EE000AFFF7F8
:10D40000D5FB8346F4F78CFC00283FF48AAE91E606
:10D410006014FF1F2DE9F04FDA4F7B69012B14BF19
:10D420000D20042083B0F3F7DFFD3B69002B40F3B0
:10D430008582D54CD54ED64DA046B2464FF0010957
:10D440007B69002B00F07F82012B40F07182206805
:10D45000D5ED007A01934042B8EEE70A1946F7EE9F
:10D46000000AFFF73DF98346F4F75AFC002840F024
:10D470006582019BBBF1000F40F06082D6ED007A1F
:10D48000D8F800000193B8EEE70AF0EE080AFFF7BB
:10D490008DFB8346F4F744FC019B002840F04E824C
:10D4A000BBF1000F40F04A82B94AD8F80000126878
:10D4B000019207EE902A19464042B8EEE70AF0EED4
:10D4C000000AFFF70DF98346F4F72AFC002840F024
:10D4D0003582BBF1000F40F03182D8F80000DAED60
:10D4E000007A4042B8EEE70AF7EE000AFFF75EFB6B
:10D4F0008346F4F715FC002840F02082BBF1000FB2
:10D5000040F01C82D5ED007A2068B8EEE70A0121D0
:10D51000F7EE000AFFF7E4F88346F4F701FC002871
:10D5200040F00C82BBF1000F40F008822068D6ED7D
:10D53000007A4042B8EEE70AF7EE000AFFF736FB42
:10D540008346F4F7EDFB002840F0F881BBF1000FB3
:10D5500040F0F4812068D5ED007A4042B8EEE70A49
:10D560000121F0EE080AFFF7BBF88346F4F7D8FB79
:10D57000002840F0E381BBF1000F40F0DF81D6EDE1
:10D58000007A2068B8EEE70AF7EE000AFFF70EFB14
:10D590008346F4F7C5FB002840F0D081BBF1000FB3
:10D5A00040F0CC81D5ED007A2068B8EEE70A012181
:10D5B000F7EE000AFFF794F88346F4F7B1FB002872
:10D5C00040F0BC81BBF1000F40F0B881D6ED007A8D
:10D5D0002068B8EEE70AF7EE000AFFF7E7FA83469D
:10D5E000F4F79EFB002840F0A981BBF1000F40F04A
:10D5F000A5812068D5ED007A4042B8EEE70A012106
:10D60000F0EE000AFFF76CF88346F4F789FB002878
:10D6100040F09481BBF1000F40F090812068D6ED7E
:10D62000007A4042B8EEE70AF0EE080AFFF7BEFAC9
:10D630008346F4F775FB002840F08081BBF1000FB2
:10D6400040F07C81D5ED007A2068B8EEE70A012130
:10D65000F1EE080AFFF744F88346F4F761FB00286F
:10D6600040F06C81BBF1000F40F06881D6ED007A8C
:10D670002068B8EEE70AF1EE000AFFF797FA834652
:10D68000F4F74EFB002840F05981BBF1000F40F049
:10D6900055812068D5ED007A4042B8EEE70A0121B5
:10D6A000F1EE0C0AFFF71CF88346F4F739FB00286B
:10D6B00040F04481BBF1000F40F040812068D6ED7E
:10D6C000007A4042B8EEE70AF0EE080AFFF76EFA79
:10D6D0008346F4F725FB002840F03081BBF1000FB2
:10D6E00040F02C812068D5ED007A4042B8EEE70A80
:10D6F0000121F0EE000AFEF7F3FF8346F4F710FB7A
:10D70000002840F01B81BBF1000F40F01781D6EDDF
:10D71000007A2068B8EEE70AF7EE000AFFF746FA4B
:10D720008346F4F7FDFA002840F00881BBF1000FB2
:10D7300040F00481D5ED007A2068B8EEE70A0121B7
:10D74000F7EE000AFEF7CCFF8346F4F7E9FA00286B
:10D7500040F0F480BBF1000F40F0F080D6ED007A8D
:10D760002068B8EEE70AF7EE000AFFF71FFA8346D3
:10D77000F4F7D6FA002840F0E180BBF1000F40F04A
:10D78000DD8007E0F813FF1F0807FF1F6014FF1F6D
:10D79000CC12FF1F2068D5ED007A4042B8EEE70AB0
:10D7A0000121F0EE080AFEF79BFF8346F4F7B8FA72
:10D7B000002840F0C380BBF1000F40F0BF8020681C
:10D7C000D6ED007A4042B8EEE70AF7EE000AFFF71E
:10D7D000EDF98346F4F7A4FA002840F0AF80BBF1DE
:10D7E000000F40F0AB80D5ED007A2068B8EEE70A74
:10D7F0000121F7EE000AFEF773FF8346F4F790FA73
:10D80000002840F09B80BBF1000F40F0978020681B
:10D81000D6ED007A4042B8EEE70AF7EE000AFFF7CD
:10D82000C5F98346F4F77CFA002840F08780BBF105
:10D83000000F40F083802068D5ED007A4042B8EEBA
:10D84000E70A0121F0EE000AFEF74AFF8346F4F7EB
:10D8500067FA002872D1BBF1000F6FD1D6ED007AC4
:10D860002068B8EEE70AF0EE080AFFF79FF9834652
:10D87000F4F756FA002861D1BBF1000F5ED1D5ED67
:10D88000007A2068B8EEE70A0121F1EE040AFEF7FB
:10D8900027FF8346F4F744FA00284FD1BBF1000F6D
:10D8A0004CD12068D5ED007A4042B8EEE70A01215C
:10D8B000F1EE080AFEF714FF8346F4F731FA002868
:10D8C0003CD1BBF1000F39D12068D6ED007A40423F
:10D8D000B8EEE70AF1EE000AFFF768F98346F4F7BD
:10D8E0001FFA58BBBBF1000F28D1D5ED007A206894
:10D8F000B8EEE70A0121F1EE0C0AFEF7F1FE8346CD
:10D90000F4F70EFAD0B9BBF1000F17D12068D5EDAE
:10D91000007A4042B8EEE70A0121F1EE0C0AFEF768
:10D92000DFFE8346F4F7FCF940B9BBF1000F05D1E7
:10D930003B6909F101094B45BFF682AD03B0BDE873
:10D94000F04FF3F7BFBC2068D6ED007A4042B8EE46
:10D95000E70AF7EE000AFFF729F98346F4F7E0F942
:10D960000028EBD1BBF1000FE8D1D5ED007AD8F853
:10D970000000B8EEE70A0121F0EE080AFEF7B0FE5B
:10D980008346F4F7CDF90028D8D1BBF1000FD5D1EB
:10D99000D8F80000DAED007A4042B8EEE70AF0EE7F
:10D9A000000AFFF703F98346F4F7BAF90028C5D156
:10D9B000BBF1000FC2D1DC4BD8F800001B6801930B
:10D9C00007EE903A4042B8EEE70A0121F7EE000A6E
:10D9D000FEF786FE8346F4F7A3F90028AED1BBF12B
:10D9E000000FABD1DAED007AD8F80000B8EEE70A04
:10D9F000F7EE000AFFF7DAF88346F4F791F900280A
:10DA00009CD1BBF1000F99D12068D5ED007A40423E
:10DA1000B8EEE70A0121F7EE000AFEF761FE834641
:10DA2000F4F77EF9002889D1BBF1000F86D1206878
:10DA3000D6ED007A4042B8EEE70AF0EE080AFFF7AA
:10DA4000B5F88346F4F76CF900287FF477AFBBF1A3
:10DA5000000F7FF473AFD5ED007A2068B8EEE70AC7
:10DA60000121F7EE000AFEF73BFE8346F4F758F972
:10DA700000287FF463AFBBF1000F7FF45FAFD6EDFA
:10DA8000007A2068B8EEE70AF7EE000AFFF78EF892
:10DA90008346F4F745F900287FF450AFBBF1000F3F
:10DAA0007FF44CAFD5ED007A2068B8EEE70A01218B
:10DAB000F7EE000AFEF714FE8346F4F731F900286A
:10DAC0007FF43CAFBBF1000F7FF438AF2068D6ED98
:10DAD000007A4042B8EEE70AF0EE000AFFF766F877
:10DAE0008346F4F71DF900287FF428AFBBF1000F3F
:10DAF0007FF424AF2068D5ED007A4042B8EEE70A03
:10DB00000121F0EE080AFEF7EBFD8346F4F708F971
:10DB100000287FF413AFBBF1000F7FF40FAFD6EDF9
:10DB2000007A2068B8EEE70AF1EE080AFFF73EF83F
:10DB30008346F4F7F5F800287FF400AFBBF1000F3F
:10DB40007FF4FCAED5ED007A2068B8EEE70A01213B
:10DB5000F1EE000AFEF7C4FD8346F4F7E1F8002871
:10DB60007FF4ECAEBBF1000F7FF4E8AE2068D6ED99
:10DB7000007A4042B8EEE70AF1EE0C0AFFF716F819
:10DB80008346F4F7CDF800287FF4D8AEBBF1000F40
:10DB90007FF4D4AE2068D5ED007A4042B8EEE70AB3
:10DBA0000121F0EE080AFEF79BFD8346F4F7B8F872
:10DBB00000287FF4C3AEBBF1000F7FF4BFAE206836
:10DBC000D6ED007A4042B8EEE70AF0EE000AFEF722
:10DBD000EDFF8346F4F7A4F800287FF4AFAEBBF165
:10DBE000000F7FF4ABAED5ED007A2068B8EEE70AFF
:10DBF0000121F7EE000AFEF773FD8346F4F790F873
:10DC000000287FF49BAEBBF1000F7FF497AED6EDFA
:10DC1000007A2068B8EEE70AF7EE000AFEF7C6FFC2
:10DC20008346F4F77DF800287FF488AEBBF1000F3F
:10DC30007FF484AED5ED007A2068B8EEE70A0121C2
:10DC4000F7EE000AFEF74CFD8346F4F769F800286A
:10DC50007FF474AEBBF1000F7FF470AE2068D6ED98
:10DC6000007A4042B8EEE70AF0EE080AFEF79EFF9F
:10DC70008346F4F755F800287FF460AEBBF1000F3F
:10DC80007FF45CAE2068D5ED007A4042B8EEE70A3A
:10DC90000121F7EE000AFEF723FD8346F4F740F872
:10DCA00000287FF44BAEBBF1000F7FF447AED6EDFA
:10DCB000007A2068B8EEE70AF7EE000AFEF776FF72
:10DCC0008346F4F72DF800287FF438AEBBF1000F3F
:10DCD0007FF434AE2068D5ED007A4042B8EEE70A12
:10DCE0000121F7EE000AFEF7FBFC8346F4F718F873
:10DCF00000287FF423AEBBF1000F7FF41FAE206835
:10DD0000D6ED007A4042B8EEE70AF0EE000AFEF7E0
:10DD10004DFF8346F4F704F800287FF40FAEBBF103
:10DD2000000F7FF40BAE01E0CC12FF1FD5ED007A9F
:10DD30002068B8EEE70A0121F0EE080AFEF7D0FCF1
:10DD40008346F3F7EDFF00287FF4F8ADBBF1000F39
:10DD50007FF4F4ADD6ED007A2068B8EEE70AF1EE74
:10DD6000040AFEF723FF8346F3F7DAFF00287FF467
:10DD7000E5ADBBF1000F7FF4E1AD2068D6ED007A90
:10DD80004042B8EEE70AF1EE080AFEF70FFF8346BD
:10DD9000F3F7C6FF00287FF4D1ADBBF1000F7FF48D
:10DDA000CDAD2068D5ED007A4042B8EEE70A0121FA
:10DDB000F1EE000AFEF794FC8346F3F7B1FF00286A
:10DDC0007FF4BCADBBF1000F7FF4B8ADD6ED007AA7
:10DDD0002068B8EEE70AF1EE0C0AFEF7E7FE83468C
:10DDE000F3F79EFF00287FF4A9ADBBF1000F7FF48D
:10DDF000A5AD2068D6ED007A4042B8EEE70AF1EE14
:10DE00000C0AFEF7D3FE8346F3F78AFF00283FF49F
:10DE10008CAD93E52DE9F04FAA4F7B69012B14BF20
:10DE20000420032083B0F3F7DFF83B69002B40F3B5
:10DE3000AC80A54CDFF89892DFF890822646CA465F
:10DE400001257B69002B00F0A580012B40F0988014
:10DE5000D8ED007A20680093B8EEE70AF0EE080AE1
:10DE6000FEF7A4FE8346F3F75BFF002840F08D80A9
:10DE7000009BBBF1000F40F08880D9ED007A30683C
:10DE800000931946B8EEE70AF0EE080A4042FEF7A2
:10DE900027FC8346F3F744FF009B002875D1BBF1B4
:10DEA000000F72D10193894B30681B68009307EE15
:10DEB000903AF0EE000AB8EEE70A4042FEF776FE2E
:10DEC0008346F3F72DFF019B00285ED1BBF1000FC5
:10DED0005BD1DAED007A30681946B8EEE70AF7EE62
:10DEE000000AFEF7FDFB8346F3F71AFF00284CD12A
:10DEF000BBF1000F49D1D8ED007A2068B8EEE70AEF
:10DF0000F7EE000AFEF752FE8346F3F709FF0028FA
:10DF10003BD1BBF1000F38D1D9ED007A2068B8EEC3
:10DF2000E70A0121F7EE000AFEF7DAFB8346F3F772
:10DF3000F7FE50BBBBF1000F27D12068D8ED007A67
:10DF40004042B8EEE70AF0EE000AFEF72FFE8346E5
:10DF5000F3F7E6FEC8B9BBF1000F16D12068D9ED82
:10DF6000007A4042B8EEE70A0121F0EE080AFEF717
:10DF7000B7FB8346F3F7D4FE38B9BBF1000F04D1E9
:10DF80003B690135AB42BFF65CAF03B0BDE8F04F73
:10DF9000F3F798B9D9ED007A2068B8EEE70A0121C5
:10DFA000F0EE080AFEF79CFB8346F3F7B9FE002863
:10DFB000EBD1BBF1000FE8D13068D8ED007A4042D8
:10DFC000B8EEE70AF0EE080AFEF7F0FD8346F3F735
:10DFD000A7FE0028D9D1BBF1000FD6D13068DAED09
:10DFE000007A4042B8EEE70A0121F0EE000AFEF79F
:10DFF00077FB8346F3F794FE0028C6D1BBF1000FF0
:10E00000C3D1324B30681B68009307EE903AF7EEAD
:10E01000000AB8EEE70AFEF7C9FD8346F3F780FE73
:10E020000028B2D1BBF1000FAFD1DAED007A306831
:10E03000B8EEE70A0121F7EE000AFEF751FB83462E
:10E04000F3F76EFE0028A0D1BBF1000F9DD1D8EDF3
:10E05000007A2068B8EEE70AF7EE000AFEF7A6FDA0
:10E060008346F3F75DFE00288FD1BBF1000F8CD102
:10E070002068D9ED007A4042B8EEE70A0121F0EEBF
:10E08000000AFEF72DFB8346F3F74AFE00287FF4D3
:10E090007CAFBBF1000F7FF478AF2068D8ED007A39
:10E0A0004042B8EEE70AF0EE080AFEF77FFD83462D
:10E0B000F3F736FE00283FF460AF03B0BDE8F04F41
:10E0C000F3F700B9F813FF1F0807FF1F6014FF1FC5
:10E0D000CC12FF1F2DE9F04FDFF8D082D8F81430B2
:10E0E000012B14BF0820032083B0F2F77DFFD8F87E
:10E0F0001030002B40F34F81A94CAA4EAA4DA146E7
:10E10000B2460127D8F81430002B00F05181012BC2
:10E1100040F03B81D5ED007A20680093B8EEE70A25
:10E12000F0EE080AFEF742FD8346F3F7F9FD0028FA
:10E1300040F03181009BBBF1000F40F02C81D6ED07
:10E14000007AD9F8000000931946B8EEE70AF0EE1D
:10E15000080A4042FEF7C4FA8346F3F7E1FD009B4C
:10E16000002840F01881BBF1000F40F014810193AA
:10E170008D4BD9F800001B68009307EE903AF0EE43
:10E18000000AB8EEE70A4042FEF710FD8346F3F7B7
:10E19000C7FD019B002840F0FE80BBF1000F40F05E
:10E1A000FA80DAED007AD9F800001946B8EEE70AED
:10E1B000F7EE000AFEF794FA8346F3F7B1FD002864
:10E1C00040F0E980BBF1000F40F0E580D5ED007A2A
:10E1D0002068B8EEE70AF7EE000AFEF7E7FC834690
:10E1E000F3F79EFD002840F0D680BBF1000F40F011
:10E1F000D280D6ED007A2068B8EEE70A0121F7EE6A
:10E20000000AFEF76DFA8346F3F78AFD002840F016
:10E21000C280BBF1000F40F0BE802068D5ED007ACF
:10E220004042B8EEE70AF0EE000AFEF7BFFC834674
:10E23000F3F776FD002840F0AE80BBF1000F40F010
:10E24000AA802068D6ED007A4042B8EEE70A0121A4
:10E25000F1EE040AFEF744FA8346F3F761FD002865
:10E2600040F09980BBF1000F40F09580D5ED007A29
:10E270002068B8EEE70AF0EE000AFEF797FC834646
:10E28000F3F74EFD002840F08680BBF1000F40F010
:10E290008280D6ED007A2068B8EEE70A0121F7EE19
:10E2A000000AFEF71DFA8346F3F73AFD002872D103
:10E2B000BBF1000F6FD12068D5ED007A4042B8EE77
:10E2C000E70AF7EE000AFEF771FC8346F3F728FD34
:10E2D000002860D1BBF1000F5DD1D6ED007A206837
:10E2E000B8EEE70A0121F7EE000AFEF7F9F98346D6
:10E2F000F3F716FD00284ED1BBF1000F4BD1D5ED41
:10E30000007A2068B8EEE70AF0EE000AFEF74EFC4D
:10E310008346F3F705FD00283DD1BBF1000F3AD14C
:10E320002068D6ED007A4042B8EEE70A0121F0EE0F
:10E33000080AFEF7D5F98346F3F7F2FC58BBBBF1A8
:10E34000000F28D12068D5ED007A4042B8EEE70AE8
:10E35000F0EE080AFEF72AFC8346F3F7E1FCD0B999
:10E36000BBF1000F17D12068D6ED007A4042B8EE1D
:10E37000E70A0121F7EE000AFEF7B2F98346F3F748
:10E38000CFFC40B9BBF1000F05D1D8F810300137F0
:10E39000BB42BFF6B7AE03B0BDE8F04FF2F792BF95
:10E3A0000807FF1FCC12FF1F6014FF1FF813FF1F89
:10E3B000D6ED007A2068B8EEE70A0121F0EE080AEF
:10E3C000FEF78EF98346F3F7ABFC0028E3D1BBF1EF
:10E3D000000FE0D1D9F80000D5ED007A4042B8EE48
:10E3E000E70AF0EE080AFEF7E1FB8346F3F798FC34
:10E3F0000028D0D1BBF1000FCDD1D9F80000DAED63
:10E40000007A4042B8EEE70A0121F0EE000AFEF77A
:10E4100067F98346F3F784FC0028BCD1BBF1000FF9
:10E42000B9D1814BD9F800001B68009307EE903AF0
:10E43000F7EE000AB8EEE70AFEF7B8FB8346F3F7FB
:10E440006FFC0028A7D1BBF1000FA4D1DAED007A50
:10E45000D9F80000B8EEE70A0121F7EE000AFEF74E
:10E460003FF98346F3F75CFC002894D1BBF1000F21
:10E4700091D1D5ED007A2068B8EEE70AF7EE000AF0
:10E48000FEF794FB8346F3F74BFC002883D1BBF1E6
:10E49000000F80D12068D6ED007A4042B8EEE70A3E
:10E4A0000121F0EE000AFEF71BF98346F3F738FC72
:10E4B00000287FF470AFBBF1000F7FF46CAF2068D1
:10E4C000D5ED007A4042B8EEE70AF1EE040AFEF715
:10E4D0006DFB8346F3F724FC00287FF45CAFBBF1AF
:10E4E000000F7FF458AFD6ED007A2068B8EEE70A47
:10E4F0000121F0EE000AFEF7F3F88346F3F710FC73
:10E5000000287FF448AFBBF1000F7FF444AFD5ED96
:10E51000007A2068B8EEE70AF7EE000AFEF746FB3D
:10E520008346F3F7FDFB00287FF435AFBBF1000F06
:10E530007FF431AF2068D6ED007A4042B8EEE70AAA
:10E540000121F7EE000AFEF7CBF88346F3F7E8FB6C
:10E5500000287FF420AFBBF1000F7FF41CAFD5ED96
:10E56000007A2068B8EEE70AF7EE000AFEF71EFB15
:10E570008346F3F7D5FB00287FF40DAFBBF1000F06
:10E580007FF409AFD6ED007A2068B8EEE70A0121E2
:10E59000F0EE000AFEF7A4F88346F3F7C1FB00286B
:10E5A0007FF4F9AEBBF1000F7FF4F5AE2068D5ED36
:10E5B000007A4042B8EEE70AF0EE080AFEF7F6FAF3
:10E5C0008346F3F7ADFB00287FF4E5AEBBF1000F07
:10E5D0007FF4E1AE2068D6ED007A4042B8EEE70A5B
:10E5E0000121F0EE080AFEF77BF88346F3F798FB6B
:10E5F00000287FF4D0AEBBF1000F7FF4CCAE2068D2
:10E60000D5ED007A4042B8EEE70AF7EE000AFEF7D1
:10E61000CDFA8346F3F784FB00283FF4B3AE03B092
:10E62000BDE8F04FF2F74EBE6014FF1F2DE9F04F2A
:10E63000974EDFF874927369012B14BF03200220F8
:10E6400083B0F2F7D1FC142192480FF035FBD9F8D2
:10E650000010914810F010F88F480FF0BDFF33699B
:10E66000002B40F39C808D4FDFF840823D46012413
:10E6700012218B480FF020FB214687480FF0FCFF4A
:10E6800085480FF0A9FFD6F814A0BAF1000F00F0EA
:10E690008B80BAF1010F7DD1142182480FF00CFB61
:10E6A000D9F800107C480FF0E7FF7B480FF094FF8B
:10E6B000D8ED007A3868B8EEE70AF0EE000AFEF707
:10E6C00075FA8346F3F72CFB002868D1BBF1000FE5
:10E6D00065D1754B28681B68019307EE903A40425C
:10E6E000B8EEE70A5146F0EE000AFDF7F9FF83465F
:10E6F000F3F716FB002852D1BBF1000F4FD16B4B43
:10E7000028681B68019307EE903A4042B8EEE70A8A
:10E71000F7EE000AFEF74AFA8346F3F701FB0028FA
:10E720003DD1BBF1000F3AD15F4B286893ED000A51
:10E730005146B8EEC00A4042F7EE000AFDF7D0FF9E
:10E740008346F3F7EDFA50BBBBF1000F27D13868D1
:10E75000D8ED007A4042B8EEE70AF7EE000AFEF77D
:10E7600025FA8346F3F7DCFAC8B9BBF1000F16D1DE
:10E770003868D9ED007A4042B8EEE70A0121F0EEA0
:10E78000000AFDF7ADFF8346F3F7CAFA38B9BBF1CB
:10E79000000F04D133690134A342BFF669AF03B05F
:10E7A000BDE8F04FF2F78EBDD9ED007A3868DFF89A
:10E7B000F8A0B8EEE70A0121F0EE000AFDF790FF9D
:10E7C0008346F3F7ADFA0028E9D1BBF1000FE6D19B
:10E7D0002868D8ED007A4042B8EEE70AF0EE000A69
:10E7E000FEF7E4F98346F3F79BFA0028D7D1BBF193
:10E7F000000FD4D12868DAED007A4042B8EEE70A7B
:10E800000121F7EE000AFDF76BFF8346F3F788FA64
:10E810000028C4D1BBF1000FC1D1244B28681B686C
:10E82000019307EE903AF7EE000AB8EEE70AFEF71A
:10E83000BDF98346F3F774FA0028B0D1BBF1000F9D
:10E84000ADD19AED000A2868B8EEC00A4042012115
:10E85000F7EE000AFDF744FF8346F3F761FA00285C
:10E860009DD1BBF1000F9AD13868D8ED007A4042B3
:10E87000B8EEE70AF0EE000AFEF798F98346F3F7E0
:10E880004FFA002883D003B0BDE8F04FF2F71ABD6D
:10E89000F813FF1FDC650200E407FF1F0807FF1FD6
:10E8A000F465020008660200CC12FF1F6014FF1F0F
:10E8B0002DE9F04FDFF88092D9F81430012B14BF06
:10E8C0000620022083B0F2F78FFBD9F81030002B1E
:10E8D00040F32781954C964E964DA046B2460127AF
:10E8E000D9F81430002B00F02981012B40F013815E
:10E8F000D6ED007A20680193B8EEE70A1946F7EEE4
:10E90000000AFDF7EDFE8346F3F70AFA002840F00F
:10E910000881019BBBF1000F40F00381DAED007A22
:10E92000D8F8000001931946B8EEE70AF7EE000A9E
:10E930004042FDF7D5FE8346F3F7F2F9019B00282C
:10E9400040F0EF80BBF1000F40F0EB80D5ED007A96
:10E95000D8F800000193B8EEE70AF0EE000A404252
:10E96000FEF724F98346F3F7DBF9019B002840F01A
:10E97000D880BBF1000F40F0D480D8F80000DAED69
:10E98000007A19464042B8EEE70AF0EE000AFDF7B9
:10E99000A7FE8346F3F7C4F9002840F0C280BBF11C
:10E9A000000F40F0BE802068D5ED007A4042B8EEFE
:10E9B000E70AF0EE000AFEF7F9F88346F3F7B0F93C
:10E9C000002840F0AE80BBF1000F40F0AA80D6EDE9
:10E9D000007A2068B8EEE70A0121F7EE000AFDF799
:10E9E0007FFE8346F3F79CF9002840F09A80BBF144
:10E9F000000F40F096802068D5ED007A4042B8EED6
:10EA0000E70AF7EE000AFEF7D1F88346F3F788F934
:10EA1000002840F08680BBF1000F40F08280206823
:10EA2000D6ED007A4042B8EEE70A0121F0EE080A7E
:10EA3000FDF756FE8346F3F773F9002871D1BBF159
:10EA4000000F6ED1D5ED007A2068B8EEE70AF7EE38
:10EA5000000AFEF7ABF88346F3F762F9002860D1AD
:10EA6000BBF1000F5DD1D6ED007A2068B8EEE70A61
:10EA70000121F7EE000AFDF733FE8346F3F750F964
:10EA800000284ED1BBF1000F4BD1D5ED007A2068A4
:10EA9000B8EEE70AF7EE000AFEF788F88346F3F7C8
:10EAA0003FF900283DD1BBF1000F3AD12068D6EDE7
:10EAB000007A4042B8EEE70A0121F0EE000AFDF7C5
:10EAC0000FFE8346F3F72CF958BBBBF1000F28D19A
:10EAD0002068D5ED007A4042B8EEE70AF0EE000A71
:10EAE000FEF764F88346F3F71BF9D0B9BBF1000FCA
:10EAF00017D12068D6ED007A4042B8EEE70A01212E
:10EB0000F7EE000AFDF7ECFD8346F3F709F940B98B
:10EB1000BBF1000F05D1D9F810300137BB42BFF669
:10EB2000DFAE03B0BDE8F04FF2F7CCBB0807FF1F24
:10EB3000CC12FF1F6014FF1FF813FF1FD5ED007AE2
:10EB40002068B8EEE70AF7EE000AFEF72FF88346D2
:10EB5000F3F7E6F80028E4D1BBF1000FE1D1834BD5
:10EB6000D8F800001B68019307EE903A4042B8EED7
:10EB7000E70AF7EE000AFEF719F88346F3F7D0F834
:10EB80000028CED1BBF1000FCBD1D6ED007AD8F85A
:10EB90000000B8EEE70A0121F0EE000AFDF7A0FD43
:10EBA0008346F3F7BDF80028BBD1BBF1000FB8D105
:10EBB0006E4BD8F800001B68019307EE903A404274
:10EBC000B8EEE70AF0EE000AFDF7F0FF8346F3F730
:10EBD000A7F80028A5D1BBF1000FA2D1D8F80000FA
:10EBE000DAED007A4042B8EEE70A0121F7EE000ABA
:10EBF000FDF776FD8346F3F793F8002891D1BBF13A
:10EC0000000F8ED1D5ED007A2068B8EEE70AF7EE56
:10EC1000000AFDF7CBFF8346F3F782F8002880D186
:10EC2000BBF1000F7FF47DAF2068D6ED007A404243
:10EC3000B8EEE70A0121F7EE000AFDF751FD834621
:10EC4000F3F76EF800287FF46CAFBBF1000F7FF490
:10EC500068AF2068D5ED007A4042B8EEE70AF0EEE2
:10EC6000080AFDF7A3FF8346F3F75AF800287FF45C
:10EC700058AFBBF1000F7FF454AFD6ED007A206897
:10EC8000B8EEE70A0121F7EE000AFDF729FD8346F9
:10EC9000F3F746F800287FF444AFBBF1000F7FF490
:10ECA00040AFD5ED007A2068B8EEE70AF7EE000A2B
:10ECB000FDF77CFF8346F3F733F800287FF431AF8C
:10ECC000BBF1000F7FF42DAFD6ED007A2068B8EECF
:10ECD000E70A0121F7EE000AFDF702FD8346F3F78C
:10ECE0001FF800287FF41DAFBBF1000F7FF419AFB0
:10ECF0002068D5ED007A4042B8EEE70AF0EE000A4F
:10ED0000FDF754FF8346F3F70BF800287FF409AFB3
:10ED1000BBF1000F7FF405AF2068D6ED007A4042CA
:10ED2000B8EEE70A0121F0EE000AFDF7D9FC8346B0
:10ED3000F2F7F6FF00287FF4F4AEBBF1000F7FF48A
:10ED4000F0AE2068D5ED007A4042B8EEE70AF7EE63
:10ED5000000AFDF72BFF8346F2F7E2FF00283FF49D
:10ED6000D7AE03B0BDE8F04FF2F7ACBA6014FF1FA6
:10ED70002DE9F047C2B041F288320521804604AD4A
:10ED800014A8BA4FBA4EF9F7E3FD00242846022230
:10ED9000032114962F940BF085FE3B680594013BEC
:10EDA000042B00F25F81DFE813F04D0151015501A2
:10EDB00059010500AF48B04C08210EF07DFF052138
:10EDC000AE480EF079FFA168AD480FF055FCAC4895
:10EDD0000FF002FCA06811F06BFC41EC100B10F07E
:10EDE000BBF951EC100B11F079FF814608FB00FADA
:10EDF0000A21A448A44C0EF05FFF4146A0480FF042
:10EE00003BFC9F480FF0E8FB0C21A0480EF054FF9C
:10EE100000230A2221689A480FF0EEFB98480FF071
:10EE2000DBFB0B219A480EF047FFA06811F052FC63
:10EE300041EC100B022192480FF026FC90480FF095
:10EE4000CBFB0B2193480EF037FF00230A226168A9
:10EE50008B480FF0D1FB8A480FF0BEFB0C218E4887
:10EE60000EF02AFF00230A22D4F8841084480FF001
:10EE7000C3FB83480FF0B0FB132188480EF01CFF42
:10EE800000230A22D4F888107D480FF0B5FB7C4897
:10EE90000FF0A2FB0E2182480EF00EFF4946784883
:10EEA0000FF0EAFB76480FF097FB796828460BF0E5
:10EEB0003BFEF96828460BF02BFE514628460BF026
:10EEC00071FE01210320F1F7E9FD2E9B42A903F118
:10EED0000B0201EB820201EB8303002743F88C5CF9
:10EEE000B7EE000A012114A842F8B47C2E97FBF774
:10EEF000EFFC169B2BB101200CF02AFC169B002B7B
:10EF0000F9D168466749684D0FF032FD6846002127
:10EF1000F2F7B4F968460FF0EBFC684663490FF06E
:10EF200027FD68460021F2F7A9F968460FF0E0FCDA
:10EF300068465F490FF01CFD68460021F2F79EF914
:10EF400068460FF0D5FC684658490FF011FD684639
:10EF50000021F2F793F968460FF0CAFC684655495C
:10EF60000FF006FD68460021F2F788F968460FF0B9
:10EF7000BFFC68464D490FF0FBFC68460021F2F7E4
:10EF80007DF968460FF0B4FC68464B490FF0F0FC81
:10EF900068460021F2F772F968460FF0A9FC68464E
:10EFA00042490FF0E5FC68460021F2F767F9684630
:10EFB0000FF09EFC61682368059A94ED027A3F4C3D
:10EFC000DFED3F6A03FB01F307EE903A06EE102AED
:10EFD000F8EE677AB8EEC66A67EE877A2368394931
:10EFE00086EE277A0A6068461A443749226067EE3F
:10EFF000267AC5ED007A0FF0BBFC00216846F2F7D7
:10F000003DF968460FF074FC2220F2F7A9FA95ED5D
:10F01000000A0020F2F748FA68462C490FF0A8FCD5
:10F0200068460021F2F72AF968460FF061FC0021DA
:10F030000320F1F733FD14A81496F9F7D3FC42B07E
:10F04000BDE8F08708212248224CB6E60821224874
:10F05000224CB2E608212248224CAEE60821224882
:10F06000224CAAE64FF0000AD146C1E66C15FF1FFC
:10F07000044B0200586602008016FF1F2C66020037
:10F08000E407FF1F80750200DC17FF1F64660200A3
:10F0900074660200806602008C6602009C660200B4
:10F0A000B0660200C06602003016FF1F604E02000C
:10F0B000D4660200E8660200FC6602004017FF1FEB
:10F0C0000000B4436815FF1F305F02007450020057
:10F0D00020660200B814FF1F346602003816FF1FB6
:10F0E000406602005016FF1F4C6602006816FF1FA4
:10F0F0002DE9F04FCE4FCF4C3A682DED028BD7B0B3
:10F100000023012A0091236008EE900A00F0888411
:10F11000C0F05E84022A00F04B82DFF86483009323
:10F120001E4601939A469B4641F28832052108AC5F
:10F1300028A8F9F70DFC0025BF4B289302220321D4
:10F140000DF16009204643950BF0ACFC5246594640
:10F1500048460BF0A7FC98ED027AD7ED0F7A7A6853
:10F160007B6A9FEDB66A67EE877A98ED007AF8EED3
:10F17000476A03FB02F307EE103A67EEA67AD8ED72
:10F18000016AB8EEC77AB8EE668A27EE067A67EEAD
:10F19000887AF8EEE88A204627EEA88AFDEEC77A3C
:10F1A00017EE901A0BF0C0FCB9680BF0B1FCFDEE45
:10F1B000C87A17EE901A0BF0F5FC019948460BF04F
:10F1C000B3FC31460BF0A4FC00990BF0EBFC0821DA
:10F1D0009B480EF071FD2B460A22396899480FF0C2
:10F1E0000BFA98480FF0F8F9082197480EF064FDE3
:10F1F0000D2196480EF060FD18EE100A11F06AFA23
:10F2000041EC100B02218F480FF03EFA8D480FF0B1
:10F21000E3F908218C480EF04FFD0C218C480EF0CC
:10F220004BFDF86B11F056FA41EC100B02218548AA
:10F230000FF02AFA83480FF0CFF9082180480EF02A
:10F240003BFD092183480EF037FDB86B11F042FAFF
:10F2500041EC100B02217B480FF016FA79480FF0B1
:10F26000BBF9082176480EF027FD0D2177480EF0F6
:10F2700023FD009973480FF0FFF972480FF0ACF9C5
:10F2800001210320F1F70AFC3968012900F09C8371
:10F29000C0F07B83022903D108460121F1F7FEFB70
:10F2A00037216D486D4E6E4DDFF8D8A10EF004FD8C
:10F2B00064480FF091F9429B56AA02EB830156A8CD
:10F2C00003F10C0200EB8202002341F8889C41F814
:10F2D0008C4CB7EE000A022142F8B43C28A84293B5
:10F2E000FBF7F6FADDF8A8B0DFF89C91BBF1000F50
:10F2F00020D06268199B32602B60F2F7DBFC00289B
:10F3000009DBDAF80000F2F7C5FCC0B2532889F82F
:10F31000000000F07B81534A13680393039913683C
:10F320000293029B5B1A092BF9D9DDF8A8B0BBF157
:10F33000000FDED13F684C496068199A0860012FC0
:10F340002A6000F06582C0F08381022F40F00981BD
:10F35000D8F80010D8F8040098ED027AD6ED006ACB
:10F360009FED426ADFF82491DFF8248101FB00F36E
:10F3700007EE903AF8EE677AF8EEE66A67EE877A7B
:10F38000384686EEA77A07EE902AB8EEE70A67EECF
:10F39000067AC9ED007AF1F78FFC354988ED000A4D
:10F3A00004A80FF0E5FA594604A8F1F767FF04A88E
:10F3B0000FF09EFA2220F2F7D3F899ED000A584692
:10F3C000F2F772F82B4904A80FF0D2FA594604A8B4
:10F3D000F1F754FF04A80FF08BFA274904A80FF0A7
:10F3E000C7FA594604A8F1F749FF04A80FF080FABC
:10F3F0002220F2F7B5F898ED000A5846F2F754F8D3
:10F400001C4904A80FF0B4FA594604A8F1F736FFD6
:10F4100004A80FF06DFA194904A80FF0A9FA59468B
:10F4200004A8F1F72BFF04A80FF062FA32E000BF46
:10F430006C13FF1FB812FF1F044B02000AD7233CB6
:10F4400010670200E407FF1FAC5F02001C670200A8
:10F450002C670200586002003C6702004017FF1F43
:10F460007412FF1F841BFF1F6815FF1F0000B443A9
:10F47000305F020074500200405F020074670200B7
:10F48000DC17FF1F1007FF1FE816FF1F3016FF1FB6
:10F490009015FF1F614904A80FF06AFA594604A8A5
:10F4A000F1F7ECFE04A80FF023FA5D4904A80FF071
:10F4B0005FFA594604A8F1F7E1FE04A80FF018FA24
:10F4C000564904A80FF054FA594604A8F1F7D6FE9D
:10F4D00004A80FF00DFA534904A80FF049FA594651
:10F4E00004A8F1F7CBFE04A80FF002FA4B4904A8D8
:10F4F0000FF03EFA594604A8F1F7C0FE04A80FF039
:10F50000F7F9494904A80FF033FA594604A8F1F76E
:10F51000B5FE04A80FF0ECF9404904A80FF028FA52
:10F52000594604A8F1F7AAFE04A80FF0E1F93F49F3
:10F5300004A80FF01DFA594604A8F1F79FFE04A88D
:10F540000FF0D6F9354904A80FF012FA594604A86D
:10F55000F1F794FE04A80FF0CBF959463846F1F7BD
:10F560009DFA00231946032063601993F1F796FA78
:10F5700008212F480EF0A0FB31682E480FF07CF8D0
:10F580002C480FF029F805212B480EF095FB29682F
:10F5900028480FF071F827480FF01EF8274B2893E2
:10F5A00028A8F9F71FFA57B0BDEC028BBDE8F08F21
:10F5B000F8693A6B9FED227ADFF88C803E6AD8F8C2
:10F5C000341002FB00F207EE902AF8EEE77A67EEBD
:10F5D000877AFDEEE77ACDED017A002900F04882C6
:10F5E000012940F04A8297ED0E0AF1F731FCDDED7A
:10F5F000007AF8EEE77A4FF0170A27EE800A4FF00C
:10F60000100BFDEEC07ACDED007A8DE528A8F9F754
:10F6100065F90C4A012313707DE600BF604E0200BD
:10F62000886702009C670200C4670200B06702009E
:10F63000AC5F0200E407FF1FD85F0200044B02002A
:10F640000AD7233CA016FF1FDC17FF1F0000B4439E
:10F6500098E80A0001FB03F307EE903A98ED027A6E
:10F66000D6ED006AD8F81070D8F80C0098ED055A5D
:10F670005FED0A5ADFF84883C649F8EE677AB8EEBC
:10F68000E66A67EE877A07EE102A00FB07F2F8EECB
:10F69000C76A86EE277AC04F04A807EE902A66EE66
:10F6A000856AF8EE677A27EE257A86EEA76A88EDF6
:10F6B000007A87ED006A0FF05BF9594604A8F1F76C
:10F6C000DDFD04A80FF014F92220F1F749FF98EDB1
:10F6D000000A5846F1F7E8FE04A8B0490FF048F9CF
:10F6E000594604A8F1F7CAFD04A80FF001F904A8CF
:10F6F000AB490FF03DF9594604A8F1F7BFFD04A846
:10F700000FF0F6F82220F1F72BFF97ED000A58468C
:10F71000F1F7CAFE04A8A1490FF02AF9594604A836
:10F72000F1F7ACFD04A80FF0E3F804A89D490FF031
:10F730001FF9594604A8F1F7A1FD04A80FF0D8F865
:10F7400004A899490FF014F9594604A8F1F796FD59
:10F7500004A80FF0CDF804A894490FF009F9594610
:10F7600004A8F1F78BFD04A80FF0C2F804A88E4995
:10F770000FF0FEF8594604A8F1F780FD04A80FF039
:10F78000B7F804A88A490FF0F3F8594604A8F1F72E
:10F7900075FD04A80FF0ACF804A883490FF0E8F851
:10F7A000594604A8F1F76AFD04A80FF0A1F804A8CF
:10F7B00080490FF0DDF8594604A8F1F75FFD04A871
:10F7C0000FF096F804A878490FF0D2F8594604A82B
:10F7D000F1F754FD04A80FF08BF804A876490FF058
:10F7E000C7F8594604A8F1F749FD04A80FF080F8BE
:10F7F00004A86D490FF0BCF8594604A8F1F73EFD86
:10F8000004A80FF075F859465846F1F747F9A8E6ED
:10F81000D8F80010D8F8040098ED027AD6ED006A06
:10F820009FED666ADFF89891DFF86C8101FB00F3C9
:10F8300007EE903AF8EE677AF8EEE66A67EE877AB6
:10F8400007EE102AB8EEC70A86EEA77A67EE067AA8
:10F85000C9ED007AF0F77CFE4E4988ED000A04A855
:10F860000FF086F8594604A8F1F708FD04A80FF038
:10F870003FF82220F1F774FE99ED000A5846F1F79F
:10F8800013FE464904A80FF073F8594604A8F1F78F
:10F89000F5FC04A80FF02CF8414904A80FF068F813
:10F8A000594604A8F1F7EAFC04A80FF021F8222039
:10F8B000F1F756FE98ED000A5846F1F7F5FD374985
:10F8C00004A80FF055F8594604A8F1F7D7FC04A88E
:10F8D0000FF00EF8334904A80FF04AF8594604A86F
:10F8E000F1F7CCFC04A80FF003F82F4904A80FF09F
:10F8F0003FF8594604A8F1F7C1FC04A80EF0F8FF40
:10F900002A4904A80FF034F8594604A8F1F7B6FCC8
:10F9100004A80EF0EDFF244904A80FF029F8594679
:10F9200004A8F1F7ABFC04A80EF0E2FF204904A8FC
:10F930000FF01EF8594604A8F1F7A0FC04A80EF039
:10F94000D7FF194904A80FF013F8594604A8F1F796
:10F9500095FC04A80EF0CCFF174904A80FF008F896
:10F96000594604A8F1F78AFC04A80EF0C1FF0E491D
:10F9700004A80EF0FDFF594604A8F1F77FFC04A887
:10F980000EF0B6FF04A80B49D3E528460121F1F794
:10F9900085F885E4305F02009015FF1F7450020067
:10F9A000405F020074670200604E02008867020038
:10F9B0009C670200C4670200B06702000000B44305
:10F9C0003016FF1F0AD7233C0846F1F767F867E4B3
:10F9D000F968BA6A1FED057A97ED0E0A3E69DFF8FD
:10F9E000AC8002FB01F207EE902AF8EEE77A1846A7
:10F9F00067EE877A4FF0050AFDEEE77A4FF0060BC7
:10FA0000CDED017AF1F754FADDED007AF8EEE77A00
:10FA100027EE800AFDEEC07ACDED007AFFF784BBB9
:10FA20007969FB6A9FED187A97ED0E0ABE69DFF8D7
:10FA30005C8003FB01F307EE903AF8EEE77A10469C
:10FA400067EE877A4FF0140AFDEEE77A4FF0150B58
:10FA5000CDED017AF1F72CFADDED007AF8EEE77AD8
:10FA600027EE800AFDEEC07ACDED007AFFF75CBB91
:10FA700097ED0E0AF1F752F9B9E500934FF0170A26
:10FA80004FF0100BFFF750BB0AD7233CDC17FF1FCA
:10FA90002DE9F04FDFF84893CE4AD9F848302DEDE4
:10FAA000028BDBB00025012B0590156000F0578418
:10FAB000C0F01584022B00F047832C4602952F4698
:10FAC0000495AB462E4641F2883205210DF13008EF
:10FAD0002CA8F8F73DFF0025BF4B2C9302220321F1
:10FAE00040460DF1700A47950AF0DCFF31465A4650
:10FAF00050460AF0D7FFD9F80020D9F810309FED12
:10FB0000B77AB74E03FB02F307EE903AF8EEE77AC6
:10FB1000404667EE877AFDEEE77A17EE901A0BF013
:10FB200003F8D9F820100AF0F3FFD9F84C30002B75
:10FB300000F06383012B40F0CD8396ED0F6A9FEDBB
:10FB4000A97AA94B0393C6EE076A1A460ACB03FBB0
:10FB500001F3B06C07EE103AD2ED027A9DED056A22
:10FB6000326B96ED0E0AB8EE477AB8EEC68A67EEAB
:10FB7000277A520067EEA67A019267EE887AFDEE48
:10FB8000E77A17EE905AF1F793F9336B5B0007EEC3
:10FB9000903AF8EEE77A80EE270A20EE088AFDEE2A
:10FBA000C87A17EE906A3B219048DFF834B20EF025
:10FBB00083F88F480EF010FD0D218E480EF07CF872
:10FBC00029468B480EF058FD89480EF005FD11219D
:10FBD00089480EF071F8894B854819680EF04CFD84
:10FBE00083480EF0F9FC0A2185480EF065F831468D
:10FBF0007F480EF041FD7E480EF0EEFC3B217B4835
:10FC00000EF05AF87A480EF0E7FC029950460AF0D6
:10FC10008BFF21460AF07CFF0E217A480EF04CF84B
:10FC2000D9F8001072480EF027FD71480EF0D4FC90
:10FC3000142175480EF040F8D9F810106C480EF0F9
:10FC40001BFD6B480EF0C8FC0D2170480EF034F817
:10FC500000230A22D9F8201065480EF0CDFC644834
:10FC60000EF0BAFC13216A480EF026F8039C604897
:10FC7000216800230A220EF0BFFC5D480EF0ACFCA8
:10FC8000112164480EF018F800230A2261685848D0
:10FC90000EF0B2FC56480EF09FFC12215E480EF0AA
:10FCA0000BF8A06810F016FD41EC100B0221504833
:10FCB0000EF0EAFC4E480EF08FFCD9F84C30002BC9
:10FCC00000F0D982012B2DD1102154480DF0F4FF02
:10FCD000DBF83C0010F0FEFC41EC100B0221444824
:10FCE0000EF0D2FC42480EF077FC0F214C480DF08C
:10FCF000E3FFDBF8380010F0EDFC41EC100B0221C3
:10FD00003B480EF0C1FC3A480EF066FC0C21454819
:10FD10000DF0D2FFDBF8301035480EF0ADFC344862
:10FD20000EF05AFC0D2133480DF0C6FF294630482D
:10FD30000EF0A2FC2E480EF04FFC0A2130480DF0C8
:10FD4000BBFF31462A480EF097FC29480EF044FCD0
:10FD50000B2135480DF0B0FF029925480EF08CFCC0
:10FD600023480EF039FC112130480DF0A5FF39462B
:10FD70001F480EF081FC1E480EF02EFC0A212C4874
:10FD80000DF09AFF04991A480EF076FC18480EF010
:10FD900023FC01210320F0F781FED9F84810012946
:10FDA00000F02283C0F01B8302290AD108460121FA
:10FDB000F0F774FE23211F480DF07EFF0C480EF073
:10FDC0000BFC019B002B40F3958000271A4CBB468F
:10FDD00034E000BFB812FF1F044B02000AD7233CD7
:10FDE0006414FF1F0000B443DC17FF1FB86102005A
:10FDF000E407FF1FF4610200046202007412FF1F97
:10FE00001862020024620200346202004C620200A6
:10FE10005C6202007062020084620200D86202002A
:10FE2000EC620200FC620200846102009461020044
:10FE3000AC6102000C630200841BFF1FD9F84C3038
:10FE4000002B00F0D881012B00D16D420021A84881
:10FE50000DF032FFA7480EF0BFFB0D21A6480DF0B4
:10FE60002BFF2946A3480EF007FCA2480EF0B4FB76
:10FE70000A21A2480DF020FF31469E480EF0FCFBFF
:10FE80009C480EF0A9FB294640460AF08BFE3146FD
:10FE900050460AF087FE469BCDF818B15AA901EBEF
:10FEA000830103F10C025AA800EB82020B4641F8D1
:10FEB0008C8CB7EE000A43F888AC022142F8B4BC3F
:10FEC0002CA8FAF705FD23680793079A2368069381
:10FED000069B9B1A042BF9D92E9B3BB1F1F7EAFE46
:10FEE000002800F370812E9B002BF7D1019B013776
:10FEF0009F42A3D10399DFED826A48680B6891EDB8
:10FF0000027A1D99D8F804207E4C7F4E7F4D2260E6
:10FF100003FB00F307EE903A06EE102AF8EE677A3C
:10FF2000B8EEC66A67EE877A07EE101AB8EEC70A0F
:10FF300086EE277A2960764D67EE267AC6ED007A3E
:10FF4000F0F706FB08A8734985ED000A0EF010FDD6
:10FF5000002108A8F1F792F908A80EF0C9FC2220A8
:10FF6000F1F7FEFA96ED000A0020F1F79DFA08A8D5
:10FF700069490EF0FDFC08A80021F1F77FF908A8F7
:10FF80000EF0B6FC08A865490EF0F2FC002108A8A6
:10FF9000F1F774F908A80EF0ABFC2220F1F7E0FAB3
:10FFA00095ED000A0020F1F77FFA08A85A490EF0F3
:10FFB000DFFC08A80021F1F761F908A80EF098FC11
:10FFC00008A857490EF0D4FC08A80021F1F756F90B
:10FFD00008A80EF08DFC08A852490EF0C9FC08A82C
:10FFE0000021F1F74BF908A80EF082FC08A84E4951
:10FFF0000EF0BEFC08A80021F1F740F908A80EF0A9
:020000021000EC
:1000000077FC08A847490EF0B3FC08A80021F1F7D7
:1000100035F908A80EF06CFC08A844490EF0A8FCBD
:1000200008A80021F1F72AF908A80EF061FC08A839
:100030003C490EF09DFC08A80021F1F71FF908A823
:100040000EF056FC08A83A490EF092FC08A80021D0
:10005000F1F714F908A80EF04BFC08A831490EF08E
:1000600087FC08A80021F1F709F908A80EF040FC68
:1000700022681D9B2549D8F8045009682D482A4458
:100080002260224A0B44082113600DF015FE2168FE
:1000900018480EF0F1FA17480EF09EFA052126488E
:1000A0000DF00AFE194B134819680EF0E5FA1148D5
:1000B0000EF092FA214B22681A6000210320F0F71B
:1000C000EDFC00210846F0F7E9FC00210120F0F7E3
:1000D000E5FC00210220F0F7E1FC194B2C932CA841
:1000E000F8F780FC5BB0BDEC028BBDE8F08F00BF81
:1000F000B4630200E407FF1FF4610200186202000B
:100100000000B4434017FF1F3016FF1F7412FF1F7B
:100110009015FF1F305F020074500200405F020024
:1001200054630200604E0200686302007C630200B8
:10013000906302009C650200106202006815FF1FB8
:10014000044B02000AD7233CD9F81C70D9F80C30B4
:100150001FED047AD9F82C40A548049403FB07F35B
:1001600007EE903AF8EEE77A0F2167EE877A4FF0C4
:10017000170BFDEEE77A1026CDED027A0DF09CFD0F
:10018000D9F80C109B480EF077FA9A480EF024FA32
:10019000152199480DF090FDD9F81C1095480EF0E6
:1001A0006BFA94480EF018FA0E2194480DF084FD75
:1001B0002B460A22D9F82C108E480EF01DFA8D48D5
:1001C0000EF00AFA7FE48E4B1868F1F763FD8D4B51
:1001D000C0B2532818707FF486AE1A218A480DF0F9
:1001E0006BFD84480EF0F8F92CA8F8F7A3FB874BB9
:1001F00001221A707EE6764228E6736B96ED117A3C
:10020000DFED835A834A03925B0007EE903AF8EEE3
:10021000E77A114687EE275A01930CCA03FB02F3D3
:1002200007EE903AC5EE256A91ED026AB8EE677A5C
:1002300067EE067A9DED057A67EEA67AB8EEC78A74
:1002400067EE887A17EE900A10F044FA41EC100B32
:100250000EF082FF51EC100B10F040FD96ED100AED
:100260000546B06CF0F724FE28EE000AFDEEC07AD9
:1002700017EE906A97E40F2167480DF01DFDDBF83B
:10028000440010F027FA41EC100B022159480EF0FF
:10029000FBF958480EF0A0F91C2160480DF00CFD48
:1002A000DBF8400010F016FA41EC100B0221514827
:1002B0000EF0EAF94F480EF08FF90D2158480DF075
:1002C000FBFCDBF834104B480EF0D6F949480EF031
:1002D00083F927E54F4B019503932E4663E4D9F844
:1002E0001470D9F804309FED4F7AD9F824404E4865
:1002F000049403FB07F307EE903AF8EEE77A0F2138
:1003000067EE877A4FF0050BFDEEE77A0626CDED16
:10031000027A0DF0D1FCD9F8041036480EF0ACF991
:1003200034480EF059F9152140480DF0C5FCD9F8B4
:10033000141030480EF0A0F92E480EF04DF90E21A1
:100340003B480DF0B9FC2B460A22D9F82410294865
:100350000EF052F927480EF03FF9FFF7B4BBD9F879
:100360001870D9F808309FED2F7AD9F82840314815
:10037000049403FB07F307EE903AF8EEE77A0F21B7
:1003800067EE877A4FF0140BFDEEE77A1526CDED78
:10039000027A0DF091FCD9F8081016480EF06CF9AD
:1003A00014480EF019F9152123480DF085FCD9F8F1
:1003B000181010480EF060F90E480EF00DF90E21DD
:1003C0001E480DF079FC2B460A22D9F8281009485E
:1003D0000EF012F907480EF0FFF8FFF774BB012189
:1003E0000020F0F75BFBECE40846F0F757FBE8E48D
:1003F00080610200E407FF1F90610200A861020013
:100400001007FF1FE816FF1F38630200A016FF1F2A
:100410000000B443DC17FF1F98620200A8620200CC
:10042000C86202000AD7233C10610200206102006A
:1004300038610200486102005861020070610200E8
:100440002DE9F04FCC4ECD4AB36C2DED028BDFB0D1
:100450000027012B0590176000F01985C0F0DC849F
:10046000022B00F04B833C4603973D460497BB4666
:10047000BA4610AF41F28832052130A8F8F768FA81
:100480004FF00008BE4B30930222032138460DF195
:100490008009CDF82C810AF005FB51465A464846A2
:1004A0000AF000FB326833699FEDB67ADFF8C8A224
:1004B00003FB02F307EE903AF8EEE77A384667EE70
:1004C000877AFDEEE77A17EE901A0AF02DFB316A73
:1004D0000AF01EFBF36CC7F80480002B00F0FE83CB
:1004E000012B40F06C849AED0F6A9FEDA77AA74B21
:1004F0000293C6EE076A19460CCB03FB02F3DAF847
:100500004800DAF830B00BF1010B07EE103AD1EDEC
:10051000027A9DED056A9AED0E0AB8EE477AB8EEBA
:10052000C68A67EE277A67EEA67A67EE887AFDEECE
:10053000E77A17EE908AF0F7BBFCDAF830305B0010
:1005400007EE903AF8EEE77A4FEA4B0380EE270A7F
:10055000019320EE088AFDEEC87A17EE90BA3B218F
:100560008B48DFF814A20DF0A7FB8A480EF034F890
:100570000D2189480DF0A0FB414686480EF07CF81D
:1005800084480EF029F8112184480DF095FB844B26
:10059000804819680EF070F87E480EF01DF80A21A8
:1005A00080480DF089FB59467A480EF065F8794885
:1005B0000EF012F83B2176480DF07EFB75480EF0E8
:1005C0000BF8039948460AF0AFFA21460AF0A0FA60
:1005D00000240E21744821940DF06EFB31686D48A3
:1005E0000EF04AF86B480DF0F7FF14216F480DF03C
:1005F00063FB316967480EF03FF866480DF0ECFF89
:100600000D216B480DF058FB23460A22316A6148E0
:100610000DF0F2FF5F480DF0DFFF132165480DF08C
:100620004BFB02995B48096823460A220DF0E4FF60
:1006300058480DF0D1FF11215F480DF03DFB2346D6
:10064000029C544861680A220DF0D6FF51480DF013
:10065000C3FF122159480DF02FFBA06810F03AF8A3
:1006600041EC100B02214B480EF00EF849480DF0FA
:10067000B3FFF36C002B00F07383012B2DD11021FD
:100680004F480DF019FBDAF83C0010F023F841EC6C
:10069000100B02213F480DF0F7FF3E480DF09CFF84
:1006A0000F2148480DF008FBDAF8380010F012F876
:1006B00041EC100B022137480DF0E6FF35480DF0F4
:1006C0008BFF0C2140480DF0F7FADAF83010314872
:1006D0000DF0D2FF2F480DF07FFF0D212E480DF0B9
:1006E000EBFA41462B480DF0C7FF2A480DF074FF86
:1006F0000A212C480DF0E0FA594626480DF0BCFFBF
:1007000024480DF069FF0B2130480DF0D5FA03990C
:1007100020480DF0B1FF1F480DF05EFF11212C485D
:100720000DF0CAFA29461B480DF0A6FF19480DF036
:1007300053FF0A2127480DF0BFFA049915480DF020
:100740009BFF14480DF048FF01210320F0F7A6F9A4
:10075000B16C012900F0DB83C0F0D48302293DD1C4
:1007600008460121F0F79AF923211B480DF0A4FA5D
:1007700008480DF031FF31E06414FF1FB812FF1F6D
:10078000044B02000AD7233C0000B443DC17FF1FD0
:10079000B8610200E407FF1FF46102000462020076
:1007A0007412FF1F18620200246202003462020009
:1007B0004C6202005C62020070620200846202000D
:1007C000D8620200EC620200FC6202008461020056
:1007D00094610200AC6102000C630200019B002BDB
:1007E00063DDDFF810A301240321AB480DF064FAA8
:1007F0002146AA480DF040FFA8480DF0EDFE04F098
:1008000001050521A6480DF057FA2946A3480DF029
:1008100033FFA2480DF0E0FEF36C002D40F0C081E4
:10082000002B00F01C82012B38D1C8F100013846A2
:1008300003930AF0B7F94A9A4A955EAB03EB820E2E
:10084000039B4EF88C7C1946B7EE000A30A84EF890
:10085000885CFAF73DF8934A13680993099913687D
:100860000893089B5B1A042BF9D900218E480DF0E0
:1008700023FA8A480DF0B0FE0D218C480DF01CFAC9
:10088000414686480DF0F8FE84480DF0A5FE329BE7
:100890003BB1F1F70FFA002800F36A81329B002B7D
:1008A000F7D1019B01349C429EDD0299DFED806A05
:1008B00048680B6891ED027A21997A687D4C7E4EEA
:1008C0007E4D226003FB00F307EE903A06EE102AFD
:1008D000F8EE677AB8EEC66A67EE877A07EE101A06
:1008E000B8EEC70A86EE277A2960754D67EE267A3C
:1008F000C6ED007AEFF72CFE0CA8724985ED000AD0
:100900000EF036F800210CA8F0F7B8FC0CA80DF09A
:10091000EFFF2220F0F724FE96ED000A0020F0F70A
:10092000C3FD0CA868490EF023F80CA80021F0F7CD
:10093000A5FC0CA80DF0DCFF0CA864490EF018F81B
:1009400000210CA8F0F79AFC0CA80DF0D1FF222092
:10095000F0F706FE95ED000A0020F0F7A5FD0CA8C3
:1009600059490EF005F80CA80021F0F787FC0CA8F7
:100970000DF0BEFF0CA856490DF0FAFF0CA800219F
:10098000F0F77CFC0CA80DF0B3FF0CA851490DF05A
:10099000EFFF0CA80021F0F771FC0CA80DF0A8FFE8
:1009A0000CA84D490DF0E4FF0CA80021F0F766FCFF
:1009B0000CA80DF09DFF0CA846490DF0D9FF0CA81E
:1009C0000021F0F75BFC0CA80DF092FF0CA8434946
:1009D0000DF0CEFF0CA80021F0F750FC0CA80DF094
:1009E00087FF0CA83B490DF0C3FF0CA80021F0F7CE
:1009F00045FC0CA80DF07CFF0CA839490DF0B8FFA0
:100A00000CA80021F0F73AFC0CA80DF071FF0CA81F
:100A100030490DF0ADFF0CA80021F0F72FFC0CA819
:100A20000DF066FF219B7A682260244A2D481360EE
:100A300008210DF041F9216818480DF01DFE1748F6
:100A40000DF0CAFD052128480DF036F91B4B13485F
:100A500019680DF011FE11480DF0BEFD234B226800
:100A60001A6000210320F0F719F800210846F0F77A
:100A700015F800210120F0F711F800210220F0F70D
:100A80000DF81B4B309330A8F7F7ACFF5FB0BDEC0F
:100A9000028BBDE8F08F00BFD8670200E407FF1F9C
:100AA000DC670200841BFF1FB4630200F4610200D4
:100AB0000000B4434017FF1F3016FF1F7412FF1FC2
:100AC0009015FF1F305F020074500200405F02006B
:100AD00054630200604E0200686302007C630200FF
:100AE000906302009C650200106202006815FF1FFF
:100AF000044B0200E816FF1F0AD7233CF569F36890
:100B00001FED037AF46AB148049403FB05F307EE82
:100B1000903AF8EEE77A0F2167EE877A4FF0170BDD
:100B2000FDEEE77A4FF0100ACDED037A0DF0C4F830
:100B3000F168A7480DF0A0FDA5480DF04DFD152169
:100B4000A4480DF0B9F8F169A1480DF095FDA04851
:100B50000DF042FD0E21A0480DF0AEF83B460A22F2
:100B6000F16A9B480DF048FD99480DF035FD80E491
:100B70009A4B1868F1F78EF8C0B253288AF8000033
:100B80007FF48CAE1A2196480DF096F890480DF03F
:100B900023FD30A8F7F7CEFE924B01221A7084E6AF
:100BA0000BB1012B07D14146384609F0FBFF5946EE
:100BB000484609F0F7FF00218B480DF07DF8844886
:100BC0000DF00AFD0D2189480DF076F84146804868
:100BD0000DF052FD7E480DF0FFFC0A2184480DF017
:100BE0006BF859467A480DF047FD79480DF0F4FC52
:100BF0004A9B5EA901EB830103F10C025EA800EBA6
:100C000082020B464FF0000E41F88C7CB7EE000AD2
:100C100043F8889C022142F8B4EC30A8CDF828E1D2
:100C2000F9F756FE734A13680B930B9913680A93EE
:100C30000A9B5B1A042BF9D910216F480DF03CF880
:100C4000214663480DF018FD61480DF0C5FC2946AA
:100C50005F480DF011FD5E480DF0BEFC1EE6CBF1C5
:100C600000014846039309F09DFF4A9A039B4A936B
:100C70005EA901EB8200024640F88C9C012142F8FB
:100C8000883CB7EE000A30A8F9F722FE594A1368EB
:100C90000793079913680693069B5B1A042BF9D9EF
:100CA000082156480DF008F8214649480DF0E4FCAB
:100CB00047480DF091FC002145480DF0DDFC44480B
:100CC0000DF08AFC0A214A480CF0F6FF59464048CC
:100CD0000DF0D2FC3E480DF07FFCDFE5DAF8342061
:100CE0009AED117ADFED465A464B0293520007EE19
:100CF000902AF8EEE77A184687EE275A0ACB03FBCC
:100D000001F307EE903AC5EE256A931C019390ED2E
:100D1000026AB8EE677A67EE067A9DED057A67EEAD
:100D2000A67AB8EEC78A67EE887A17EE900A0FF0B7
:100D3000D1FC41EC100B0EF00FFA51EC100B0FF040
:100D4000CDFF9AED100A8046DAF84800F0F7B0F8C7
:100D500028EE000AFDEEC07A17EE90BAFFF7FFBB4F
:100D60000F2129480CF0A8FFDAF844000FF0B2FC7C
:100D700041EC100B022116480DF086FC14480DF0D2
:100D80002BFC1C2121480CF097FFDAF840000FF0F3
:100D9000A1FC41EC100B02210D480DF075FC0C4834
:100DA0000DF01AFC0D211A480CF086FFDAF8341009
:100DB00007480DF061FC06480DF00EFC8DE4114B68
:100DC00002930223C3460193FFF7C9BB806102006F
:100DD000E407FF1F90610200A86102001007FF1FD7
:100DE00038630200A016FF1FB4630200F461020022
:100DF00018620200841BFF1FE4670200EC67020018
:100E00000000B443DC17FF1F98620200A8620200D2
:100E1000C86202000AD7233C756973681FED037A24
:100E2000746A3D48049403FB05F307EE903AF8EE2C
:100E3000E77A0F2167EE877A4FF0050BFDEEE77A30
:100E40004FF0060ACDED037A0CF036FF7168334897
:100E50000DF012FC31480DF0BFFB152130480CF0AD
:100E60002BFF71692D480DF007FC2C480DF0B4FBE9
:100E70000E212C480CF020FF3B460A22716A2748BD
:100E80000DF0BAFB25480DF0A7FBFFF7F2BAB569E4
:100E9000B3689FED257AB46A2448049403FB05F3F4
:100EA00007EE903AF8EEE77A0F2167EE877A4FF077
:100EB000140BFDEEE77A4FF0150ACDED037A0CF036
:100EC000FBFEB16815480DF0D7FB14480DF084FB0C
:100ED000152117480CF0F0FEB16910480DF0CCFB5D
:100EE0000E480DF079FB0E2112480CF0E5FE3B4652
:100EF0000A22B16A09480DF07FFB08480DF06CFB2F
:100F0000FFF7B7BA01210020EFF7C8FD66E40846F5
:100F1000EFF7C4FD62E400BF10610200E407FF1FA9
:100F200020610200386102000AD7233C48610200B8
:100F300058610200706102002DE9F04FD44C2DED94
:100F4000088B2168D4ED107AD4ED0CBAD4F8509007
:100F50000129C1B0B0EE409AF0EE60AAB0EE418A2D
:100F6000B0EE61AAF8EEE78A00F08481C0F07381E8
:100F7000022900F026814FF0000ADFEDC69A55469F
:100F80004FF0050B062429461BEE900AEFF7C8FF29
:100F900001210320EFF782FD02AF41F288320521E3
:100FA00012A8F7F7D5FC4FF000085A462146BA4E72
:100FB0009FEDBABA12963846CDF8B48009F072FDAA
:100FC00007EE905A69EE8B9AF8EEE77A384669EEAA
:100FD000A77AB34DB34CFDEEE77A17EE901A09F0FD
:100FE000A3FD514609F094FDFDEEC97ACDF80C80C1
:100FF00017EE903A002BB8BF5B4207EE903AF8EE3E
:10100000E77A67EEAA7A17EE900A0FF063FB41ECDD
:10101000100B0EF0A1F851EC100B0FF05FFE014623
:101020008246384609F0BEFD68EE8B8AF8EEEB7A10
:10103000284668EEA77AFDEEE77A17EE901A09F0D7
:1010400073FD494609F064FDFDEEC87AC5F80480D9
:1010500017EE903A002BB8BF5B4207EE903AF8EEDD
:10106000E77A67EE8A7A17EE900A0FF033FB41ECCD
:10107000100B41EC180B0EF06FF851EC100B0FF049
:101080002DFE01468146284609F08CFD2821864820
:101090000CF012FE85480DF09FFA0D2184480CF0EB
:1010A0000BFEB0EE480AF0EE680A02217F480DF010
:1010B000EBFA7E480DF090FA14217E480CF0FCFD0E
:1010C00049467A480DF0D8FA78480DF085FA112192
:1010D00079480CF0F1FD514674480DF0CDFA734893
:1010E0000DF07AFA2C9BCDF8B08040A903F10C02E8
:1010F00001EB830E01EB820212A84EF88C5C4EF8D5
:10110000887CB7EE000A022142F8B48CF9F7E0FBC4
:10111000149880B1F0F704FE002840F08480236822
:101120000193019A23680093009B9B1A042BF9D921
:1011300014980028EED1044600210320EFF7AEFCFE
:1011400000210846EFF7AAFC5C4FDFF88C810021F4
:101150000120EFF7A3FC112159480CF0ADFD3968CF
:1011600052480DF089FA51480DF036FA0398D8F834
:1011700000103A686B6802440B4451483A601121F0
:10118000C8F800300CF098FD396848480DF074FA42
:1011900046480DF021FA14214A480CF08DFDD8F88C
:1011A000001042480DF068FA40480DF015FA12A8F8
:1011B0001296F7F717FC204641B0BDEC088BBDE84E
:1011C000F08F08460121EFF769FCD4ED137A3E4811
:1011D000E56BD4F85CA00721F8EEE79A0CF06CFD03
:1011E000E16B32480DF048FA30480DF0F5F9062170
:1011F00036480CF061FD00230A22E16D2B480DF00A
:10120000FBF92A480DF0E8F90D2131480CF054FDA6
:10121000E16C26480DF030FA24480DF0DDF94FF06E
:10122000170B1024AFE617212A480CF045FD1F4884
:101230000DF0D2F912A8F7F77DFB00210320EFF79C
:101240002DFC00210846EFF729FC00210120EFF7D3
:1012500025FC012470E701210020EFF71FFCD4EDED
:10126000119A656BD4F854A0F8EEE99A4FF0050B8B
:10127000062488E60846EFF711FCD4ED129AA56B18
:10128000D4F858A0F8EEE99A4FF0140B15247AE63A
:10129000F813FF1F00000000044B02000AD7233C94
:1012A0007812FF1F841BFF1FF8670200E407FF1F6F
:1012B000F4610200246802003C6802007412FF1FFF
:1012C000046202009065020088610200B0610200C1
:1012D00098610200D86402004017FF1F2DE9F04F0B
:1012E000B54BDFF814B31A68DBF8001091FBF2F38A
:1012F000FFB002FB1319074641F28832052150A8BE
:10130000F7F726FB002502220321DFF8F0A2CDF833
:1013100040A110A86B9509F0C5FB0522062120A865
:1013200009F0C0FB1422152130A809F0BBFBA34C27
:10133000172240A8102109F0B5FB119523680193ED
:10134000019AC9F1000923680093009B9B1A0E2B98
:10135000F9D99B4D9B4E696DDFF8A48210A809F066
:10136000E3FBA96D09F0D4FB494609F01BFC1D21E4
:1013700095480CF0A1FC95480DF02EF910219448E9
:101380000CF09AFC494691480DF076F98F480DF023
:1013900023F918218F480CF08FFC31688B480DF031
:1013A0006BF98A480DF018F912218B480CF084FC77
:1013B000D8F8001085480DF05FF984480DF00CF95D
:1013C00001210320EFF76AFB032F00F23A87DFE8E1
:1013D00017F01B01A7005C0004006A9BDFF8249251
:1013E0007EA903F10B0201EB830301EB820210A93A
:1013F00043F88C1C0023B7EE000A42F8B43C0121EC
:1014000050A86A93F9F764FA529B744E744DF3B185
:1014100021996E480DF030F96C480DF0DDF8F0F7C9
:1014200049FC002807DB3068F0F734FCC0B25328D1
:10143000287000F03D8123680993099A2368089376
:10144000089B9B1A092BF9D9529B002BE0D1654EC2
:10145000119B3360012F00F0B782022F00F0B082A1
:10146000002F00F08B82D9F800300A2B00F2BE81E9
:10147000DFE813F0FA01BC01FD0393030905C4047E
:1014800059056104F60222014E03D8F80030419359
:1014900023680793079A23680693069B9B1A132BCE
:1014A000F9D90C215048DFF85C910CF005FC41990A
:1014B00046480DF0E1F845480DF08EF8E96E40A879
:1014C00009F032FB296F09F023FB316809F050FB6A
:1014D000162146480CF0F0FB00230A22296F3B48F6
:1014E0000DF08AF839480DF077F801210220EFF766
:1014F000D5FAD9F800206A9B002A40F08A827EA99A
:1015000001EB8300034640AD40F88C5CB7EE000A67
:10151000012150A843F8882C6A92F9F7D9F973E7AA
:10152000D8F80030319323680593059A2368049313
:10153000049B9B1A132BF9D90C212D48DFF8C4907A
:101540000CF0BAFB319921480DF096F81F480DF0C8
:1015500043F8696E30A809F0E7FAA96E09F0D8FAE5
:10156000316809F005FB162122480CF0A5FB002389
:101570000A22A96E15480DF03FF814480DF02CF81A
:1015800001210846EFF78AFAD9F800206A9B002A61
:1015900040F059827EA901EB8300034630AD40F84C
:1015A0008C5CB7EE000A012150A843F8882C6A929F
:1015B000F9F78EF928E700BFCC18FF1F841BFF1F27
:1015C000DC17FF1FB812FF1F50680200E407FF1F5F
:1015D0007068020084680200A06802001007FF1F04
:1015E000E816FF1F4017FF1F04690200146902007C
:1015F000DC680200EC6802006815FF1F044B020063
:101600007412FF1F4C07FF1FD8F800302193236886
:101610000393039A23680293029B9B1A132BF9D915
:101620000C218648DFF83C920CF046FB2199844857
:101630000DF022F882480CF0CFFFE96D20A809F0E8
:1016400073FA296E09F064FA316809F091FA1621EB
:101650007C480CF031FB00230A22296E78480CF0FC
:10166000CBFF77480CF0B8FF01210020EFF716FA06
:10167000D9F800206A9B002A00F0BA817EA903F104
:101680000C027EA801EB830100EB82020B46B7EE51
:10169000000A20A841F88C0C002510A943F8881CEA
:1016A00050A8022142F8B45C6A95F9F711F9ABE64B
:1016B00050A8F7F73FF9BEE663490CA80DF058F9BA
:1016C00000210CA8EFF7DAFD0CA80DF011F95F4925
:1016D0000CA80DF04DF900210CA8EFF7CFFD0CA8D8
:1016E0000DF006F958490CA80DF042F900210CA89C
:1016F000EFF7C4FD0CA80DF0FBF854490CA80DF051
:1017000037F900210CA8EFF7B9FD0CA80DF0F0F89F
:101710004F490CA80DF02CF900210CA8EFF7AEFDF5
:101720000CA80DF0E5F849490CA80DF021F90021AD
:101730000CA8EFF7A3FD0CA80DF0DAF845490CA8AA
:101740000DF016F900210CA8EFF798FD0CA80DF08C
:10175000CFF83E490CA80DF00BF900210CA8EFF7CB
:101760008DFD0CA80DF0C4F83B490CA80DF000F954
:1017700000210CA8EFF782FD0CA80DF0B9F822208B
:10178000EFF7EEFED6ED007A0020B8EEE70AEFF7AD
:101790008BFE32490CA80DF0EBF800210CA8EFF7F6
:1017A0006DFD0CA80DF0A4F82D490CA80DF0E0F883
:1017B00000210CA8EFF762FD0CA80DF099F822208B
:1017C000EFF7CEFED8ED007A0020B8EEE70AEFF78B
:1017D0006BFE22490CA80DF0CBF80CA80021EFF706
:1017E0004DFD0CA80DF084F8D9F80030002B40F026
:1017F000BA80032F09D8DFE817F0F0000400EB00EF
:10180000F50000233193C8F8003000210320EFF7E2
:1018100045F900210846EFF741F900210120EFF7D3
:101820003DF900210220EFF739F950A8CDF840A189
:10183000F7F7D8F87FB0BDE8F08F00BFB4680200BA
:10184000E407FF1FC4680200406B0200604E020004
:10185000586B0200706B0200305F0200745002008F
:10186000405F02004C07FF1F032F40F0A2839F49F7
:101870000CA80DF07DF800210CA8EFF7FFFC0CA8D8
:101880000DF036F89A490CA80DF072F800210CA85A
:10189000EFF7F4FC0CA80DF02BF894490CA80DF010
:1018A00067F800210CA8EFF7E9FC0CA80DF020F870
:1018B0008F490CA80DF05CF800210CA8EFF7DEFCB6
:1018C0000CA80DF015F88B490CA80DF051F800216B
:1018D0000CA8EFF7D3FC0CA80DF00AF884490CA86B
:1018E0000DF046F800210CA8EFF7C8FC0CA80CF08E
:1018F000FFFF81490CA80DF03BF800210CA8EFF781
:10190000BDFC0CA80CF0F4FF79490CA80DF030F8E0
:1019100000210CA8EFF7B2FC0CA80CF0E9FF774906
:101920000CA80DF025F800210CA8EFF7A7FC0CA8D7
:101930000CF0DEFF2220EFF713FED6ED007A002038
:10194000B8EEE70AEFF7B0FD6D490CA80DF010F8FE
:101950000CA80021EFF792FC0CA80CF0C9FFD9F8F5
:101960000030002B3ED000231193C8F80030319393
:1019700033602193CBF80030419346E7219BC8F8B0
:101980000030D9F800300A2B3FF630AF01A252F8F0
:1019900023F000BFB31F0100ED1701006F1C010011
:1019A0009B1B0100871E0100FD1D0100271F010078
:1019B000371D0100611A0100B9160100111B010059
:1019C000419BC8F80030DCE7319BC8F80030D8E70D
:1019D00000234193C8F8003017E700232193C8F88B
:1019E000003012E7002311933360CBF800300CE78E
:1019F0007EA901EB8300034620AD40F88C5CB7EE76
:101A0000000A012150A843F8882C6A92F8F760FF79
:101A1000FAE47EA901EB83017EA803F10C0200EB3E
:101A200082020B4640A841F88C0C002510A843F810
:101A3000880CB7EE000A022150A842F8B45C6A95FF
:101A4000F8F746FFE0E47EA903F10C027EA801EB63
:101A5000830100EB82020B46B7EE000A30A819E6BC
:101A600028490CA80CF084FF00210CA8EFF706FC15
:101A70000CA80CF03DFF1E490CA80CF079FF0021CA
:101A80000CA8EFF7FBFB0CA80CF032FF1D490CA8CB
:101A90000CF06EFF00210CA8EFF7F0FB0CA80CF087
:101AA00027FF13490CA80CF063FF00210CA8EFF7E7
:101AB000E5FB0CA80CF01CFF13490CA80CF058FF18
:101AC00000210CA8EFF7DAFB0CA80CF011FF084975
:101AD0000CA80CF04DFF00210CA8EFF7CFFB0CA8D1
:101AE0000CF006FF0CA809492AE600BF2C69020089
:101AF000604E02004069020054690200305F02003B
:101B0000745002008C4E02004C4E02002C6B0200FE
:101B1000AB490CA80CF02CFF00210CA8EFF7AEFB92
:101B20000CA80CF0E5FEA7490CA80CF021FF002141
:101B30000CA8EFF7A3FB0CA80CF0DAFEA0490CA848
:101B40000CF016FF00210CA8EFF798FB0CA80CF086
:101B5000CFFE9C490CA80CF00BFF00210CA8EFF75E
:101B60008DFB0CA80CF0C4FE97490CA80CF000FFEC
:101B700000210CA8EFF782FB0CA80CF0B9FE9149EC
:101B80000CA80CF0F5FE00210CA8EFF777FB0CA8D1
:101B90000CF0AEFE0CA88D49D2E58D490CA80CF0D6
:101BA000E7FE00210CA8EFF769FB0CA80CF0A0FEE3
:101BB00084490CA80CF0DCFE00210CA8EFF75EFBBA
:101BC0000CA80CF095FE82490CA80CF0D1FE002167
:101BD0000CA8EFF753FB0CA80CF08AFE79490CA86F
:101BE0000CF0C6FE00210CA8EFF748FB0CA80CF087
:101BF0007FFE78490CA80CF0BBFE00210CA8EFF783
:101C00003DFB0CA80CF074FE6E490CA80CF0B0FE65
